:10400000008000108D100400C1100400F3E50300CF
:10401000F7E50300FBE50300FFE5030000000000F7
:10402000000000000000000000000000CB100400B1
:1040300003E6030000000000F5BA0000D110040000
:10404000ADA50000A5BA0000A5B7000011B00000A2
:10405000DD10040007E603000BE603000FE6030093
:1040600013E60300E7100400E9100400EB1004005D
:10407000ED100400EF100400F1100400F310040030
:10408000F5100400F7100400F9100400FB10040000
:10409000FD100400FF1004000111040003110400CE
:1040A0005164010007110400091104000B11040000
:1040B000B15201000F11040011110400131104008A
:1040C00015110400171104001911040010B5054C56
:1040D000237833B9044B13B10448AFF300800123B4
:1040E000237010BD580200100000000004D105002C
:1040F00008B5064B1BB106480649AFF300800648D9
:10410000036813B1054B03B1984708BD00000000D8
:1041100004D105005C0200105802001000000000ED
:10412000024B1A6801321A60704700BF7402001017
:10413000014B1868704700BF74020010F8B51E4E9E
:10414000012303704370B36900251C491C4A837026
:10415000C570044613680868E36060602574657480
:10416000A574E57425756575A575E575257665767F
:10417000A576E57680277169B2692581678104F1AA
:104180001C0043F070FBB2692946A0181C30C2F134
:10419000100243F08CFB2946402204F12C0043F02E
:1041A00086FB29463A4604F16C0043F080FB054B40
:1041B0001868C4F8EC00F8BD00000820CC0000101E
:1041C000880A001060C704002DE9F041214E82B03A
:1041D00034684FF035082046FFF7B0FF1E4B4FF014
:1041E000010C186ADD69C4F8F500986A03270423F6
:1041F0003621322284F8F08084F8F1C084F8F2701D
:1042000084F8F31084F8F920C4F8FB0084F8F43043
:1042100084F8FA30E5B1284643F013FF04F20113A5
:10422000C7B24FF00C0E84F8000184F8FFE0294675
:104230003A46184643F017FBC4192146FF2301F8FC
:10424000013B3068091A02B0BDE8F04101F034BD0D
:10425000FF34F2E7840A00100000082070B51C4DFE
:104260002C682046FFF76AFF1A4B3520DA693721A0
:10427000012384F8F00084F8F31084F8F13084F816
:10428000F230C2B10426032006210C2284F8F53056
:1042900084F8F46084F8F60084F8F71084F8F820C5
:1042A000F9342146FF2301F8013B2868BDE870403E
:1042B000091A01F001BD0322062184F8F53084F8C3
:1042C000F42084F8F62084F8F710F834E9E700BF0A
:1042D000840A0010000008202DE9F0412F4B1C68D3
:1042E0002378022B02D00020BDE8F081201D2C494C
:1042F000042243F0A9FA06460028F4D1294D04F11E
:104300001C00AA69696943F09FFA024610B1304661
:10431000BDE8F081244904F1F003098820691944BB
:104320008B42A862144623D205F1240805F1200C23
:1043300005F1340705F130062C350DE0032A28D0AD
:10434000062A22D0012A02D1D3F8020028605A7826
:104350000232134499420BD91A78332A10D0EDD97E
:10436000362A08D0FF2A03D0352AF0D19C78EEE710
:104370002046BDE8F081D3F80200CCF80000E6E763
:10438000D3F80200C8F80000E1E7D3F8020030607B
:10439000DDE7D3F802003860D9E700BF840A0010D7
:1043A000CC000010000008209E0A001030B50D4C13
:1043B00083B04FF6FF736061A161002501A84FF43F
:1043C0008641E261A570ADF80430ADF8063000F02A
:1043D00007FD606010B14FF4884383800023238081
:1043E00003B030BD0000082070B57F4C2388B3F5C2
:1043F0009A7F00F0BC802FD940F24D12934200F01A
:10440000A480B3F5A77F5BD340F25912934209D041
:10441000B3F5B57F28D17548218A01F0D3FC40F26D
:1044200059132380724B1B789B0705D46F4801F00A
:10443000D7FC002800F0C2806B4D05F1080001F0A8
:10444000CFFC002800F0BC802B8AB3F57A7F40F2C5
:10445000BF8000232B8070BDB3F58E7F12D0B3F5E3
:10446000957F04D0002B77D00023238070BDA378E4
:10447000022B00F0B2805D48218A01F0A3FC4FF4CA
:104480008E7323805A4D2B789E0713D5564E06F116
:10449000080001F0A5FC00286BD0338A41F26F724E
:1044A00093429CBF5B003382FFF7D8FE4FF49573B5
:1044B000238070BD4D4801F093FC0028E6D170BD0B
:1044C00040F243129342CFD1A378032B25D0484D1D
:1044D0004648218A01F076FC4FF49A7323802B78AA
:1044E000990704D4414801F07BFC002867D03E4E78
:1044F00006F1080001F074FC30B1338AB3F57A7F1D
:1045000048D90023338070BD2B789A0746D5FFF732
:10451000E3FE052842D10323B37033480FF08AFC31
:10452000606A00BA3EF084FE0022324B3EF0F6FE96
:10453000314B00223EF0F2FE3FF0B2F901462B482B
:1045400001F040FC40F24D132380274D05F1080097
:1045500001F046FC30BB70BD284B01201A68642175
:1045600002441A60A0702182FFF778FE83E7204D95
:10457000B5E72B78980799D5FFF7AEFE022895D1BD
:10458000B0701E4B64211A68218201321A60FFF755
:104590001BFE9DE764333382FFF716FE40F24313A0
:1045A000238070BD16480FF0CFFB144B64211A68AE
:1045B000298201321A60FFF707FE2CE770BD70BD3B
:1045C000FFF78AFE05280AD04FF4B573238070BD2B
:1045D00064332B82FFF7F8FDF6E7054DD1E7094874
:1045E0000FF0B2FB9CE700BF000008200800082085
:1045F0009C0A00100000E03F00005940CC00001071
:1046000064C7040078C70400034B9B7813B9034ABE
:1046100013805380704700BF00000820880A0010F4
:104620002DE9F0073B4B3C4EB3F81CC0B3F81E809D
:104630003A4D33460122002705E0092903F10C0316
:1046400017D017460A461888511CC9B20028F4D062
:104650005C88002CF1D06045EFD14445EDD1304A63
:10466000304C1068918822782F70586019819A72A6
:1046700024E0294B0122002701E017460A4618884A
:10468000511CC9B21C4610B9588800283CD00929D1
:1046900003F10C03F1D1082A2A70224B11D093F8B0
:1046A00000C0214923460A4652F8060D096892883F
:1046B00043F8041B60609A8084F80AC0BDE8F007E4
:1046C00070470027DFF864A0DFF86490124A93F87F
:1046D00000C0B8463B46917ADCB2C1EB0C01B9424E
:1046E00003F10103C4BFA046CFB2082B02F10C02B4
:1046F000F1D108EB48048AF8007089F8008085F849
:10470000008006EB8404CCE7064B2F7093F800C0C2
:10471000C7E700BF98000820380008207802001082
:10472000AE0008207B020010B400082079020010BF
:104730007A020010F0B4154A154D1678154B013663
:10474000F6B216700027012205E02A70CAB2092AC3
:1047500003F10C0318D05C881888511C204380B2E8
:104760000028F2D0987A301A7728EEDD184600F843
:10477000017B01302A70CAB25F70092A00F8017B00
:10478000077003F10C03E6D1F0BC70477B02001008
:1047900078020010380008202DE9F84F304C2388AB
:1047A000292B12D92F4D0026AB8A2680B3F5807FA6
:1047B00004D0B3F5007F0CD0BDE8F88F2A4FEA8C07
:1047C0003B889A4212D0BDE8F88F00232380BDE8D1
:1047D000F88F254BE98C1A889142F4D12A8D5B8899
:1047E0009A42F0D1BDE8F84FFFF71ABF2A8D7B88B7
:1047F0009A42E8D1FFF714FF022329466B7551F85E
:10480000168F1A4BB1F804C01A689B88C5F820802F
:10481000A5F824C0C5F81620B5F824B08B80D5F8CB
:1048200020A0B5F81C90B5F81E80B7F800C07F88AE
:10483000082006216B81C5F806204FF02A03A5F851
:1048400004B0C5F800A02E75A5F82690A5F828801C
:10485000A5F81CC0EF83287369732380BDE8F88F27
:104860009E0A001098000820880A00108C02001090
:104870002DE9F84F504E4FF6FF73F28B95B29D42E3
:104880004FD0DFF858814D4BB8F8000019886840C8
:1048900008423BD04A4B4B4F1D885B883D807B8054
:1048A000DFF83CA1B7F80290474B01244FF0000C11
:1048B00005E0092A03F10C030DD0A446144619881B
:1048C000621CA942D2B21846F3D159884945F0D1A9
:1048D0008AF800C003E0082C8AF800402AD003467A
:1048E00053F8040F9B883060B380384A384B156802
:1048F0001F88948837480E3700210822C6F80650D2
:1049000084801F8071733273BDE8F88F318CB8F8E2
:1049100002005B8848401842BCD12A4F3A80798017
:10492000BEE7338CAB42ACD12B4B18689B88306010
:10493000B380DAE7FF2106221F4842F0B8FF234B7D
:10494000244A798898881F68B8F80090002302F1FB
:10495000300B3473DFF88CA0B8F80280F58434741F
:1049600006250424C6F80670C6F81670908090825A
:10497000174A4FF02A0C318586F82030012186F83D
:10498000213086F8223086F8233086F8243086F8E5
:104990002530B574F474CAF800B0A6F81C90A6F8D7
:1049A0001E80A2F800C03375B37373747175F17310
:1049B0007573BDE8F88F00BF98000820800A0010CA
:1049C000900A00107C020010380008208C020010B1
:1049D0009E0A00109E0008208CC70400880A001060
:1049E00078020010840A001010B590F820300446B8
:1049F000062B0ED00B4A238A12686068518A8B42BC
:104A000098BF194601F058F9062384F82030012098
:104A100010BD054B1B7803F0040303F0FF00002BCF
:104A2000E8D110BD7C0A00109C0A001090F82030DC
:104A3000062B01D000207047104B1B7813F00103A8
:104A400019D00F4A038A1268528A934209D84268E1
:104A50000021134443600123018280F8203018466E
:104A6000704741689B1A03820A440123426080F820
:104A70002030184670471846704700BF9C0A001047
:104A80007C0A0010024B1878C0F34000704700BF4A
:104A90009C0A001038B543880446A3B1D52B0ED12B
:104AA0002046FFF7C3FF05462046FFF79DFF28403D
:104AB00010F0FF0006D0228A6AB984F82020002373
:104AC0006380022038BD4AB192B20282416080F810
:104AD0002030002AF1D0D5236380E1E74280012015
:104AE00038BD00BFF8B5458804460E4617462DB1BF
:104AF000F42D14D0002363800220F8BD01B31046CA
:104B00008847114B20821B6884F8205063600F4B4C
:104B10001B785B0701D53846B047F42363802046F5
:104B2000FFF784FF05462046FFF75EFF284010F0A0
:104B3000FF00E2D0238A002BE9D184F82030D9E7A6
:104B400061800120F8BD00BF840A00109C0A00109B
:104B5000C269038BD01A80B2704700BF70B543881A
:104B600082B00446002B2FD040F22112934226D16E
:104B7000438A002B32D02B4A2B4B12681B88022011
:104B8000A260638284F82000228B002A37D013B3FE
:104B9000A268636910781870638A228BA6686569B9
:104BA000013B013A9BB292B20136013581426382E8
:104BB0002283A6606561E8D1A38B93422DD00023A8
:104BC0006380022002B070BD808BE268638A20831C
:104BD0006261002BD8D140F22113638094F8203019
:104BE000022B06D00191FFF74DFF01990028E9D073
:104BF000C1E70323002084F8203002B070BD002BF1
:104C0000E9D0A06810F8015B013B9BB2A942638226
:104C1000A060D1D0002BF5D1DDE7002084F8200082
:104C20006080CFE7840A00109E0A00100023C16054
:104C30004161C261028380F8203043820380438057
:104C4000704700BF013A30B48D18A94214D20B4608
:104C50001C785A78023302EB042292B2104480B2DC
:104C6000824284BF013080B29D42F1D8CB432B44B5
:104C700023F0010302331944A94201D030BC70472C
:104C80000B7830BC1B02184480B2834284BF0130D1
:104C900080B2704738B50E4C0822637C257C04F145
:104CA0001A0103EB0525ADB2A5F10E0080B2FFF7A6
:104CB000C9FFA5F1140292B204F12201FFF7C2FF6D
:104CC00010B94FF6FF7038BD40BA80B238BD00BF92
:104CD0009800082070B4C478134B0C44E4B2DC7024
:104CE00082780D0A2A44D2B29A70467895425E7054
:104CF0000078187003D90136F6B25E708EB1C9B271
:104D00008C420CDA0132D2B29A70074B3AB95A7817
:104D10000132D2B25A7012B91A7801321A7070BCCC
:104D2000704701301870EAE7980A001010B5084C77
:104D3000014620680830FFF7CDFF064A2368507807
:104D400014789178D2781C7258729972DA7210BD08
:104D50007C0A0010980A001008B5002005491422AA
:104D6000FFF770FF10B94FF6FF7008BD40BA80B270
:104D700008BD00BFA6000820FFF78CBF30B4154B5C
:104D800015490022154C04204FF4806583F8B921A1
:104D900083F8D92183F8F92183F8192283F839227D
:104DA00083F8592208702580A3F89421A3F896214E
:104DB000A3F89821A3F89A21A3F89C21A3F89E2197
:104DC000A3F86422A3F8A822A3F8EC22A3F83023C6
:104DD00030BC704798000820940200108802001030
:104DE0002DE9F0012A4C2B4EB4F864523288B4F805
:104DF000A872B4F8ECC2B4F83083013292B2B2F5C2
:104E0000FA4F1ED34FF480521023AB42F5D0BB4271
:104E1000F3D06345F1D04345EFD032801E4A0426DB
:104E200095B1B4F8A8520127194C45B3B4F8EC5227
:104E30000DB3B4F8304334B316700020BDE8F00170
:104E4000704753BA9BB2E0E715702C4604EB04148C
:104E5000124EA4003219F0D09380D18048B103885B
:104E6000335343885380402313721046BDE8F0014A
:104E700070473051F7E7022425461570E6E73D46B6
:104E80003C461570E2E7032425461570DEE700BFB7
:104E9000980008208802001094020010F8020820F0
:104EA000DFF850C02DE9F001DFF84C80BCF89461C8
:104EB000002388F80030AEB101231F460CF5CA71FB
:104EC00000E02F4631F8024F5A1C1E46D5B2134659
:104ED00034B1062AF5D188F80050BDE8F0017047DA
:104EE00088F800700CEB4606A6F89401BDE8F001C6
:104EF000704700BF98000820940200102DE9F04F81
:104F0000BC4D042887B02B6821D0DFF80CB3BA4E13
:104F1000BA4F0BF13602032832603A6070D0022893
:104F200000F0E680052800F087819BF80E30452BC5
:104F300000F02981B2480EF007FFDFF8EC82B14C97
:104F40000023238088F8003007B0BDE8F08FDFF839
:104F5000D882AC4CAC4A1388002BF1D003F11C0171
:104F6000AA4ADFF8B4B289B21268080A8BF81000B6
:104F70008BF81110167A08335BBA11250020ABF8B4
:104F800026308BF816608BF81750ABF82800908805
:104F90009F4BABF82200D58818885B88ABF824506B
:104FA000ABF81C30ABF81A001088934BABF81E001E
:104FB00050880BF136022180ABF820001A60954929
:104FC00000230A884520013292B2140A8BF813207C
:104FD0008BF812408BF80E008BF80F308BF81530E1
:104FE0008BF81430ABF818300A80FFF7B5FEC043D9
:104FF000ABF81800002388F8003007B0BDE8F08F48
:105000005A7E02F00F02032A97D11A8ADFF818821B
:10501000002A94D1082288F800207A4C01930EF0DF
:10502000F7FF794A019B98F8000000F0200101F099
:10503000FF05002900F08F8100211420DFF8D091B6
:10504000597611808BF82F002822228050228BF86D
:105050002E201A7A06268BF82A205A7AB9F80210DE
:105060008BF82B209A7AB9F800508BF82C20D87A3C
:10507000694A8BF82D00187B8BF82600587B8BF83B
:105080002700987B8BF82800D87B8BF817608BF86B
:1050900029009888ABF82200D888ABF81A50ABF8F2
:1050A0002400ABF81C101988ABF81E105988ABF817
:1050B00020105B7EDB0640F14781002382F831300F
:1050C00082F83030228800234021100A8BF811200A
:1050D0008BF810008BF816108BF835308BF83430C5
:1050E000ABF83230FFF7D6FDC043ABF8320066E7CD
:1050F0004A4AD1780131C9B2D17061B99178013190
:10510000C9B2917039B951780131C9B2517011B930
:10511000117801311170587E3A4C3B4A00F0FD0580
:105120000021052D2180118000F0A08000285ED094
:10513000198A002900F0F780997E4D1E9D7600297E
:1051400055D1D97E082900F0A281451E012D40F2DB
:105150009B8104299CBF4FF0030C0CFA01FC00F06A
:105160000F0094BF5FFA8CFC4FF0300C0131451EEC
:10517000D97683F81AC0072D39D8DFE805F089A35E
:10518000A681388138811F4C9BF810A09BF8112014
:10519000238802EB0A2A9A4526DC9BF814301FFA72
:1051A0008AFA9906A4F800A040D19BF81530002B8C
:1051B0003CD1DFF85C90B9F80030002B40F0A280C1
:1051C000B9F80220002A40F09D800193FFF7C4FD4A
:1051D0004FF6FF718842019B00F0208110480EF0CD
:1051E000B3FDDFF84480ABE60E480EF0ADFDDFF80E
:1051F0003880A5E67C0A0010840A0010940A00108A
:1052000094C704009E0A00108C0A0010A00A001027
:10521000880A001082020010980008208402001002
:1052200004C80400BCC704009C0A0010B3480EF078
:105230008BFDDFF8F48283E6B14B1B689B88002B63
:105240003FF47BAEAF4AB04CDFF8DC8200230BF1B9
:105250002A0108201380316039602B60238088F890
:1052600000000292FFF7C0F8029A74E69A7E0132BB
:10527000D2B2782A9A76BAD15976DFF8AC825FE654
:10528000DFF8A482DFF8A49211228BF82F20DBE64E
:10529000DFF8989212204FF0020E042701265A25BB
:1052A0002C2160228BF82F008BF836E08BF83770BA
:1052B0008BF838608BF8395021808BF82E20DFF87E
:1052C0006882C6E6DFF86492E5E7DFF85C820421D5
:1052D00088F80010029201930EF09AFE029A019B48
:1052E00011883A683260002900F0A8801A8A002AE2
:1052F00000F0A4802832182122808BF82F10DFF8CC
:105300002C92A3E69BF817208049112ACA8B34D02F
:1053100093427FF46CAFBBF82010B9F802209142A1
:105320007FF465AF51E700F00F000328DFF8F88144
:105330007FF406AE082188F80010029201930EF067
:1053400067FE029A019B6EE601215A2382F8301013
:1053500082F83130B6E600F0100101F0FF0C0029B0
:1053600079D0012604201121DD761E825876158021
:10537000DFF8B8918BF82F1066E64FF6FF70824287
:10538000C6D1098C9142C3D1BBF824E0AAF11C0319
:105390005F49BBF822A0BBF81A80BBF81CB0238081
:1053A000DFF85C91CDF80CB001F1440301F5AA706F
:1053B000059403E0443383427AD0614633F8402CAD
:1053C0009C46002AF6D07245F4D133F83E2C0AB13F
:1053D0005245EFD133F8442C002A4CD133F842BC6B
:1053E000BBF1000F06D04245E4D133F8422C039CB8
:1053F000A242DFD1434AC9F80010DFF82C814549A9
:1054000000230220138088F80000316039602B608F
:10541000059C0292FEF7E8FF029A9CE59BF81710A4
:10542000DFF8E88006294CD01129ADD0012954D0ED
:1054300039480EF089FCDFF8F08081E598F800200B
:1054400097077FF57DAD2821102221808BF82F2032
:10545000DFF8D890FAE511882A4D49B1C00747D541
:10546000A3F810C0588A814288BF10801188198221
:105470000022DA7635E74FF6FF74A242B3D133F853
:1054800042BCA345AFD1B5E705297FF462AE002247
:10549000DFF894805A76802288F8002001930EF07D
:1054A000B7FD14228BF82F20DFF88090019BCBE50D
:1054B0001A48059CC9F800C0DFF86C800EF044FC67
:1054C0003EE50290FFF7E6FB029A904230D0144886
:1054D0000EF03AFCDFF8508032E598F82220082AD6
:1054E00000F0AD800F480EF02FFCDFF83C8027E580
:1054F000188A0028B6D028800146B9E7ECC7040016
:10550000A00A00108C0A00109E0A001098000820C3
:10551000F8020820C200082018C804004CC8040083
:1055200070C8040034C804009C0A0010880A0010E7
:10553000B8F822C0B8F81A10B8F81C30B8F824002F
:1055400008F5E072CDF80CC00491059308F5207CB5
:10555000CDF800A012F8071CA2F1200321B132F807
:105560001C8C804500F08A8020326245F2D19BF885
:105570002F30CC4903F03F03022B00F0C880DFF846
:105580003C839BF82F20C74B52073FF5D9AC93F8CB
:10559000295093F82DE093F82C7093F82B6093F832
:1055A000262093F8280093F8271093F82AC0013595
:1055B000DFF80CA3EDB283F829E083F828704FF0F0
:1055C000140E282783F82760502683F82D5083F87F
:1055D0002C0083F82B108AF8002083F82A2083F807
:1055E00026C083F82FE0278083F82E6065B901304C
:1055F000C0B283F82C0038B90131C9B283F82B103E
:1056000011B9013283F82A20BBF82230BBF824609C
:10561000BBF81A50BBF81C00A34FB9F80010B9F83A
:1056200002203B80ABF82430ABF82260ABF81E5070
:10563000ABF82000ABF81A10ABF81C2042E5B8F824
:1056400024204FF6F6718A424FF000008CBF0932D9
:10565000083288F82200A8F82420BBF81C10BBF8F8
:105660001A20B9F80200ABF82010ABF81C00ABF818
:105670001E20ABF81A30DFF84482BBE432F81A8CF3
:10568000DDF80CA0D0457FF46FAF32F8208CDDF848
:1056900010A0D0457FF468AF32F81E8CDDF814A05E
:1056A000D0457FF461AF9BF82F20DFF810820020F7
:1056B00012F0040FDDF800A02B6088F80000DFF87E
:1056C000E4C140F051829CF82EC0AAF114004FEAC8
:1056D0001C1C4FEA8C0CCCEB0000DFF8E4A101F0BD
:1056E0000F0180B2022920808AF800C000F0F0800B
:1056F00010B9910700F0F180BBF826C018896949FC
:10570000844500F03C8210228BF82F209CE4B1F8F5
:105710009461654ADFF8A8A10027864210808AF8C4
:10572000007011D0012601F5CA718AF8006002E00C
:10573000072E2CD0334631F8027F5E1CB842F6B2F9
:10574000F6D100238AF800309BF8B90120B300217C
:10575000564F0B4601260CE0062E5FFA86FE00F03F
:10576000B48097F83900314620370136002800F020
:10577000A9800728F0D148010BEB000E23B19EF859
:10578000BAE1997E8E45E7D9484B0344E4E7DFF858
:105790002C818AF80030F4E60146DFF810C10CEBEA
:1057A0004113002B77D00321002604209976197627
:1057B0009E75DE76D875BBF824003D499880BBF80D
:1057C00022002B60D880BBF81A0091F800E0188006
:1057D000BBF81CC04F788D78C978012058761882A4
:1057E000A3F802C083F80CE05F739D73D9739BF834
:1057F0002910D9729BF8281099729BF827105972BA
:105800009BF82610197202920193FFF78FFA9BF80A
:105810002E10029A01F0F0005028019B7FF73AAD5C
:105820000F092449053F0D78BF008AF80060304613
:10583000B8422CDA0BEB000696F83650B64635B374
:10584000012D09D0022D0AD09EF8376006EB000E1C
:10585000EEB15FFA8EF0EBE70130C0B2E8E796F800
:1058600037C0BCF1040FEFD196F8387096F8396064
:105870008AF8000046EA0726B6F5AD7F34BF304609
:105880004FF4AD700D7016805882988202E58AF848
:1058900000000D70FEE408480EF056FADFF81C8098
:1058A000FFF74EBB98000820800200103802082045
:1058B000840200109502001084C804009C0A0010A5
:1058C000940200108AF800E067E78AF800E068E7D1
:1058D00002F03F0112297FF40BAFD20601D5198ADD
:1058E000D1B95A7E02F00F01013907293FF628ABE2
:1058F0000FF2040C5CF821F08B5B00001D5B0000D4
:10590000535A0000115A0000EF590000D959000005
:1059100007570000BD59000003F10C000193FFF789
:10592000D9F9A74A9BF82A001178019B0391DDF869
:105930000CC0A4498445D4D192F801C091F82B0041
:10594000CDF814C08445CCD191F82C000490DDF83A
:1059500010C090786045C4D191F82D10D2788A4259
:10596000BFD1039993F81BC01973059998735973A4
:10597000DA73BCF1000F19D1187E997E9A7D411A15
:10598000A1EBD201C9B20A44D0B2CAB212F0800F60
:1059900018BF4A42D97D18BFD2B2A1EB91010A4487
:1059A000D2B2987502EBD0001876DA75187E012114
:1059B0000022987688F800101A8292E798F8001072
:1059C000814ACE077FF5BCAA0021597610231370B7
:1059D0000EF01EFBFFF7B4BA98F80020D2077FF54F
:1059E000AFAA0721002259769A76FFF7A9BA208834
:1059F00018B10193FFF79AF9019B9BF82F20D1076B
:105A000000F1A3802288002A7FF47DAEFFF798BAC8
:105A1000208818B10193FFF789F9019B9BF82F208B
:105A200012F0010200F0968098F80020D50740F1AE
:105A300089800022072159769A761A8201200193E3
:105A4000FFF774F9102288F800200EF0E1FA019BAC
:105A500059E69BF82F10CD0724D5D00622D41A8AF8
:105A6000002A7FF46DAA20880193013080B2FFF7ED
:105A70005DF998F80020208842F0100188F80010A5
:105A8000019B514910B142F012020A7001930EF0CD
:105A9000BFFA019B01200821002218825976DA768C
:105AA000FFF7F2BB89060BD59BF834C09BF8350095
:105AB0003168258840EA0C200144281A3160208092
:105AC000208858B1D20609D498F8002042F002028A
:105AD00088F800200193FFF729F9019B9BF830001B
:105AE0009BF83110394A01EB0021988A89B2814232
:105AF000118000D801B91080118898F800205982CF
:105B000095073FF41DAA324A0021118002920193A9
:105B10000EF07EFA019B029AFFF785BA98F80020F2
:105B2000D20706D59BF82F10264A01F03F01122913
:105B300052D0202388F800300EF06AFA2B68002239
:105B40005A761EE506225A7678E707210022597612
:105B50009A7673E798F80010C8077FF553AF0521D0
:105B60001A825976FFF7ECB958761A480EF0ECF81D
:105B7000202388F800300EF04BFAFFF7E1B9088DCA
:105B8000598988427FF4BFADA7E698F800100E4A05
:105B9000C9077FF5D5A920884FF0030E40250021C5
:105BA00083F819E01570198228B142211170019310
:105BB000FFF7BCF8019B064A00211180FFF7BDBB2F
:105BC000980A0010980008209C0A0010800200101B
:105BD0008C0A0010A8C8040092F82E2002F0F001F0
:105BE000502939DD2F491209A2F1050E087800224B
:105BF0004FEA8E0E8AF8002072454EDA0BEB020552
:105C000095F83600AC46002847D0012842D002283B
:105C100008D09CF8375005EB020C002D3DD05FFA00
:105C20008CF2E9E795F83790B9F1040FF1D195F8C6
:105C300038E095F83950DFF874C045EA0E2EBEF50D
:105C4000AD7F34BF75464FF4AD758AF800200870FB
:105C5000ACF800E05D829D829BF828009BF829103B
:105C60009BF826E09BF8275003229872D9725A7647
:105C700083F808E05D7201200193FFF757F8019B5C
:105C8000094A0021422019822180118088F80000F1
:105C9000FFF753BB0132D2B2AEE78AF8002008709A
:105CA000DAE700BF950200108C0A00108002001095
:105CB00040BA80B2704700BF0A1E034609DD05489E
:105CC000054900680A80834203D0194692B241F028
:105CD000CABD7047940A00108C0A00102DE9F041EB
:105CE000334CE37D062B03D0BDE8F0410EF0EAB95A
:105CF000304D2B88B3F5C17FF6D3363B9BB25F089E
:105D0000B3EB470F07F128034FF000064FEA1322C9
:105D1000CCBF07F10108B84622742B80637484F865
:105D2000326084F83360FFF727F8C0436086267638
:105D30006676FFF711F82B88C0430E3320832B8043
:105D40000EF0C0F91C4A08F1280310689BB24FEA14
:105D5000132E4246C11984F810E02B80637441F081
:105D600082FD39461548FEF7B5FF154B84F83260C1
:105D700059789A781878DB7884F8271084F82930D5
:105D800084F8282084F8336084F82600FEF7F4FFB6
:105D9000C043608626766676FEF7DEFF2B88C0431A
:105DA0000E3320832B80BDE8F0410EF08BB900BF8D
:105DB000980008209E0A0010840A0010BE000820E7
:105DC000980A001010B541600446FEF7B1F9206052
:105DD00010BD00BF90E80C0013440360704700BF83
:105DE00010B50446FEF7A4F994E80C00801A984216
:105DF00034BF0020012010BD70B4134E75682A789E
:105E0000A2B103780D2B11D00A2B0FD09A4214D1D6
:105E1000002306E0C25C0D2A08D00A2A06D094426C
:105E20000BD10133DBB2EC5C002CF3D1B268F36828
:105E3000012081E80C0070BC70473668002EDDD16F
:105E4000304670BC704700BFE0C8040010B5064C77
:105E5000206837F0ADF9054A00231068236040F050
:105E600047FE012010BD00BFA00200109C020010E0
:105E700070B5038D82B0B3F5987F0446164600F0E6
:105E80009B8018D9B3F59B7F00F089802FD8B3F59C
:105E9000997F33D0B3F59A7F24D100F12805654866
:105EA00042F0CFF8634902462846FEF7F3FDC8B931
:105EB000002002B070BDB3F5947F5FD059D940F295
:105EC0002912934234D0B3F5977F0BD104F1280502
:105ED000594842F0B6F8584902462846FEF7DAFD1E
:105EE0000028E5D000230220238502B070BDB3F561
:105EF0009C7F10D0B3F59D7FE8D0F3E700F1280533
:105F00004E4842F09EF84D4902462846FEF7C2FD33
:105F10000028E7D1CCE700F12805494842F091F884
:105F2000474902462846FEF7B5FD0028DAD1BFE70B
:105F300000F12805434842F084F8424902462846C9
:105F4000FEF7A8FD0028B3D0002ECBD004F1B4009A
:105F50002E2142F0DEF8064600284ED03A4831465F
:105F6000052242F0AEF8002833D14FF49873238510
:105F700024E0002BB6D14FF49473038508460191B9
:105F800042F05FF804F12805024601992846FEF721
:105F900081FD00288CD040F229132385CAE700F147
:105FA00028052A4842F04DF8284902462846FEF7BF
:105FB00071FD002896D17BE700F12805244842F0C6
:105FC00040F8234902462846FEF764FD002889D19F
:105FD0006EE720483146042242F073F818B94FF4B6
:105FE000997323858CE71C483146042242F069F8F6
:105FF00038B94FF49A73238551E74FF4977323858B
:1060000066E716483146042242F05BF818B94FF4AF
:106010009B732385C5E731461148042242F051F8AD
:1060200018B94FF49C73238577E74FF49D7323854C
:106030004EE700BF2C1C0500201A0500481C050077
:10604000DC1B0500141B05005C1A0500A41C0500E0
:10605000101C05006C1A0500641A05000C1B0500D5
:10606000D41C050038B5038D044603B3B3F5857F12
:1060700019D100F1280528460E492246FEF732FDC7
:10608000A0B1B4F83C21D4F83431D4F830119B1AC3
:10609000002B0A44C4F83431C4F8302103DD4FF436
:1060A00085732385E7E700232385022038BD00F1AF
:1060B0002805F4E70161000038B50E4B0E4D1B6852
:1060C00004465A8A0121D0F83831286841F0ACF8EA
:1060D000002803DDA4F83C0180B238BD074A2B68D4
:1060E000108891781880002299700220A4F83C2131
:1060F00038BD00BF7C0A0010840A00101082050021
:106100000A4B10B51A68D0F83431528A04469342CB
:10611000D8BF9AB2064BA0F83C21D4F830111868C9
:1061200041F0A1FBB4F83C0110BD00BF7C0A001097
:10613000840A001038B505460C4631B3D8B1D1F801
:1061400054010EF099FB092805DD2146124841F063
:1061500061FC002038BD21462A46104841F05AFC17
:106160002846D4F8544141F051FF014620460EF034
:106170006BFB012038BD0A4841F04CFCD4F85401B7
:1061800029460EF061FB012038BD064841F042FC73
:106190004FF0FF3038BD00BF501D0500341D050015
:1061A0001C1D0500F01C050038B5134D0C460A46B1
:1061B0002B68012141F092FAA04204D0FFF746FE7D
:1061C0000023184638BD0D4B1A681044B0F5C87F3F
:1061D00003DA18600123184638BD002228681A60C7
:1061E00040F086FC064B0749186840F023FF012366
:1061F0002860184638BD00BF9C02001098020010AD
:10620000A0020010741D05002DE9F047A54EA64D13
:1062100031782F68480682B0FC695ED4002C00F00B
:10622000F88101F0080303F0FF0223BB227011F094
:10623000300F2BD10A0629D494F82D31032B00F00E
:10624000D380A28840F2ED118A4200F01E82B2F59E
:10625000F77FC0F09180B2F50F7F00F0E68140F249
:106260004D218A4200F09681B2F5017F00F01C8238
:106270000022A280B5E023780133DBB2272B237004
:10628000D5D98A4841F07AFC202333702B6888489E
:10629000D98849BA89B241F0BDFBD4F838311BB175
:1062A000844B186840F024FCD4F8400108B136F063
:1062B0007FFFD4F850313BB1D4F854010EF0FAFA14
:1062C000D4F850010EF05CFC204636F071FF2B68CC
:1062D0000022DA6102B0BDE8F0874FF4AE7036F00C
:1062E00061FF0446002800F09A81F8613888FFF7C2
:1062F000DFFC2B6882461888FFF7DAFC2B688146A2
:106300005888FFF7D5FC2B6880465888FFF7D0FCEB
:106310002B685FFA80FCB3F806E004F150079EFAA0
:106320009EFE1FFA8EF0C8F30F23CDF800C0CAF30B
:106330000F215FFA89F201905F4841F06BFB39460B
:10634000201D6322FEF772FC394604F12800632207
:10635000FEF76CFC0023A4F84C30A4F84E3084F80F
:106360002D312370C4F83831C4F84031C4F85431A9
:10637000C4F85031317854E7002A00F02281B2F598
:10638000EF7F7FF475AF251D28462021FEF7E6FB41
:10639000002800F03B8104F15007384647490322AA
:1063A00041F08FFE002840F072810123444984F8B7
:1063B0002C31444841F02EFB40F2ED13A3802846D7
:1063C0002021FEF7CBFB002800F0208194F850300C
:1063D0002F2B00F0AD8100231022A38094F82D31E3
:1063E0003270032B7FF476AFB4F84C30B3F5AF7F47
:1063F00000F0C68124D940F2711293421BD0B3F54C
:10640000B97F3ED2B3F5B37F00F0268340F24782D6
:1064100040F2671293420ED0B3F5B87F2DD12046DB
:1064200029490122FFF724FD00283FF453AF40F231
:106430007113A4F84C302046FFF714FED8B949E791
:10644000B3F5A87F00F0DA8242D9B3F5AB7F00F054
:10645000E98240F2B88140F25B12934270D0B3F50A
:10646000AE7F0AD104F1280018490822FEF712FB7A
:1064700000283FF42FAF102333700023A4F84C30D2
:1064800028E740F27F12934200F06582B3F5C07FA7
:10649000C0F08B81B3F5C17F00F06E82B3F5C37F8E
:1064A000C9D0EAE79C0A00107C0A0010E01D050034
:1064B000F81D05009C020010A81D0500DC1C05004D
:1064C000881D0500281E0500401A05001020050043
:1064D000B3F5A57F00F06F8240F24B12934200F0BB
:1064E0005A81002BC9D194F82C31032B00F05F8224
:1064F00004F1B405022B284640F05283B94941F01B
:1065000073FD002800F073822846B74941F06CFD06
:10651000002800F080822846B44941F065FD00283B
:1065200040F08982B24894F84A1141F073FA94F825
:106530004A31002B40F0208140F25B13A4F84C302C
:106540002046AC490122FFF793FC00283FF4C2AE7D
:106550004FF4AE73238585E7A74841F00FFB94F80D
:106560002C31032B984600F08D82012B00F089829C
:10657000022B40F0CD8004F1B40738469B4941F02E
:1065800033FD002840F05A83042384F82D3140F273
:106590004D23A380B4F84E30D4F80C90E78A002B3A
:1065A00000F0838140F2C11293420ED00023A4F880
:1065B0004E3000220323E28284F8242084F82D3117
:1065C00056E64FF4EF73A380DDE694F84B31012BD0
:1065D00019D033789B0719D5884B894A1D88012328
:1065E000106884F84B31002D40F0F181D4F84471EB
:1065F000002F40F3FD8240F2C113A4F84E3094F80E
:106600004B31012BE5D1002384F84B3194F82D3127
:10661000E7E67C4841F0FEF9202333705AE67A48D9
:1066200041F0ACFA2023337054E6251D28460A2198
:10663000FEF794FA0028E9D02846FEF789FA0023ED
:10664000204480F84F302846D4F84471FEF780FA91
:1066500004F150033A1A19461F46C4F844216B4806
:1066600041F0D8F93846D4F850110EF077F9B4F863
:1066700058310133A4F85831D4F84431022B40F397
:1066800039834FF40F73A380D0E7251D97E6384672
:106690005F49042241F015FD002840F047810223A4
:1066A00084F82C315B4984E6251D28460A21FEF733
:1066B00055FA0028AAD02846FEF74AFA00232044BB
:1066C00080F84F3094F850300D2B3FF445AF04F173
:1066D00050073946504841F09DF938464F4910223D
:1066E00041F0EFFC8046002800F0E18138464C493B
:1066F0000B2241F0E6FC8046002800F0ED81384690
:1067000048490F2241F0DDFC0746002800F00182D5
:1067100094F82D1101292BD0022900F0B78104290A
:106720003FF435AF404841F075F994F82D319FE5BD
:1067300094F85130202B00F09C812846FEF708FA8F
:1067400004F1B4072044002380F84F3004F15001D5
:1067500038463C2241F0CBFC3946344841F05AF9E6
:106760000023012284F82D21C4F8443184F84C31EF
:106770004FF40173A38098E74FF4AF73A4F84C3043
:1067800020462B490122FFF773FB00283FF4A2ADFE
:1067900040F25F13238504F1280026490422FEF706
:1067A00079F900287FF467AE94E540F27B129342BA
:1067B0007FF463AE204620490022FFF759FB0028F2
:1067C0007FF459AE86E5B3F5A97F7FF456AE238DED
:1067D000D32B33D0D92B47D0002B57D00023238580
:1067E00049E600BFBC1E0500C81E0500541E05007A
:1067F000FC1F0500641C0500441E05009E0A0010D5
:10680000840A0010C41D05008C1D05000C1F050026
:10681000741A0500781D05005C1E0500FC1B0500B0
:10682000881E0500941C0500941F0500341E0500F9
:10683000C01C0500A41F05005C1B0500D4F8540112
:106840000EF01AF800287FF745ADD4F854010EF089
:1068500045F80146C4F84001002800F03082B748EE
:1068600041F0D8F8D9232385D4F84051284641F087
:10687000E8FB2946024604F12800FEF70BF9002840
:106880003FF428ADD4F8400136F092FCD3232385A1
:10689000D4F854010DF0F0FF0028D6DC1AE540F2E0
:1068A0005F1293423FF477AFE7E504F1F005DFF8BC
:1068B000ECA22946A248D4F8442141F0ABF8DAF81A
:1068C000000008B136F074FC284641F0BAFB0530F0
:1068D00036F068FC9B4B8046294640F8043BCAF8DA
:1068E000008041F08BFB4046974940F0A3FB974B5B
:1068F0008046DFF8A8A21860002800F089812946A8
:10690000934841F087F8002F6ED048463946FFF78C
:106910004BFC0546002800F0AE81D4F84431DF1B63
:10692000C4F84471012384F84B3161E63846894943
:10693000072241F0C6FB002840F0E680032384F8DC
:106940002C31854935E52946844841F063F840F209
:106950007F13A4F84C30204681490122FFF788FAC2
:1069600000283FF4B7ACD4F83831002B00F0B181E7
:106970004FF4C173A4F84C30238D002B00F0C1807C
:10698000B3F58C7F7FF42AAF04F1280528467549BA
:106990002246FEF7A7F800283FF49CACB4F83C71FF
:1069A000002F00F02E814FF48C732385EEE74FF417
:1069B000A573A4F84C3020466B490122FFF758FA22
:1069C00000283FF487AC40F24B132385E3E62946C9
:1069D000FFF7EAFB0746002800F02881D4F844714D
:1069E0007F1BC4F8447103E6D4F844719AE75F480A
:1069F00041F0C4F84FF4A873A4F84C30204658492D
:106A00000122FFF735FA00283FF464AC4FF4A97374
:106A1000A4F84C30DBE6564841F0B0F84FF4AB73C5
:106A2000A4F84C3020464E490122FFF721FA0028F5
:106A30007FF421AD4EE429464E4840F0EBFF04F5CB
:106A400098714D48FFF7D8F928464B4941F0D6FADE
:106A50004FF4B373A4F84C30204648490122FFF7A5
:106A600007FA00283FF436AC40F26713A4F84C3024
:106A7000E1E404F1B407384641493C2241F037FBD8
:106A80006AE6032384F82D31FFF7F2BB94F82C81DA
:106A900004F1B407B8F1020F00F0D280394639484A
:106AA00040F0B8FF032384F82D31FFF7E1BB2846FF
:106AB000FEF74EF804F16007204480F84E80384617
:106AC0003FF0AAFF39460246C4F844012E4840F080
:106AD000A1FF94F82D111DE62846FEF739F804F1C0
:106AE000F007204480F84E8004F15C013B223846D8
:106AF00041F0FDFA3946254840F08CFF94F82D11FD
:106B000008E604F128054EE73946214840F082FFA7
:106B100061E42846FEF71CF8204480F84E7004F12A
:106B20005F0108221B4841F0CCFA011C18BF01216B
:106B300084F84C11184840F06DFFE9E5C41F0500CA
:106B40003C1F05002F73642F541F05009C0200108A
:106B50009C2005007C1C0500801D05008820050088
:106B6000C01C0500B96000007C1A0500AC1F0500C0
:106B7000DC1F05001C200500D01B0500401A050085
:106B8000E41C0500D81E0500701E0500981E0500B7
:106B9000101E0500881C0500AC1E0500A002001098
:106BA0005C49042241F08DFA00286CD129465A48EC
:106BB00040F030FF2846594940F03CFAC4F838010B
:106BC000002800F09F8094F84C31002B3FF4BBAEBE
:106BD000D4F8380120B13FF08BFF0023C4F83831DE
:106BE0004F4840F0CBFF40F27B13A4F84C30E1E576
:106BF000FFF72CF9012384F84A314A4840F0BEFFE0
:106C0000D4E4D4F838013FF073FFC4F83871E5E5F7
:106C1000DAF8000036F0CCFA4348CAF8008040F0B9
:106C2000ADFF84F84A81A4F84E80C2E43F4840F0AA
:106C3000A5FF84F84A71A4F84E70BAE484F82D8157
:106C400038463B4941F0D0F9002848D03846394908
:106C500041F0CAF900287FF421AFC4F85001D4F8FC
:106C6000441100239942A4F858317FF70AAF324803
:106C700040F0D0FE00E5314840F080FF84F84A51F2
:106C8000A4F84E5095E4002304F59877C4F8383101
:106C900039462846FFF7B0F8002894D1284840F03C
:106CA0006DFF39462748FFF7A7F82846254941F0E8
:106CB000A5F94FF4B873A4F84C30FFF7B0BBB4F8A3
:106CC0005831013B9BB2A4F85831002B3FF486ADFC
:106CD000DCE54FF4C373A4F84C30FFF7ACBB0DF008
:106CE000A9FD2146C4F8540117480DF029FFC4F846
:106CF0005001B4E7154840F041FF032384F82D31DB
:106D0000FFF7B6BA1248294640F084FE04F598779A
:106D1000C4E700BF3020050038200500D4A60500D8
:106D200074200500841F0500581F0500741F05000E
:106D3000BC1E0500C81E0500F01E05006C1F0500E6
:106D400060200500D01B0500356100002C1F0500E8
:106D50004C2005004FF4A040FEF7A2B8042808D844
:106D6000064B53F8203023B122B91A6822EA0101F8
:106D7000196070471A68114319607047B020050008
:106D8000042804D8024B53F8203003B199617047AE
:106D9000B0200500042804D8024B53F8203003B17A
:106DA000D9617047B02005001F2811D9203803226F
:106DB000824001FA00F00E4BD3F8AC1121EA020236
:106DC000C3F8AC21D3F8AC211043C3F8AC01704731
:106DD000032282408140064BD3F8A80120EA020238
:106DE000C3F8A821D3F8A8211143C3F8A81170470C
:106DF00000C00F4001290AD041B9094A094BD2F815
:106E0000C4100B4023EA0003C2F8C4307047044AA0
:106E1000044BD2F8C41003400B43C2F8C43070478F
:106E200000C00F40DEF7EFEF38B50446F8B1012897
:106E300021D1214A214B126889089508A3FB050539
:106E4000AD0C05FB01F5FE2D24D85508A3FB050567
:106E5000AD0C05FB01F5FE2D25D8A3FB0205AD0CFD
:106E600005FB01F5FE2D4FF000000BD838BD21F0D9
:106E70000301FE2901D8002038BD4FF0804359603E
:106E8000012038BD2146FFF78FFF4FF08043204699
:106E90005D6038BD00200146FFF786FF4FF080435C
:106EA00020465D6038BD00200221FFF77DFF4FF0D6
:106EB000804320465D6038BD9801001083DE1B438F
:106EC00038B5054600200C460146FFF76DFF4FF030
:106ED00080431A69012C22F003021A611A6945EAFB
:106EE00002051D6103D11A7842F002021A7038BD02
:106EF00010B54FF080442369014603F00300FFF70B
:106F000093FF237843F00103237072B64FF0804360
:106F1000AA21552219721A7262B610BD4FF0804331
:106F20001A7802F0FB021A70704700BF72B64FF079
:106F30008043AA21552219721A7262B6704700BFA7
:106F400030B4427803210F2A88BF103A4FEA420238
:106F500001FA02F18478037804FA02F24FEA43035B
:106F600088BF01339B0003F1804303F530331C6875
:106F700024EA01011960196803240A431A6042785F
:106F8000C1780F2A88BF103A4FEA420204FA02F48D
:106F900001FA02F10378154A4FEA430388BF01332F
:106FA00052F8235025EA040442F8234052F82340C3
:106FB000214342F8231002790378012A41780BD04B
:106FC00030BC012202FA01F1094A52F8230020EAFA
:106FD000010142F8231070478A4030BC044850F841
:106FE00023100A4340F82320704700BF40C00240EE
:106FF00068C002407F2810B40ED981B90E4B01E061
:10700000802915D033F8022F8CB2824201F10101A0
:10701000F6D104F1800080B25DF8044B7047FF2880
:1070200006D8064B803833F810005DF8044B7047E3
:1070300000205DF8044B7047A2220500A422050041
:1070400061280AD00749002201E0834206D031F8C6
:10705000023F0132002BF8D170470022024B33F877
:1070600012007047C4200500A423050000487047A3
:107070008425050000487047942505000249034A0D
:1070800001608260704700BFE046050050C6050001
:1070900010B50A4B0A4A044603F1540103F14800B3
:1070A000C4F890002360C4F89410C4F8982004F148
:1070B000940004F0DBF8204610BD00BF80470500B7
:1070C000A02D0500A0F19800FFF7E2BFA0F1940009
:1070D000FFF7DEBF10B5074B044603F1300103F1A3
:1070E00048022360616040F8082F04F0BFF8204692
:1070F00010BD00BFA0440500A0F10800FFF7EABFE3
:1071000010B5044A044B04460260836003F0C8FDD6
:10711000204610BDE046050050C6050010B50B4BDB
:107120000B4A044603F1540103F148002360C4F8FC
:107130009000C4F89410C4F8982004F1940004F06E
:1071400095F8204603F0ACFD204610BD80470500B1
:10715000A02D0500A0F19800E0E700BFA0F1940089
:10716000DCE700BF10B5084B044603F1300103F122
:1071700048022360616040F8082F04F077F8204649
:1071800003F08EFD204610BDA0440500A0F10800CC
:10719000E8E700BF38B50E4B044603F15C0503F188
:1071A000680103F1800284E82800A16040F89C2F68
:1071B00004F05CF8074B204603F14C0103F1580240
:1071C00023606160A2600EF0EDFD204638BD00BF77
:1071D000E830050040430500A0F19C00FFF7DABF4E
:1071E00010B5034B0446036005F0FEFF204610BDBA
:1071F000802A050010B5054B0446036005F0F4FF36
:10720000204603F04DFD204610BD00BF802A05003A
:1072100038B50F4B044603F15C0503F1680103F137
:10722000800284E82800A16040F89C2F04F01EF83A
:10723000084B204603F14C0103F1580223606160C2
:10724000A2600EF0AFFD204603F02AFD204638BDB7
:10725000E830050040430500A0F19C00D8E700BFDE
:107260002DE9F041B74CA6B004F10A05204601F023
:1072700079F920460021023401F07CF9AC42F5D1C5
:10728000AC203BF01DF8044601F08CFEAE4AAF4B3B
:1072900012686068A3FB02120368920CAC499B68F9
:1072A0009847656801A82B689E68FFF7DFFE0746D0
:1072B00001A8FFF7DFFE3A460346A6492846B04735
:1072C000A54810F089F9D0F1010838BF4FF0000847
:1072D000B8F1000F00F0CB81A04D5421286803F0D5
:1072E000C3FB064622F0AAFB3146204602F01EFAF6
:1072F0000821286803F0B8FB064624F099FC3146C3
:10730000204602F013FA1021286803F0ADFB064670
:1073100023F08CFF3146204602F008FA102128683D
:1073200003F0A2FB064627F0FDFB3146204602F0A3
:10733000FDF9B421286803F097FB06461FF094FA84
:107340003146204602F0F2F901203AF0B9FF064634
:107350001FF022F9304603F0A3FC01203AF0B0FF01
:10736000064614F097F9304603F09AFC01203AF0F3
:10737000A7FF064618F044FD304603F091FC20209C
:107380003AF09EFF064619F083F93146204602F096
:10739000CDF94FF48871286803F066FB064625F0A6
:1073A000A3FC3146204602F0C1F93421286803F0DD
:1073B0005BFB074603F06AFF694B384640F8183B11
:1073C00000F0E0FA97F83030002666F3041387F8EF
:1073D000303039463E627E62BE62204602F0A6F937
:1073E0001021286803F040FB027B002366F30002B3
:1073F0000273436083600660074603F047FF594B02
:1074000039463B60204602F091F90421286803F0D8
:107410002BFB074603F03AFF534B39463B602046AF
:1074200002F084F940203AF04BFF07460CF092FC42
:107430003946204602F07AF91821286803F014FB37
:10744000074618F083FD3946204602F06FF92021E7
:10745000286803F009FB074613F032FE3946204640
:1074600002F064F928203AF02BFF3146074626F057
:107470004DFD3946204602F059F93C4805F034FDEF
:1074800020463B4902F052F920463A4902F04EF9B3
:10749000324633464EF6D321606903F017F9314680
:1074A00003F0CAFE03F0B2FE002840F0F480002290
:1074B000134644F20901606903F008F9002103F062
:1074C000BBFE03F0A3FE002840F0D7800022134645
:1074D0004DF2BD11606903F0F9F8274903F0B8FED9
:1074E00003F0DCFD254905463CF014FD002863D07F
:1074F00004203AF0E5FE2249064628463CF04EFBC1
:107500003CF04EFD00220146304603F02FF8314694
:10751000204602F00BF928463BF0ACFE66680246B6
:1075200035680B46AD6830461649A84720461649CF
:1075300002F0FCF8606903F083F894F8A830DB07E8
:1075400040D423E0A40200109801001083DE1B4306
:10755000AC250500C825050000C00720FC0200106E
:1075600010620500206F0500884A050020C0072032
:10757000C8C007203CC2072000002041CDCCCC3D34
:10758000002474490C260500BCC00720B8F1000F88
:1075900023D14A4C2368DA68986992F855110BF0A8
:1075A0009FFD2368D86A04F047F82368986A03F0BF
:1075B000C1FC26B0BDE8F0816068414903689B6862
:1075C0009847B3E701213F4800F0D4FF3E484146C9
:1075D00000F0D0FFB8F1000FDBD03C483C493FF051
:1075E00029FD06460028D4D060683A490368374A26
:1075F0009B689847DFF8F480374F8421324605A80E
:107600003FF00AFC26AD354905AA38B36068036827
:107610009B6898479DF8143005A93B2B02AA4FF0B0
:10762000000E04A8E9D045F88C8DCDF810E03BF0B1
:1076300029FC20462A46012102F07EF8049BA3F192
:107640000C00B842D9D053F8042C511E002A43F83C
:10765000041CD2DC02A93BF07BF9CEE7606820492C
:1076600003689B68984730463FF042FA91E76068AC
:107670001C4903689B6898472EE628684C2103F054
:10768000F3F91949054605F035FA9DB1291D204643
:1076900002F04CF81AE7C021286803F0E5F9124916
:1076A000064610F0C5FA3EB106F19401204602F0FC
:1076B0003DF8FCE62946EAE73146F7E7E402001028
:1076C00030260500A4020010AA0200105026050072
:1076D000D4A6050064260500640A00108C26050067
:1076E00094260500EC25050020C00720100300109B
:1076F00070B5FFF7B5FD0D4C0025264620686A1CC5
:1077000090F8A83092B2DB0706D5C5F300310848DF
:10771000154600F02FFF306800210A4602F00CF8F1
:1077200020680321002202F007F8E7E7E4020010D6
:10773000A6020010F0B52B4B2B4C83B02B4E0093C0
:10774000204601332A492B4A0FF0CCFB04F12005D7
:107750003246294920463AF0D8FD284605F0F0FC8B
:1077600004F5D4773246284624493AF0CEFD29461E
:10777000384610F05DFA32463846214904F1C00718
:107780003AF0C3FD2946224638460EF07DFE3246C9
:1077900038461C4904F51A771B4D3AF0B6FD2246CF
:1077A00038461A4903F02EF93246384618493AF05D
:1077B000ACFD2846174900F0C9FEA81C164900F088
:1077C000C5FE281D154900F0C1FEA81D144900F092
:1077D000BDFE144905F1080003B0BDE8F04000F01B
:1077E000B5BE00BF06C0092000C00720C8000010B9
:1077F00009C0092008C009207D70000095710000B3
:1078000091700000D5700000A4020010B42605009D
:10781000E171000032C0092033C0092034C00920C2
:1078200035C009209CC0092010B44379002B2FD10A
:1078300003790F2B19D802225B0002FA03F3504A96
:107840000124116C0B4313640379116CA34004FAF7
:1078500003F321EA030313644379CBB903790F2BB4
:1078600003D800205DF8044B704702225B0002FA47
:1078700003F3434A0124516C0B4353640379516C65
:10788000103BA34004FA03F321EA03035364437952
:10789000012B1DD0022B48D0032B5BD0042BE0D151
:1078A00003790F2BDDD95B0002229A40344B01246F
:1078B000596E0A435A660279596E103AA24004FA88
:1078C00002F221EA020200205A665DF8044B70477A
:1078D00002790F2A14D80221520001FA02F2284933
:1078E0008C6C22438A6404798A6C6400A34022EA87
:1078F00003038B644379012BCCD102790F2AB0D9D1
:107900000223520003FA02F21D4B0124D96C0A43F0
:10791000DA640279D96C103AA24004FA02F221EA40
:107920000202DA644379022BB6D102790F2A98D881
:1079300052009340124A0124116D0B4313650379E1
:10794000116DA34004FA03F321EA0303136543799D
:10795000032BA3D103790F2B83D95B0002229A401A
:10796000074B0124D96D0A43DA650279D96D103AC3
:10797000A24004FA02F221EA0202DA6543798DE7B5
:1079800000C00240827910B402F0FE0220246FF39E
:10799000410200210471827101605DF8044B70475F
:1079A00010B5837904469B0714D543793BB9037915
:1079B00001229A401B4B996E0A439A664379012B28
:1079C00012D0022B19D0032B21D0042B04D0204637
:1079D000FFF72AFF204610BD237901229A40114B60
:1079E000996F0A439A67F2E721790E4A8B40D16E6C
:1079F0000B43D3666379022BE5D1237901229A40A8
:107A0000084B196F0A431A676379032BDDD1237979
:107A100001229A40034B596F0A435A676379042B3A
:107A2000D5D1D9E700C00240837930B49B071ED579
:107A30004379F3B1012B4BD0022B00F08B80032B49
:107A400072D0042B13D103790F2B10D95B000122C4
:107A50009A404A4B0224596E0A435A660279596E7B
:107A6000103A520004FA02F221EA02025A6630BCCD
:107A7000704703790F2B16D801225B0002FA03F33B
:107A80003E4A0224116C0B4313640379116C5B00B2
:107A900004FA03F321EA030313644379002BC9D1E9
:107AA00003790F2BE3D901225B0002FA03F3334A77
:107AB0000224516C0B4353640379516C103B5B00FF
:107AC00004FA03F321EA030353644379012BB3D18E
:107AD00002790F2A14D852009340284902248D6C51
:107AE0002B438B6403798A6C5B0004FA03F322EA6C
:107AF00003038B644379012B9ED102790F2AB6D9F7
:107B00000123520003FA02F21C4B0224D96C0A43EF
:107B1000DA640279D96C103A520004FA02F221EACE
:107B20000202DA64437987E703790F2B9FD95B0060
:107B300001229A40114B0224D96D0A43DA65027979
:107B4000D96D103A520004FA02F221EA0202DA6513
:107B5000437976E702790F2A89D8520001219140B2
:107B6000064A146D214311650479116D6400A34028
:107B700021EA03031365437961E700BF00C00240B7
:107B8000837910B49B0716D54379BBB1012B34D050
:107B9000022B5DD0032B4ED0042B0CD103790F2B7D
:107BA00009D9103B03225B0002FA03F32F4A516EFE
:107BB00021EA030353665DF8044B704703790F2BEA
:107BC0000ED803225B0002FA03F3284A116C21EA63
:107BD000030313644379002BD8D103790F2BEAD91F
:107BE000103B03225B0002FA03F3204A516C21EAA6
:107BF000030353644379012BCAD103790F2B0ED8A9
:107C000003225B0002FA03F3184A916C21EA030392
:107C100093644379012BBBD103790F2BCBD9103B54
:107C200003225B0002FA03F3104AD16C21EA03033A
:107C3000D3644379ACE702790F2ABCD9103A5200D9
:107C400093400A49CC6D24EA0303CB654379A3E74B
:107C500003790F2BAFD803225B0002FA03F3034A28
:107C6000116D21EA03031365437993E700C00240D5
:107C7000837910B49B0715D54379B3B1012B31D06B
:107C8000022B57D0032B49D0042B0BD103790F2B98
:107C900008D9103B03225B0002FA03F32C4A516E11
:107CA0000B4353665DF8044B704703790F2B0DD8D7
:107CB00003225B0002FA03F3254A116C0B431364A1
:107CC0004379002BDAD103790F2BEBD9103B032238
:107CD0005B0002FA03F31E4A516C0B435364437971
:107CE000012BCDD103790F2B0DD803225B0002FAB3
:107CF00003F3174A916C0B4393644379012BBFD173
:107D000003790F2BCED9103B03225B0002FA03F359
:107D10000F4AD16C0B43D3644379B1E702790F2A40
:107D2000C0D9103A520093400949CC6D2343CB652A
:107D30004379A9E703790F2BB4D803225B0002FA39
:107D400003F3034A116D0B43136543799AE700BFB0
:107D500000C002402DE9F0410F4686B004464A4972
:107D600038463AF0A9FD38B9A37960F34103A3710D
:107D7000204606B0BDE8F081444E01AD0FCE0FC5E0
:107D8000A279D7F800803368002142F0020206AFE2
:107D900047F8181DA271694640460A222B6041F03F
:107DA000CDF8009BC0B2434560710AD9042808D8B9
:107DB00006AA02EB800050F8142C22601A782E2AB2
:107DC0000FD0A27900230199202002F0FD0263F375
:107DD000000220712046A2716371216006B0BDE8E7
:107DE000F0815D1C0A2269462846009541F0A6F8FC
:107DF000009AC0B295422071E3D21F28E1D8012336
:107E000003FA00F02368196921EA0001196110786A
:107E100088B9ADE76F2827D0762820D05E2828D0F3
:107E200001F094FE0028A3D0009A1346013200927C
:107E3000587800289CD040280CD0EBD821281DD0A1
:107E40002D28EDD1A3799B07EFD52046FFF7ECFC59
:107E5000009AEAE72046FFF7E7FD009AE5E72046AB
:107E6000FFF706FF009AE0E72046FFF799FD009A2A
:107E7000DBE72046FFF784FE009AD6E7A37943F0BC
:107E80000103A371D1E700BFCC260500B826050089
:107E900010B54379012B13D0022B27D0032B0DD122
:107EA0000379192B49D01A2B08D108203AF008FA87
:107EB0004A49044638F054FE204610BD002010BD4B
:107EC0000379122B42D0142B49D0152B50D0172BED
:107ED0002AD0182B55D01A2BF0D108203AF0F0F9FF
:107EE0003F49044638F03CFE204610BD037993B16B
:107EF000012B4FD0022B56D0032B5DD0042B64D026
:107F0000052BDBD108203AF0DBF93649044638F07E
:107F100027FE204610BD08203AF0D2F93249044627
:107F200038F01EFE204610BD08203AF0C9F92F494E
:107F3000044638F015FE204610BD08203AF0C0F97E
:107F40002B49044638F00CFE204610BD08203AF0BC
:107F5000B7F92849044638F003FE204610BD082032
:107F60003AF0AEF92449044638F0FAFD204610BD37
:107F700008203AF0A5F92149044638F0F1FD2046E1
:107F800010BD08203AF09CF91D49044638F0E8FD80
:107F9000204610BD08203AF093F91A49044638F0FB
:107FA000DFFD204610BD08203AF08AF91649044644
:107FB00038F0D6FD204610BD08203AF081F913496B
:107FC000044638F0CDFD204610BD08203AF078F97F
:107FD0000F49044638F0C4FD204610BD7AC0092080
:107FE0003AC0092045C0092040C0092037C00920F7
:107FF00079C0092032C0092034C0092035C00920C9
:1080000038C0092041C0092042C0092043C00920CE
:1080100044C0092038B503468079C0F3400080B1E0
:108020001A79012191401A68106820EA0101116053
:10803000587910F0FD0F05D09A7900206FF34102B6
:108040009A7138BD197938F0A5F8054660203AF0E4
:1080500037F92946044639F05DFA204638BD00BF9D
:1080600038B5084B05280C461B680ADC80011D1832
:10807000A91D281D3E22C4F30B143FF0FDFBA5F8FB
:10808000424038BDB002001038B5094B04464C20C0
:108090001C603AF015F9082205464FF47A7104F095
:1080A000E7F928462560034904F09EFC204638BDC8
:1080B000B0020010618000000B68134A934205D0A3
:1080C000124A93420FD04FF0FF3070470B79172BB5
:1080D00012D0182B12D0192B12D00D481A2B18BF02
:1080E0004FF0FF3070470B791E2B0BD009481F2B28
:1080F00018BF4FF0FF307047074870470748704778
:10810000074870470748704700C0092020C0092071
:108110001AC009203FC0092017C0092018C0092033
:1081200019C009203EC0092038B50446FFF7C4FF36
:1081300005460146206804F0C7FA04EB801040228F
:10814000002104303FF0B3FB2068012104F0F2FB72
:1081500020682946012204F0C3FA2068294601223A
:10816000BDE8384004F008BC88422DE9F04781465C
:108170008A462BD0851CA94228D0074637F8026FC3
:10818000B9F800302C46B34205F1020810D837F890
:10819000023C9E4207D2AA1E2380154632F8023DB9
:1081A0002C469E42F8D3D0452E800FD04546E5E7B9
:1081B000C9EB07035B1005D05A00C2EB0800494623
:1081C0003FF05AFBD045A9F80060EFD1BDE8F08739
:1081D0002DE9F00102F1FF3808EBD8784FEA680882
:1081E0004145B8BF0C464CDA651C6C0004F10046F2
:1081F000013E30F816C030F825602746B4450744E4
:1082000000EB850504D9013C30F8146000EB44050F
:10821000444527F8026CE7DBD60705D4023A02EBA7
:10822000D272B4EB620F20D0621E02EBD2728C428B
:108230004FEA620215DD30F81260B34206D810E052
:1082400030F815601446B34209D92A46551E05EB8D
:10825000D575914220F814604FEA6505F0DB00EB1C
:1082600042052B80BDE8F00170470134640004F141
:108270000042013A30F81220013C2A8000EB44050C
:10828000D2E700EB41050C46C6E700BF2DE9F84FE9
:108290000B1A212B8246934640F39380002A6BD021
:1082A00000F102099B103AF81320BAF802400BF1D2
:1082B000FF3B944231F8020C44D2824246D38442BE
:1082C00051D2BAF80050AAF8000021F8025CBAF8BE
:1082D0000260BAF80040A6420F464B461DD2023358
:1082E000984633F8026BA642FAD3A542A7F10203DF
:1082F00018D93B1F1F4633F80259A542FAD8B84592
:1083000013D2434623F8025B3E80B8F80260BAF805
:10831000004037F8025CA642E1D3A5429846A7F197
:108320000203E6D81F46B845EBD340465A46FFF74E
:10833000ADFFCAEB0803212B41DDBBF1000F1CD0C0
:108340004146AFE784420ED38242BAD3BAF8000066
:10835000AAF800202AF81300BAF8026031F8025C8B
:10836000BAF80040B7E7BAF80060AAF80040AAF8E7
:10837000026031F8025CAEE788465E10B41E6410FD
:10838000651C0AEB450500E0013C5046214632469B
:1083900035F8023DFFF71CFF002CF5D1BAF800209C
:1083A00038F8023C28F8022DCAEB08046210504647
:1083B0000021FFF70DFF032CF0DCBDE8F88FBDE8CE
:1083C000F88FBDE8F88F00BFF0B591B00446FFF715
:1083D00073FE0146206804F077F9064672B604EB96
:1083E00080131C1D03F1440E6F4620686168A2686B
:1083F000E3683D460FC5103474452F46F5D162B68B
:108400000A22684610A9FFF741FF684608A9FFF74E
:10841000ABFE0FAF07A88588041D30F8023FAB42C2
:1084200034D902462380114632F8023D0C469D4263
:10843000F8D3B8420D80EED10DF12E000DF10E03F0
:10844000002233F8021F83420A44FAD112499208EB
:1084500001EBC6039C885888DC80988031F8364050
:1084600090B25C8021F8362059889A880844DB88CD
:10847000104418443BF03EFB4FF07A513BF08EFB2A
:108480003CF092FB3BF08CFD11B0F0BD2146B842B0
:108490000D80C0D1D0E700BFB402001001207047AA
:1084A000002070470120704710B5054B044603605B
:1084B000406834F07DFE034B2046236010BD00BFB2
:1084C000D8260500A02D0500064B10B50446036014
:1084D000406834F06DFE044B2046236002F0E0FB60
:1084E000204610BDD8260500A02D050038B54068EF
:1084F0000D460A493EF09EFD044670B128463FF005
:10850000A0FD01210246234628463FF0E7F8054634
:1085100020463EF0EDFA284638BD38BD741D0500F2
:1085200010B582B0047841780023022268468DF8A5
:1085300000408DF801108DF802308DF804308DF870
:108540000320FEF7FDFC02B010BD00BF10B5C1F363
:10855000421301F01F01044603704170FFF7E0FF72
:10856000204610BD41780122007802FA01F1FEF7A1
:10857000F5BB00BF10B543780C4601210078994047
:108580001CB9FEF707FC204610BDFEF7F9FB20469C
:1085900010BD00BF014B0360704700BF00270500FE
:1085A00010B5034B0446036002F07AFB204610BD71
:1085B00000270500F0B50B6887B01A780C46232A0F
:1085C00071D053F80C3C022B6DD908460022474964
:1085D00002233AF058F9461C054664D023681B5C18
:1085E000232B60D00223204640492A463AF016F950
:1085F000431C074653D03D4920463A4602233AF0F1
:1086000042F906460130216850D08B5D232B4DD0B6
:1086100051F80C2C7B1B95424ED82A46214602A8C5
:108620003AF0ECFB02A904A801F0DAF9142039F0C1
:1086300047FE054602F0FCFCBDF81010BDF8122004
:10864000BDF814300120A874A981EA812B82721C24
:108650000523204626493AF0E1F8421C226818BF5B
:10866000C6EB000352F80C2C08BF0346964223D8F1
:108670002146324603A83AF0C1FB284603A93AF046
:1086800068F8039B1B4CA3F10C00A04217D1029B7E
:10869000A3F10C00A0421DD1284607B0F0BD21680F
:1086A00015483FF0B7F9002007B0F0BD13483FF080
:1086B000B1F9002007B0F0BD11483AF070FC53F852
:1086C000042C511E002A43F8041CE0DC01A93AF0F6
:1086D0003FF9DCE753F8042C511E002A43F8041C30
:1086E000DADC03A93AF034F9D6E700BF2027050009
:1086F00080270500640A001024270500882705004C
:108700006827050038B51546FFF754FF044618B131
:108710002846214600F032FA204638BDF0B583B035
:1087200014460F4601AA19491E4605463AF0AAFB0F
:1087300021463846FFF73EFF044660B18289338800
:108740009A420BD02368124AA3F10C00904212D136
:10875000204602F0A5FA284603B0F0BDC28973880E
:108760009A42EFD1B388028A9A42EBD12846214639
:108770003AF007FBE6E753F8042C511E002A43F8B1
:10878000041CE5DC01A93AF0E3F8E1E7D834050080
:10879000640A0010704700BF704700BF704700BFF9
:1087A000704700BF704700BF704700BF704700BFF1
:1087B000704700BF704700BF704700BF10B5034B44
:1087C0000446036002F052FD204610BDC02705009C
:1087D00010B5054B0446036002F048FD204602F048
:1087E0005FFA204610BD00BFC027050010B5044643
:1087F00002F04CFD201DFFF7C5F806480023FF21BD
:108800004FF0FF322060E1602261237663612046F1
:1088100010BD00BFC0270500002905DBC3689942D1
:10882000A8BF19460161704700210161704700BF70
:10883000036981F30801002BC16004DB9942B8BFD2
:108840000B4603617047002303617047C06870479F
:10885000837A4FF0FF3202619A070CD503F00103CF
:108860008B42037A4FF0010202FA03F2436801D00F
:108870009A617047DA617047026930B4FF2A034693
:1088800024D8002A2FD0FF2A40D044696FF0FF057A
:10889000B4F5007FB4BF20464FF400701C7EA842A0
:1088A000B8BF28465861A4B902447F2A5A612ADC1D
:1088B0009A7A90070AD502F00102A2421A7A4FF082
:1088C000010000FA02F25B6819D09A61084630BCD8
:1088D0007047A2F5807210440028D8BF0024586168
:1088E000D8BF1C76E4E7827A9507EFD512F0010F26
:1088F000027A4FF0010000FA02F25B68E5D130BC69
:108900000846DA61704701241C76D1E7827A940721
:10891000DCD512F0010F027A4FF0010000FA02F2EA
:108920005B68D2D0EBE700BF024900220160C26061
:10893000704700BFF827050010B5044A002304461D
:108940000260C36002F0ACF9204610BDF8270500B4
:10895000F0B587B09DF81440104F04F0FE04104E9F
:10896000ADF80800ADF80A10ADF80C20386801AA7F
:108970006FF3410405211D4604938DF814400196C0
:1089800000F0DAFE9DF8142012F0010003D09307E6
:1089900044BF049B2B6007B0F0BD00BFE402001091
:1089A000F827050070B586B09DF814500D4E0E4C9A
:1089B00005F0FE05ADF80800ADF80A10ADF80C2082
:1089C000306845F00205062101AA04938DF8145081
:1089D000019400F0B1FE9DF8140000F0010006B013
:1089E00070BD00BFE4020010F827050000220260FD
:1089F00042608260704700BF2DE9F04190E860005E
:108A0000B54282B080461CD0154F55F8044B3CB19E
:108A10002368A3F10C02BA4215D1204602F040F9B6
:108A2000AE42F2D1D8F800000023C8F80030C8F8F0
:108A30000430C8F8083008B102F032F902B0BDE8DD
:108A4000F0812846F0E753F8041C481E002943F83B
:108A5000040CE2DC104601A939F07AFFDDE700BF23
:108A6000640A001010B50446FFF7C6FF206808B17D
:108A700002F016F9204610BDF8B590E85000B44257
:108A80000F4602D10DE0A6420BD054F8045B3846E5
:108A900005F10C0106223EF0D7FE0028F3D128464E
:108AA000F8BD00252846F8BD2DE9F04F90E82002DA
:108AB0004D458BB00F4624D0012600E0464655F8C0
:108AC000044BD7F800A0E389B4F80CB00093238AD4
:108AD00006F10108019322680292A37C0393E37CD0
:108AE0000493A0683AF0C6FBCDE9060162685B46D4
:108AF0000892DAF80840384603493246A047A945AB
:108B0000DCD10BB0BDE8F08F00280500F8B5426855
:108B100003680446D31A9B100F4605D05A009342AF
:108B200026D96FF0030600E00426304639F0C8FB72
:108B3000054694E809001B1A9B109A003968AF1883
:108B400007D045F8231094E809001B1A9B109A00DF
:108B5000AF1823B1014628463EF08EFE2068043748
:108B600008B102F09DF82E44A66084E8A000F8BD8C
:108B7000B2F1804FD5D2DE00D7E700BF2DE9F04338
:108B800090E8500083B0B4428046019117D08946E6
:108B900001F10C0701E0A64211D0216838460C31E2
:108BA0000622254604343EF04FFE0028F3D1C5F8D6
:108BB00000900D483EF0E2FF03B0BDE8F083D8F826
:108BC00008309E420AD0019B16B13360D8F8046089
:108BD0000436C8F8046003B0BDE8F083404601A93C
:108BE000FFF794FFE8E700BF5C280500F8B542688E
:108BF00003680446D31A5B100F4605D05A0093420F
:108C000021D96FF0010600E00226304639F058FB0A
:108C1000054694E809001B1A5B1039885A00AF1802
:108C200018BF25F8131043B9023708B102F038F81D
:108C30002E44A66084E8A000F8BD014628463EF018
:108C40001BFE2068F0E7B2F1004FDAD29E00DCE7AD
:108C50002DE9F04190E89000BC4282B0884602D1F4
:108C600014E0A74212D054F8045B2E8A9642F8D141
:108C7000AE894645F5D1596898688E1C814208D066
:108C8000E88901B10880A7425E60ECD102B0BDE87E
:108C9000F081184605F10E0101920093FFF7A6FF3F
:108CA000009B019ADDE700BF38B5094B094D04462A
:108CB000036002460721286800F094FD28682246D8
:108CC000082100F08FFD204602F0D0FA204638BD82
:108CD00090280500E402001010B50446FFF7E4FFF9
:108CE000204601F0DDFF204610BD00BF012919D04C
:108CF00041B1CB0715D490F83830022202FA03F3C1
:108D000019420ED0837E9A070BD513F0010F037E14
:108D10004FF0010202FA03F2436901D19A617047F0
:108D2000DA617047837E9A07FBD5027E13F0010F4C
:108D300001FA02F1436914BF9961D961704700BF1C
:108D400001B17047837E9A070AD513F0010F037EA5
:108D50004FF0010202FA03F243690CBF9A61DA6133
:108D6000038F6FF349230387704700BFF8B50446AC
:108D70001D4616460F4602F089FA334A234643F849
:108D8000042B97E8030083E8030004F10C0396E842
:108D9000030083E8030004F1140395E8030083E86B
:108DA00003006879297902F04FFB0023E362228FE8
:108DB000264863F34922228794F83910A27E244E74
:108DC0004FF07E57002541F00401A0629007236315
:108DD00027626662656384F839100AD5237E12F033
:108DE000010F4FF0010202FA03F263690CBF9A61AE
:108DF000DA61A37A99070AD513F0010F237A4FF0AD
:108E0000010202FA03F2636814BF9A61DA61A37C7B
:108E10009A070AD513F0010F237C4FF0010202FAE2
:108E200003F2E36814BF9A61DA61238F20466FF37F
:108E300008232387072102F02FFA2046082102F099
:108E40002BFA2046F8BD00BF902805000000C07F27
:108E50000000484210B5044601620846616B3AF0D2
:108E60009DFE3BF073FE2063E06210BD10B504462A
:108E700041630846216A3AF091FE3BF067FE2063A9
:108E8000E06210BD41630263C2627047036B4163DD
:108E90001A440263704700BF10B504460846216AB1
:108EA0003AF07CFE3BF052FE236BC01A10BD00BFAF
:108EB00038B5837E04469A070D460FD54269017E78
:108EC000506903F00103C84000F00100984205D04A
:108ED000002B47D0012303FA01F1916194F8393056
:108EE00003F00103AB4215D0238FA27C65F3082366
:108EF000900723870BD5237C02F00102AA424FF092
:108F0000010202FA03F2E36814BF9A61DA610120F8
:108F100038F038F8A37A99070AD513F0010F237AAD
:108F20004FF0010202FA03F263680CBF9A61DA6142
:108F3000032038F027F8A37A9A070AD513F0010F17
:108F4000237A4FF0010202FA03F2636814BF9A61B8
:108F5000DA61E26A002D0CBF01234FF0FF331344A6
:108F6000E36238BD012303FA01F1D161B6E700BF26
:108F7000F8B5046900F10806B4420F464FF0000549
:108F80000DD02069394603685B6998478542B8BFB0
:108F90000546204639F042FAB0420446F1D128464F
:108FA000F8BD00BFF8B5314B0446436300F1B4018E
:108FB00000F14803002243F80C2C43F8082C43F836
:108FC000042C0C338B42F6D194F8A830284A03F0D5
:108FD000FD036FF3C30384F8A8304FF48C70146062
:108FE00039F06EF92349244A4FF41653054606F02A
:108FF00055FA2560102039F063F9054601F0BCFBF5
:1090000028466561012101F029FB206810B1036841
:109010005B689847002525601C2039F051F91749F5
:10902000034600F108020160026142610572C560F9
:10903000856113496360012204F1340039F034FD85
:10904000104A4FF2FF03D1680B4043F0BF6343F473
:109050000033D36035F004FB032800F29581DFE88C
:1090600010F04F0171012D01130000BF700A0010B4
:10907000E402001002C0092003C00920C82805002E
:10908000E828050000ED00E042F6AA22002344F2A1
:10909000ED11606901F01AFB4FF4165102F0CCF8A3
:1090A00001F0FCFFB94B4FF48C710646186801F0D3
:1090B000DBFC054630463AF04DFFB5490346B54A5C
:1090C000284606F0EBF925602B46002B00F078814E
:1090D0000022134660694CF6DF1101F0F7FA002117
:1090E00002F0AAF802F092F894F8A83080F001009B
:1090F000002260F3000384F8A8306069134648F248
:10910000AE0101F0E3FA002102F096F802F07EF8D9
:1091100094F8A830002260F3820384F8A8306069D4
:10912000134645F68B3101F0D1FA012102F084F8A3
:1091300002F06CF8236894F8A820196860F3041210
:1091400084F8A82018468A689047282039F0B8F893
:10915000054601F087FE2B68A5629B682846984764
:109160003C2039F0ADF8054602F0B2FAE5624FF462
:10917000C27039F0A5F80646FEF786FF864A4FF220
:10918000FF01D068854B014041F0BF614FF0100CEA
:109190004FF0080E282541F40031202718202663BF
:1091A000D16083F801C383F802E383F8037382F884
:1091B000220083F8165383F8185393F8052345F2D9
:1091C0009E51D20818BF83F80553744B93F80623B9
:1091D000D2081CBF282283F80623704B93F807237C
:1091E000D2081CBF282283F807236C4B93F808236E
:1091F000D2081CBF282283F8082300221346606986
:1092000001F064FA664902F017F801F047FF3AF0FE
:10921000C7FE00221346A0634AF25D51606901F067
:1092200055FA012102F008F801F038FF0546A06B5D
:109230003AF05CFCE66A0146304602F00BFA294639
:10924000E06A02F025FA282039F03AF8054609F0DC
:1092500043FE2B68A5619B6828469847182039F083
:109260002FF8054605F036FF2B68A5609B68284659
:1092700098474FF4AC7039F023F8054608F06AFBC4
:109280002B68E5609B6828469847042039F018F859
:10929000054601F0FBFF434B28462B60256225F075
:1092A0006BFE182039F00CF8054606F053F92561DD
:1092B000012039F005F8E0612046F8BD42F6AA2207
:1092C000002344F2ED11606901F000FA4FF41651E9
:1092D00001F0B2FF01F0E2FE2C4B4FF48C71064618
:1092E000186801F0C1FB054630463AF033FE2E49BE
:1092F00003462E4A284606F0D1F825602B46E4E6C0
:1093000042F6AA22002344F2ED11606901F0DEF971
:109310004FF4165101F090FF01F0C0FE1B4B4FF4CB
:109320008C710646186801F09FFB054630463AF0FE
:1093300011FE1F4903461F4A284606F0AFF8256074
:109340002B46C2E642F6AA22002344F2ED116069E0
:1093500001F0BCF94FF4165101F06EFF01F09EFED2
:109360000A4B4FF48C710646186801F07DFB0546E8
:1093700030463AF0EFFD10490346104A284606F001
:109380008DF825602B46A0E623689EE6FC020010BF
:1093900000C0092001C0092000ED00E000E100E06C
:1093A000A0860100888B05000AC009200BC0092097
:1093B00002C0092003C009200FC0092010C00920E5
:1093C00042F6AA2244F2ED11606901F07FF94FF4F0
:1093D000165101F031FF01F061FE094B4FF48C7121
:1093E0000646186801F040FB054630463AF0B2FDEB
:1093F00004490346044A284606F050F8256067E60B
:10940000FC02001002C0092003C009202DE9F0472A
:10941000AB4BB6B0036080468A464FF44C4044F6EE
:109420008A5100220DF11F03FFF792FA08B98DF857
:109430001F004046A349012239F024FC9AF8A830C5
:109440009E0700F130819DF81F20002A40F03181F5
:109450001D0740F1838040469B49052239F012FCEC
:10946000DAF80C30D3F80091CDF83890D3F8FC60DE
:109470000F96D3F8F800109093F83430DB0740F1E2
:10948000FC8092493AF03EFC39F0F4FE04460D4669
:1094900030468E493AF036FC39F0ECFE06460F466F
:1094A00048468A493AF02EFCCDE90045CDE90267ED
:1094B00039F0E0FE0DF15809CDE90401844A80211C
:1094C00048463EF0BFFC834904460522404639F039
:1094D000D9FB4946224639F0D5FB11A80EAADAF885
:1094E0000C1006F0EFFADAF80C30139893F83430D9
:1094F000DA0740F1CD8075493AF004FC39F0BAFE44
:1095000004460D46129871493AF0FCFB39F0B2FE60
:1095100006460F4611986D493AF0F4FBCDE9004537
:10952000CDE9026739F0A6FE6B4ACDE90401484651
:1095300080213EF087FC694904460522404639F007
:10954000A1FB4946224639F09DFB4046644903226F
:1095500039F098FB404636B0BDE8F087DAF81800DD
:1095600009F090FC04464046002C40F0C1800422E3
:109570005C4939F087FBDAF80C601194B5681294F5
:109580002F681394F86A149415943AF0B3FA396A70
:109590003AF0B8FB6C681190E06A3AF0ABFA216AD5
:1095A0003AF0B0FBAC681290E06A3AF0A3FA216A94
:1095B0003AF0A8FB736811A91A6813901846D3688B
:1095C00008AA9847DAF80C30089893F83430DC078A
:1095D00040F19E803D493AF095FB39F04BFE044640
:1095E0000D46099839493AF08DFB39F043FE06469D
:1095F0000F460A9835493AF085FBCDE90045CDE99B
:10960000026739F037FE0DF15809CDE90401304AFF
:10961000802148463EF016FC2E490446052240466D
:1096200039F030FB2246494639F02CFB089B0A9D55
:10963000099CDAF80C100BA80EAA10930E950F9443
:1096400006F040FADAF80C300D9893F83430D90768
:1096500053D51E493AF056FB39F00CFE04460D4630
:109660000C981A493AF04EFB39F004FE06460F46B4
:109670000B9816493AF046FB50E739F0FBFD0446DB
:1096800030460D4639F0F6FD06460F4648460BE7D4
:1096900039F0F0FD044612980D4639F0EBFD064610
:1096A0000F4611983AE740460F49062239F0EAFA88
:1096B000D6E640460D49052239F0E4FAD0E600BF6F
:1096C000700A0010EC280500002905003333CB4157
:1096D000182905002C290500342905004829050012
:1096E0005029050010290500F0280500F82805007C
:1096F0000D49052239F0C6FAB2E639F0BBFD044641
:109700000C980D4639F0B6FD06460F460B9805E756
:1097100039F0B0FD044609980D4639F0ABFD064618
:109720000F460A9869E700BF0829050008B50B68CD
:1097300008469B68984708BD2DE9F04F072983B07C
:109740008B46824690463CD0012301930BEB4B02A3
:1097500092000AF13C01881846688C58B4421CD02B
:109760001F4F07EBCB02556805F001096D1006E0AD
:10977000284457F83B2041469047A6420DD054F864
:10978000040BB9F1000FF3D0415957F83B2028449E
:109790008A5841469047A642F1D1BBF1070F02D04B
:1097A00003B0BDE8F08F9AF8A8309B07F8D5019B6D
:1097B000002BF5D1DAF80C0003B0BDE8F04F06F04D
:1097C00071BB90F8A820D8F1010138BF002161F3E6
:1097D000410280F8A820806909F054FB0190B5E7A8
:1097E000282D050001EB410138B53C308B00C51830
:1097F0006C68C058A0420DD00368934218BF031D87
:1098000003D108E00168914205D0A342184603F154
:109810000403F7D138BD011D8C4206D0631A9A109B
:1098200003D092003EF028F86C68043C6C6038BDB0
:1098300070B50C46064609B90AE02C463046E16888
:10984000FFF7F6FFA568204601F02AFA002DF4D1B3
:1098500070BD00BF054B10B5044640F8043BE168FD
:10986000FFF7E6FF024B2046236010BDC828050025
:10987000A02D0500074B10B5044640F8043BE168F5
:10988000FFF7D6FF044B2046236001F009FA20467B
:1098900010BD00BFC8280500A02D0500F8B542681E
:1098A00003680446D31A9B100F4605D05A00934212
:1098B00026D96FF0030600E00426304638F000FD9C
:1098C000054694E809001B1A9B109A003968AF18E6
:1098D00007D045F8231094E809001B1A9B109A0042
:1098E000AF1823B1014628463DF0C6FF2068043773
:1098F00008B101F0D5F92E44A66084E8A000F8BDB7
:10990000B2F1804FD5D2DE00D7E700BF00B501EB42
:1099100041013C3000EB81004368816883B08B4299
:10992000019207D00BB11A6043680433436003B05F
:109930005DF804FB01A9FFF7B1FFF8E770B4056813
:109940002878F8B10024104E2146084480FB0623F5
:10995000C217C118C2EBE111C1EB0121411A0C443D
:1099600084FB0623E2172344C2EBE313C3EB032378
:1099700015F8010FE31A89B29CB20028E5D141EA3B
:10998000042080B270BC70478180808070B40278FF
:109990000AB30024114E21468D1885FB0623EA17D1
:1099A000E918C2EBE111C1EB0121691A0C4484FBF7
:1099B0000623E2172344C2EBE313C3EB032310F89F
:1099C000012FE31A89B29CB2002AE5D141EA0424AE
:1099D000A0B270BC70471046FBE700BF818080805A
:1099E0002DE9F04F0B68002753F80C3C87B08846F0
:1099F0000190078047808780002B63D04E4CBA4689
:109A0000012340464D49524638F008FF4C4B05466D
:109A10000493431C5DD0D8F80020CAEB050352F82C
:109A20000C2C924579D805AE52463046414639F065
:109A3000E5F904A8314638F08CFE059BDFF8089163
:109A4000A3F10C0048455DD1DDF810C09CF8003052
:109A500043B34FF0000B5946604601EB030A8AFB03
:109A600004230AEB03014FEAEA73C3EBE111C1EBF4
:109A70000121C1EB0A018B448BFB04230BEB030296
:109A80004FEAEB73C3EBE212C2EB022210F8013F84
:109A9000C2EB0B0289B21FFA82FB002BDDD141EA37
:109AA0000B218BB2019AACF10C00D3536A1C1CD071
:109AB000484505F1010A33D1D8F8003053F80C3C81
:109AC0009A4502D307B0BDE8F08F0237062FF9D0D0
:109AD00096E7D8F8003053F80C3C53451DD305AE3B
:109AE0005246304641462B46A1E74845EAD05CF84D
:109AF000043C5A1E002B4CF8042CE3DC314638F0B1
:109B000027FFDFE753F8042C511E002A43F8041CFA
:109B10009ADC03A938F01CFF96E70A4839F03FFAAF
:109B20005CF8043C5A1E002B4CF8042CC4DC314673
:109B300038F00EFFC0E700BF8180808000C80400BD
:109B4000700A001068270500640A0010202804D05D
:109B5000B0F109035842584170470120704700BFD7
:109B6000F0B50F4E83B006600C68054654F80C7CC7
:109B70002744BC4201D10FE02E6814F8010B3FF0DE
:109B800061FDC0B256F80C1C00220090012328464B
:109B900038F05CFFA742EFD1284603B0F0BD00BF0C
:109BA000700A001070B584B00C4602AA1C49064623
:109BB00003A839F067F903990022204651F80C3CBC
:109BC00038F061FE421C18BF00250FD0014601226B
:109BD000144B0095204639F077F90399204651F847
:109BE0000C3C002238F04FFE431CEFD10E4B039A81
:109BF0002168A3F10C05A2F10C00A842316023609A
:109C000002D1304604B070BD52F8043C591E002BFE
:109C100042F8041CF5DC02A938F09AFEF1E700BF17
:109C200054290500D8340500700A001070B50C46A0
:109C3000012384B0054621492046002238F0EEFD7C
:109C4000431C06461ED00022334602A8214639F0A6
:109C5000D5F82368721C53F80C3C9A4220D8214650
:109C600003A839F0CBF8204603A938F072FD039B16
:109C7000134AA3F10C00904215D1029B28462B6099
:109C800004B070BD214603A839F06FF820460D4995
:109C9000002238F009FF039B28462B6004B070BDFA
:109CA000094839F07CF953F8042C511E002A43F876
:109CB000041CE2DC01A938F04BFEDEE74833050066
:109CC000640A0010D83405006827050030B50D4639
:109CD000012383B0044611492846002238F09EFD36
:109CE000431C0FD02B68421C53F80C1C4B1C8A429F
:109CF000C0EB03030ED82946204639F07FF82046F2
:109D000003B030BD2046064901AA39F0BBF8204611
:109D100003B030BD034839F042F900BF48330500B5
:109D2000D83405006827050010B5054900683DF0E6
:109D300081F904463CF0DCFE201C18BF012010BD58
:109D4000D4A6050010B590B14FF0804401220E4B0F
:109D500022611868000939F0C9FE3AF021F903219F
:109D6000AA225523606021702272237210BDBFF3B6
:109D70004F8F064A064BD16801F4E0610B43D36074
:109D8000BFF34F8FFEE700BF9801001000ED00E029
:109D90000400FA05F0B5A14D85B02B680C460746C6
:109DA00003F1340102A838F0E0FF236853F80C2CCB
:109DB000002A00F09A8053F8042C002A03DB204686
:109DC00038F02CFE23681A782F2A00F0CB80944DAF
:109DD00000220323214603A839F010F803A8914973
:109DE00038F06AFD039B0646A3F10C02AA4240F03C
:109DF000C780002E37D1236853F80C3C022B40F269
:109E0000CC804FF0FF332146032203A838F0F6FF41
:109E1000204603A938F09DFC039BA3F10C00A84247
:109E200040F0BE8080494FF0FF32012302A838F095
:109E30000FFD02A90346002203A838F0DFFF02A8A5
:109E400003A938F086FC039BA3F10C00A842BFD005
:109E500053F8042C511E002A43F8041CB8DC01A955
:109E600038F076FDB4E700220223214603A838F03B
:109E7000C5FF03A86D4938F01FFD039B0646A3F1FB
:109E80000C02AA4240F0BA80002E35D0029B53F853
:109E9000042C53F80C1C002A01F1FF3603DB02A846
:109EA00038F0BCFD029B9B5D02A92F2B60D003A85C
:109EB00038F05BFF2F22012103A838F01DFF03A813
:109EC000214638F0B6FE5A4A03683B600260039BA5
:109ED000A3F10C00A84240F08580029BA3F10C0086
:109EE000A84269D1384605B0F0BD296838463431FA
:109EF00038F03BFF4A4DF0E7236853F80C3C012B48
:109F00004BD94FF0FF332146022203A838F076FFE9
:109F1000204603A938F01DFC039BA3F10C00A842C6
:109F200055D141494FF0FF32012302A838F090FC8F
:109F300002A90346002203A838F060FF02A803A983
:109F400038F007FC039BA3F10C00A8429ED053F805
:109F5000042C511E002A43F8041C97DC01A938F098
:109F6000F7FC93E7324A3B60A2F10C052260B4E7AC
:109F7000384638F0FAFE3846214638F05AFEACE74B
:109F800053F8041C481E002943F8040C3FF731AF76
:109F9000104601A938F0DCFC2BE7264838F0FFFF1B
:109FA00053F8042C511E002A43F8041C3FF73AAF23
:109FB00001A938F0CDFC35E753F8042C511E002AD6
:109FC00043F8041C8EDC03A938F0C2FC8AE753F87E
:109FD000042C511E002A43F8041CA2DC01A938F00D
:109FE000B7FC9EE753F8042C511E002A43F8041CCA
:109FF0003FF773AF01A938F0ABFC6EE753F8041CD0
:10A00000481E002943F8040C3FF73EAF104601A953
:10A0100038F09EFC002E7FF439AF6DE7E4020010AB
:10A02000640A001074290500E82805004C3F05006B
:10A03000700A0010682705002DE9F04191E8100131
:10A04000444582B0074616461FD002B308340020AC
:10A0500001E0864216D914F8082C451C3A5454F8ED
:10A06000040C39F007F907EB050E731BCDE900016D
:10A07000084A704619463DF0E5FEA045284404F123
:10A080000804E6D102B0BDE8F0810020FAE71046EE
:10A09000F8E700BF7829050030B585B00D4603AA62
:10A0A0001749044638F0EEFE052D23680CDC3435E4
:10A0B000EDB253F80C1C204600950022012338F025
:10A0C000C5FC204605B030BD392253F80C1C204693
:10A0D00000920123002238F0B9FC204609490122F0
:10A0E00038F0D0FD2B350368EDB253F80C1C00227C
:10A0F0000095012338F0AAFC204605B030BD00BF12
:10A100008029050000C8040070B5054636F012F835
:10A11000074E044602E03068FFF70EFB36F00AF8FF
:10A12000001BA8424FF003014FF00002F3D370BDB3
:10A13000E40200104FF47A7303FB00F0FFF7E4BF72
:10A14000F8B5426803680446D31A9B100F4605D041
:10A150005A00934221D96FF0030600E004263046EE
:10A1600038F0AEF8054694E809001B1A9B103968D0
:10A170009A00AF1818BF45F8231043B9043708B147
:10A1800000F08EFD2E44A66084E8A000F8BD0146D4
:10A1900028463DF071FB2068F0E7B2F1804FDAD23B
:10A1A000DE00DCE7F8B5426803680446D31A9B106A
:10A1B0000F4605D05A00934221D96FF0030600E004
:10A1C0000426304638F07CF8054694E809001B1A4E
:10A1D0009B1039689A00AF1818BF45F8231043B98F
:10A1E000043708B100F05CFD2E44A66084E8A000AE
:10A1F000F8BD014628463DF03FFB2068F0E7B2F18C
:10A20000804FDAD2DE00DCE72DE9F04742680368D0
:10A2100082B0C3EB02095FEAA90907460E4648D09F
:10A220004FEA4903994555D96FF00309484638F07C
:10A2300047F897E83000291B891000EB810380461E
:10A2400000F1040A23B13368254A40F82130326016
:10A25000AC4231D0231DC3EB050C4FEA9C0C04F13A
:10A2600008061F4806EB8C06424622B153F8041C30
:10A27000116043F8040C0433B34202F10402F4D138
:10A2800008EB8C0C174E0CF1080A54F8043BA3F1B0
:10A290000C02B24212D1A542F7D1386808B100F0E1
:10A2A000FFFC08EB0903BB6087E8000502B0BDE8CE
:10A2B000F0874FF00409B9E72046EFE753F8041C94
:10A2C000481E002943F8040CE5DC104601A938F0CB
:10A2D0003FFBE0E7B3F1804FA6D24FEAC909A5E7FB
:10A2E000700A0010640A00102DE9F04FDFF80C81AD
:10A2F000002385B082460F461646036043608360A4
:10A30000A8F10C093B78B3424FD0002B4DD07B1CF9
:10A3100000E024B11D4613F8014BB442F9D1AF421D
:10A3200054D0002F3CD0C7EB050B5846002101AAA2
:10A3300038F0E2FABBF1010F044600F10C0328D11A
:10A340003A7822734C452C4F44D1DAF80420DAF8DD
:10A35000081003938A4233D01AB11360274BCDF80B
:10A360000C800432CAF80420A3F10C00B84238D1A2
:10A370002B786F1C002BC5D1504605B0BDE8F08F7F
:10A380002846294601AA38F0B7FAAB46044600F140
:10A390000C03184639465A463DF065FA0346D1E7A4
:10A3A000002DEDD0164838F0F4FDDAF80420DAF884
:10A3B0000810124B8A423D460393A3F10C07CBD100
:10A3C000504603A9FFF720FF039BCDE70B4BA3F1FA
:10A3D0000C07BAE70022C4F800B0A26003F80B2013
:10A3E000B3E753F8042C511E002A43F8041CBFDCC9
:10A3F00002A938F0ADFABBE7640A0010700A001039
:10A4000084290500F0B585B004462C2201A8FFF789
:10A410006BFF019D029E0023B54223606360A36031
:10A4200029D055F8040B00213EF0EEFC6368A268C9
:10A43000009093421AD01A1D03B118606260AE42B8
:10A44000EFD10198029E86420AD0114F054655F879
:10A45000043BA3F10C00B8420FD1AE42F7D10198F2
:10A4600008B100F01DFC204605B0F0BD204669464D
:10A47000FFF766FEE3E72846F2E753F8042C511E87
:10A48000002A43F8041CE8DC694638F061FAE4E786
:10A49000640A0010F0B585B00446174601A82C22C6
:10A4A000FFF722FF019D029E0023B54223606360F7
:10A4B000A3602AD0002155F8040B3A463EF03EFD39
:10A4C0006368A16800908B421AD0191D03B118600F
:10A4D0006160AE42EED10198029E86420AD0114FD1
:10A4E000054655F8043BA3F10C00B8420FD1AE422B
:10A4F000F7D1019808B100F0D3FB204605B0F0BDBC
:10A5000020466946FFF74EFEE3E72846F2E753F898
:10A51000042C511E002A43F8041CE8DC694638F07C
:10A5200017FAE4E7640A0010FCF700BD08B5032140
:10A5300000F0B2FEBDE80840FCF7F8BC10B5034BD4
:10A540000446036000F092FE204610BDB8290500C5
:10A5500010B5054B0446036000F088FE204600F06D
:10A560009FFB204610BD00BFB829050070B51546F9
:10A570000E46044600F08AFE0A4B291C18BF012132
:10A5800023600020FCF79CFC3046FCF7B1FCFCF794
:10A59000CDFC2DB9044B01210822196083F800235A
:10A5A000204670BDB829050000E100E008B50E4B5B
:10A5B0001B6893F8A830DB070FD500210B48FDF787
:10A5C000D9FF01210A48FDF7D5FF00210948FDF711
:10A5D000D1FF09480121FDF7CDFFFCF79FFCFCF7F7
:10A5E000A5FC00BE08BD00BFE4020010A4020010DC
:10A5F000A6020010A8020010AA02001010B50368FD
:10A600000A4A0446A3F10C00904282B002D12046CF
:10A6100002B010BD53F8042C511E002A43F8041C4C
:10A62000F5DC01A938F094F9F1E700BF640A0010E5
:10A630000B460068114647F26932FEF709BB00BFBE
:10A6400038B5046805462CB12046FEF70BFA2046C3
:10A6500000F026FB00232B6038BD00BFF8B50C4688
:10A660000546FFF7EDFF0C2037F02AFE0746FEF700
:10A67000BDF92F606CB16C68AE68B44209D0394640
:10A6800000E0296854F8040B03689B689847A642C9
:10A69000F7D1F8BD10B504684CB12046FEF7ECF9CF
:10A6A00000B110BD064800F0D9FC0548F9E7054B9C
:10A6B00005491B68586803689B689847204610BD89
:10A6C000E8020010E4020010E829050000B583B09C
:10A6D000ADF800106946ADF80220ADF80430FFF780
:10A6E000D9FF03B05DF804FBF8B54268036804467F
:10A6F000D31A9B100F4605D05A00934226D96FF00B
:10A70000030600E00426304637F0DAFD054694E8FB
:10A7100009001B1A9B109A003968AF1807D045F83A
:10A72000231094E809001B1A9B109A00AF1823B15C
:10A73000014628463DF0A0F82068043708B100F033
:10A74000AFFA2E44A66084E8A000F8BDB2F1804FB5
:10A75000D5D2DE00D7E700BF38B54368846802462B
:10A76000A34206D009680BB11960436804335360F3
:10A7700038BDFFF7B9FF38BD2DE9F041002306468B
:10A7800084B043608360C360054646F8043B1020F4
:10A7900037F096FD04AC07466E4903F0B5FC44F86B
:10A7A000047D30462146FFF7D7FF01AA6A492046BB
:10A7B00038F068FB2046FFF7B7FA039B674FA3F119
:10A7C0000C02BA42804640F0B7802046B8F1000F34
:10A7D0005ED0614901AA38F055FB102037F070FDBA
:10A7E00021465F4A804602F069FF039BA3F10C00FB
:10A7F000B84277D1B8F1000F05D030462146CDF8E8
:10A800000C80FFF7A9FF01AA5649204638F03AFB11
:10A810002046FFF789FA039B8046A3F10C02BA4257
:10A8200049D1B8F1000F1ED04E4901AA204638F098
:10A8300029FB102037F044FD21464B4A804602F0A8
:10A840003DFF039BA3F10C00B84240D1B8F1000FCB
:10A8500005D030462146CDF80C80FFF77DFF284615
:10A8600004B0BDE8F08101AA4049204638F00AFB57
:10A870002046FFF759FA039B8046A3F10C02BA4227
:10A880004BD1B8F1000FEAD001AA20463749CEE7F4
:10A8900001AA374938F0F6FA2046FFF745FA039B3C
:10A8A0008046A3F10C02BA4227D1B8F1000FAAD01A
:10A8B00020462F498EE753F8041C481E002943F810
:10A8C000040CAEDC104602A938F042F8A9E753F8B0
:10A8D000042C511E002A43F8041CB7DC02A938F0EE
:10A8E00037F8B3E753F8042C511E002A43F8041C30
:10A8F00080DC02A938F02CF87CE753F8041C481ED1
:10A90000002943F8040CD0DC104602A938F020F8E6
:10A91000B8F1000F3FF477AFCAE753F8041C481EA4
:10A92000002943F8040CACDC104602A938F010F8FA
:10A93000B8F1000F93D0A7E753F8041C481E002974
:10A9400043F8040C3FF741AF104602A938F000F875
:10A950003BE700BF242A05002C2A0500640A0010EA
:10A960003C2A0500582A0500B4260500642A050083
:10A97000442A050010B5054C204600F059FB20463E
:10A980000349044ABDE8104037F0BFBCE80200109C
:10A99000FDA50000C8000010002202604260826035
:10A9A000C260704708B5D0F8440203689B689847B6
:10A9B00008BD00BF08B5D0F8440203689B699847FA
:10A9C00008BD00BF08B5D0F8440203681B6898476B
:10A9D00008BD00BF08B5D0F8440203685B6898471B
:10A9E00008BD00BF08B5D0F8440203681B6A984749
:10A9F00008BD00BF08B5D0F844020368DB6898477B
:10AA000008BD00BF38B50446154602F0AFFC034B45
:10AA1000C4F844522360204638BD00BF802A050098
:10AA200010B50021044690F840020EF0CDFF94F8D6
:10AA3000400204F110010EF0C7FF002010BD00BF5E
:10AA4000F0B4084C002725684FEA122C41600281BF
:10AA50008F70CF7081F801C00A7005602060F0BC73
:10AA6000704700BF040300108B0718BF21F00301DB
:10AA70002DE9F00118BF0431456801F1040C1FFAFB
:10AA80008CFC2B4610E093F801809A7841EA08216B
:10AA900041EA024141EA046161450A461EDA018940
:10AAA00013446A18934215D8DA781978D70902F056
:10AAB0007F041646E7D05E789C7841EA062141EA99
:10AAC000044102F07F0241EA0262018913446A18DC
:10AAD0009342E9D90020BDE8F001704746F08006B6
:10AAE0008C45DE7027DA03EB0C02D478CCEB010145
:10AAF00067F3C71404F08004C1F306652543C1F36E
:10AB00000726C1F3074403F80C10D57056709470F3
:10AB1000DC782CF0004C04F0800400214FEA1C2566
:10AB200083F800C05D70DC70997044680189121B65
:10AB30008A4200DB00BEBDE8F001181D704700BF6F
:10AB40002DE9F00311F8013C11F8034C11F8042C25
:10AB500011F8025C6FF3C71342EA042242EA05428D
:10AB600003F07F0442EA04620F1F01F8013CBB18A6
:10AB7000DC78E50925D1456806895D1BB54200F3FF
:10AB80008D80BE5C93F801C09D7846EA0C2343EAB1
:10AB9000054304F07F0443EA046411F8015C224495
:10ABA000C2F3066325F07F051D43C2F30724C2F3F9
:10ABB000074301F8042C01F8015C01F8034C01F88B
:10ABC000023C466833787578B278F47843EA052316
:10ABD00043EA024304F07F0443EA0464324616E089
:10ABE00004891A46A54206EB040C54DA1D7893F842
:10ABF000019093F80280DC7845EA092545EA08458A
:10AC000004F07F0455EA046445D0634543D2131928
:10AC1000951BBB422544E3D1D378DE09C3F3C015AD
:10AC200039D111F8046C11F8039C11F8028C11F859
:10AC300001CC46EA092646EA08460CF07F0C46EAB3
:10AC40000C66344423F07F08C4F3066CC4F3072673
:10AC5000C4F307432B432C4348EA0C0C2E4382F8E1
:10AC600003C056709370147011F8043C11F8032C53
:10AC700011F8024C11F8011C43EA0222436842EA2F
:10AC8000044201F07F0142EA0161FB1A02890B4490
:10AC9000934200DB00BEBDE8F003704700BE70E7E2
:10ACA000084B01461B684BB15A689142FAD3188988
:10ACB00002449142F6D21846FFF742BF084632F0EE
:10ACC00077BA00BF040300102DE9F04F0A6844680A
:10ACD00080469568084683B00F462346B8F808209A
:10ACE00024494FF00009A847DFF898B0D8F804606D
:10ACF000CA4602E0042D33D92C44E2783B68D209DD
:10AD00001D4A9D6808BF5A46009260782378A17852
:10AD1000E27843EA002343EA014302F07F0243EA78
:10AD200002620192A31B154922463846A8472178A2
:10AD30006578E378A27841EA0525D8F8046045EA09
:10AD4000024503F07F0245EA0265DB09C6EB040217
:10AD5000B8F808302A4408BFA9449A42AA44C9DB7B
:10AD6000396852468C684B4638460549A04703B0BF
:10AD7000BDE8F08FC82A0500B82A0500E82A0500BA
:10AD80000C2B0500C02A05004368F0B405891C4659
:10AD9000002002E0042A14D91344D9785F78CA0944
:10ADA0001A789E7842EA072201F07F0142EA0642C1
:10ADB00042EA0162C4EB0301114408BF8018A942B2
:10ADC000E8DBF0BC704700BF032100F065BA00BFAC
:10ADD00010B5064B04464068236008B1FFF760FFDA
:10ADE000204600F043FA204610BD00BF382B050076
:10ADF00038B5104D04462B6893F8A830DB0708D50A
:10AE00000D4B0E4819884A1CC1F300311A80FDF71A
:10AE1000B1FB72B6636A53B1636A013B636262B6A7
:10AE2000042128680022BDE83840FEF785BC62B6E0
:10AE300038BD00BFE40200100C030010A80200108F
:10AE400010B5074B04464068236008B1FFF728FFA0
:10AE5000204600F00BFA2046FFF722FF204610BDE7
:10AE6000382B0500F0B585B0044600F00FFA294AEA
:10AE7000002304F1180522606360A360E3602846A4
:10AE8000FCF780FD244B254901AA03A81C6037F07C
:10AE9000F9FF284603A9FCF75DFF83799B0707D5D7
:10AEA000037901229A400368196821EA02021A60B4
:10AEB000FCF766FE039B1A4AA3F10C0090421ED1D8
:10AEC0001849194BD1F8C46003250022174846F4ED
:10AED0008006C1F8C4605D615A600168144E89083B
:10AEE000A6FB010605202061B60801272046666101
:10AEF0009E615D605F602162626205B0F0BD53F8E3
:10AF0000042C511E002A43F8041CD9DC02A937F096
:10AF10001FFDD5E7382B050008030010682B05003E
:10AF2000640A001000C00F400000094098010010A2
:10AF3000CDCCCCCC0349044B0120082248601A60D8
:10AF4000704700BF0000094000E100E0074A30B44C
:10AF50001268074B9208B2FBF1F10325012441610D
:10AF600099615D605C60026230BC704798010010BE
:10AF700000000940F8B5446885680646AC4241695E
:10AF800002D112E0A54210D054F8043B5A69521A7B
:10AF9000002A5A61F6DA18691F6802445A61BFB183
:10AFA0000020B847A5427169EED1336A591A0029C9
:10AFB00031621BDBB37F9A0708D5B169327F4969DB
:10AFC00021FA02F25340DB0700D5F8BD00BEF8BD00
:10AFD0005A68002AD6D09F68D86887B1C10710D4B4
:10AFE00002EB60000021B8477169CBE7074A736A3A
:10AFF0001268013301EB920131627362DAE7C30731
:10B00000C0D5401013581044DF59EBE798010010E9
:10B01000054B1A68D20703D51A6842F001021A607C
:10B02000024B1868FFF7A6BF000009400803001094
:10B0300010B5084900220023044601608360827431
:10B04000C2748281C28102824260034937F02CFDC2
:10B05000204610BD700A0010D834050000220021DF
:10B0600081608274C2748281C2810282426001491D
:10B0700037F01ABDD8340500837C10B5044633B9C7
:10B08000044B05491B68586803689B68984720462D
:10B0900010BD00BFE4020010702B0500F0B5837CEA
:10B0A00087B004460BB9C37C03BB0023214605A827
:10B0B000039337F05AFE04A805A9FEF773FD059B1C
:10B0C0001F4DA3F10C00A8422FD1049E03A93046C6
:10B0D0003DF09AFE039B0746B3420AD9049BA3F1B5
:10B0E0000C02AA4215D1384607B0F0BD806807B0FF
:10B0F000F0BD144BB4F80EE01B68268A586822682D
:10B100000168A389CDF800E001968C680E49A0473C
:10B11000E4E753F8041C481E002943F8040CE2DC61
:10B12000104605A937F014FCDDE753F8042C511E36
:10B13000002A43F8041CC8DC02A937F009FCC4E764
:10B14000640A0010E4020010CC2B0500F0B5837CEB
:10B1500087B004460BB9C37C0BBB0023214605A86E
:10B16000039337F002FE04A805A9FEF71BFD059B1B
:10B17000204DA3F10C00A84230D1049E03A9304613
:10B180000A223DF0DBFE039B0746B3420AD9049B2B
:10B19000A3F10C02AA4215D1384607B0F0BD4068B1
:10B1A00007B0F0BD144BB4F80EE01B68268A58684F
:10B1B00022680168A389CDF800E001968C680F49E8
:10B1C000A047E4E753F8041C481E002943F8040C88
:10B1D000E2DC104605A937F0BBFBDDE753F8042C91
:10B1E000511E002A43F8041CC7DC02A937F0B0FB4B
:10B1F000C3E700BF640A0010E40200105C2C0500E5
:10B2000010B5044637F0B1FD204610BD08B5837C6B
:10B210000BB9C37C43B907490022032337F0FEFA78
:10B22000013018BF012008BD4068003018BF012060
:10B2300008BD00BFE82C050010B50123044641609D
:10B240000846E37438F056FCA060204610BD00BFED
:10B2500001228160C2747047837C10B504461BB91B
:10B260000123C37437F08DFD204610BD014B0360F0
:10B27000704700BFF82C050010B5034B044603606F
:10B28000FFF70EFD204610BDF82C0500014B0360B2
:10B29000704700BFF82C0500024B02461868FEF705
:10B2A00035BB00BFE4020010014B0360704700BFD4
:10B2B000A02D0500014B0360704700BFA02D0500C5
:10B2C00010B5034B04460360FFF7EAFC204610BDAF
:10B2D000A02D050010B5034B04460360FFF7E0FC0A
:10B2E000204610BDA02D050008463CF0AABE00BFB8
:10B2F0000EB42DE9F04392B019AC54F8049B02AEA1
:10B30000234605464A463046402101943FF0ACFAB8
:10B31000471C3F2F04460ADC2B6831465B692846F0
:10B320009847204612B0BDE8F04303B07047384656
:10B3300036F0C4FF39464A46019B80463FF094FAF6
:10B340002B6841465B6928469847B045E9D0B8F17B
:10B35000000FE6D0404636F0DDFFE2E710B4054BC3
:10B36000054C18461C600549054A5DF8044B36F04B
:10B37000CCBF00BF10030010782D0500B5B200004F
:10B38000C8000010F0B4104BDFF854C00F4F104E3F
:10B3900000225CF80200B9581C6941EA000524EA61
:10B3A00005041C615C699861B4500432142AD961A7
:10B3B00003F12003EDD107490748084B0522086037
:10B3C0001A60F0BC704700BF00C0092028030010BD
:10B3D000140300103C03001080C009205403001027
:10B3E00040030010F0B4114ADFF858C0104F114E5E
:10B3F00000235CF80340F9581569F05821430433E1
:10B4000025EA010501EA0004142B21EA0001156177
:10B410009461D16102F12002EBD107490748084B42
:10B42000052208601A60F0BC704700BF00C0092008
:10B4300040030010140300103C03001080C00920DA
:10B44000540300102803001004280AD81F2908D824
:10B45000012202FA01F1034B53F820200A4343F87A
:10B46000202070474003001004280AD81F2908D85C
:10B47000012202FA01F1034B53F820200A4343F85A
:10B480002020704728030010022994BF50F82100A3
:10B49000004870470000C07F2DE9F84F164603466C
:10B4A0000022D1F80490D6F808A043F8042B42609B
:10B4B0005A6004460D464846514638F06FFBD5F8B1
:10B4C0000880776883463946404638F067FB014676
:10B4D000584638F059FA366820603146404638F010
:10B4E0005DFB2D6880462946504638F057FB0146E3
:10B4F000404638F049FA29466060384638F04EFB3D
:10B5000031460546484638F049FB0146284638F0A2
:10B510003BFAA0602046BDE8F88F00BF70B5044636
:10B520000D460068096838F039FB696806466068AE
:10B5300038F034FB0146304638F028FAA968064650
:10B54000A06838F02BFB0146304638F01FFA70BD7A
:10B550000346806870B501465D681E6838F01EFBC2
:10B5600029460446284638F019FB31460546304640
:10B5700038F014FB0146284638F008FA0146204608
:10B5800038F004FA70BD00BF70B5034604460020D1
:10B5900043F8040B58600D46606008681168164651
:10B5A00038F0F2F971682060686838F0EDF9B16838
:10B5B0006060A86838F0E8F9A060204670BD00BF60
:10B5C00070B503460446002043F8040B58600D464E
:10B5D000606008681146164638F0E0FA314620608F
:10B5E000686838F0DBFA31466060A86838F0D6FA4F
:10B5F000A060204670BD00BF0346002270B543F82E
:10B60000042B426004465A6008460D46FFF7A0FF2F
:10B6100039F022FD06460146286838F073FB3146B2
:10B620002060686838F06EFB31466060A86838F0CA
:10B6300069FBA060204670BD054B10B404210224B4
:10B6400000221C6019605DF8044B4263704700BF24
:10B6500000E100E038B50D4B0446216118680D4645
:10B6600038F044FA4FF07A5138F098FA294638F019
:10B6700049FB39F007FA38F093FC4FF040230321DF
:10B6800001226061986159605A6038BD98010010CC
:10B6900038B50C4B0D46186838F028FA4FF07A513F
:10B6A00038F07CFA08490446284638F02BFB01465E
:10B6B000204638F073FA39F0E5F938F071FC034BA5
:10B6C000986138BD98010010002474490080004042
:10B6D000F8B5194F194E0025194A4FF040230321A0
:10B6E000C5624563386085609E6159615D60D2F8CE
:10B6F000C410144F03F5804341F0040105260446AD
:10B70000C2F8C4109F6110495E615D60FFF7A2FF3F
:10B7100020460E49FFF7BCFF94F83830E56265F328
:10B72000440384F8383094F83830256365F3000317
:10B7300084F838302046F8BD5803001080969800F1
:10B7400000C00F4040420F000050C3470000C842F5
:10B7500030B490F83850C5F34305FDB100230124FF
:10B7600002E00133AB4219DA04FA03F1C26A114272
:10B77000F7D000F1180252F82320917A11F0020F4D
:10B78000EFD011F0010F117A526804FA01F103F1C0
:10B79000010314BF9161D161AB42E5DB0023C362B9
:10B7A00030BC7047044B054A1968106841F001012C
:10B7B0001960FFF7CDBF00BF0080004058030010A4
:10B7C0002DE9F041066B002E4ED090F83810C1F3F1
:10B7D0004301002942D00023746D98464FF0010CBC
:10B7E00003E00133DBB28B4230DA04EB43125269DF
:10B7F000002AF6D003F01F080CFA08F800EB8302C9
:10B800009269376D957C18EA070F0CBF0027012756
:10B8100005F00108AD070BD5B84592F810800CFA79
:10B8200008F5D2F80C8014BFC8F81850C8F81C509E
:10B83000158F013367F308251587158FDBB245F4A3
:10B8400000758B424FF001081587CEDB0023436360
:10B85000B8F1000F03D00120BDE8F0814163044B33
:10B860001B68986907F062FC0020BDE8F08100BF0A
:10B87000E40200102DE9F04F90F8383083B0DA0779
:10B880000446DFF81CB240F1D280DBF8000090F8EB
:10B89000A8300190C3F34003002B40F08B8094F854
:10B8A0003860C6F34306002E00F09080D4F8309044
:10B8B000D4F834C0D9F854101D4615E0009800287B
:10B8C00032DD57683844B0F1804F506031DA04EB14
:10B8D0008302926992F8392012F0020F18BF0125F5
:10B8E0000133DBB2B34274DA4FEA431801EB0802CA
:10B8F00050690028F4D0D2F81CA0976851F80800CD
:10B90000E2450744009741F80870D7D1D9F8447050
:10B910006745D9F8487000F0A2806745CED10098FD
:10B92000D76800289760CCDC002741F808704FF0FA
:10B93000804000F140405060906904EB8307D7F8E5
:10B94000188000F1010AC2F818A098F80A008707C9
:10B950000CD598F808704FF0010A0AFA07F710F0B2
:10B96000010FD8F804000CBF8761C76198F839004F
:10B97000D8F82C7010F0010F0CBF01204FF0FF30F1
:10B980003844C8F82C0098F83970042BC7F34007E6
:10B990007FD8012003F01F0A00FA0AFAE06A40EAA1
:10B9A0000A00E062002F38D097695069874234D08E
:10B9B00042468FE794F8382000236FF3000284F8A2
:10B9C00038206363236303B0BDE8F08FD4F834C03C
:10B9D0003546E36A0CF10102626323B12E4B032169
:10B9E000012259605A60002DEDD1019A656390697A
:10B9F00007F09CFBDBF8003004F13001986907F098
:10BA0000C9FC00283BD194F83830256365F3000366
:10BA100084F8383003B0BDE8F08F00275761B8F8DC
:10BA2000380042466FF34920A8F8380052E7DBF8A7
:10BA3000003000F13001986907F0ACFC0028C2D05A
:10BA40002046FFF7BDFE94F8383060F3000384F819
:10BA5000383094F83830DB073FF517AFB3E7D9F843
:10BA60004CA0002057459060BFF457AF6745D761A1
:10BA70003FF455AF1769009741F808701EE720465C
:10BA8000FFF79EFE94F8383060F3000384F83830F6
:10BA900099E7024837F083FA00800040C02D050086
:10BAA000E40200104FF040231968034A41F00101FD
:10BAB00019601068FFF7DEBE5803001010B490F84C
:10BAC0003820C2F34304631C03F00F0300EB84042B
:10BAD00063F3440280F83820581EA1615DF8044BDE
:10BAE000704700BF826808B512B1C368984708BDA7
:10BAF00037F058FA08B5034B186883680BB1FFF7A5
:10BB0000F1FF08BD5803001070B4074E074D084CF4
:10BB100008490022C6640565446581650270426477
:10BB2000826470BC704700BF0123456789ABCDEFCD
:10BB3000FEDCBA9876543210F0B48AB10C46002379
:10BB4000A5786678CF5C2D0445EA0625E6783D4366
:10BB500045EA0665C55004339A4204F10404EFD85F
:10BB6000F0BC704730B4A2B1034600240D68043322
:10BB7000055551F8045B04342D0A03F8035C31F8D1
:10BB8000025CA24203F8025C11F8015C03F8015C5C
:10BB9000ECD830BC704700BF2DE9F04F91B004469F
:10BBA00040226846266D656DA76DD4F84C80FFF77E
:10BBB000C3FFDDF800E0E24B05EA0602F04427EAA5
:10BBC000060C43444CEA020C9C44019A06EB7C6C44
:10BBD000DC4B25EA0C000CEA06013A44134440EA27
:10BBE0000107029A1F440CEB3757D74B26EA070090
:10BBF00007EA0C012A44134440EA01051D44039955
:10BC000007EBF535D14B05EA07022CEA05000E4497
:10BC1000334410431844049ACD4B05EBB020134431
:10BC200027EA000100EA05029C441143059E614495
:10BC3000C84B00EB7161334425EA010201EA0006BA
:10BC40001F4432433A44C44E069F01EB325220EA6D
:10BC5000020C3E4402EA010735444CEA07032B4438
:10BC6000BE4F079D02EBF33321EA030C2F4403EA96
:10BC7000020538444CEA0506089F0644B84D03EB1C
:10BC8000B62606EA03003D4422EA0607294447EAAD
:10BC9000000C8C44B348099906EB7C6C23EA0C0534
:10BCA00008440CEA0601294302440A9D0A440CEBAD
:10BCB0003257A5F5244226EA070007EA0C014F3A5D
:10BCC000134440EA01051D440B98A74A07EBF535DC
:10BCD0002CEA050105EA07030244164441EA030081
:10BCE00030440C99A14B05EBB02027EA000800EA8C
:10BCF00005020B449C4448EA020161440D9A9C4BA6
:10BD000000EB716125EA0108134401EA000C48EADE
:10BD10000C0C1F44674401EB3752964B0E9F6FEAA1
:10BD2000020909EA00083B4402EA010C48EA0C0C4B
:10BD30001D4405EB0C0302EBF3330F9DDFF860C2EB
:10BD40006FEA030808EA010BAC4403EA020A4BEA73
:10BD50000A0A6044019E5044DFF848C203EBB02059
:10BD600000EA020AB44403EA09094AEA09096144FB
:10BD7000069E4944DFF830B200EBF16101EA030CA2
:10BD8000B34400EA08084CEA08085A440B9E4244AF
:10BD9000DFF818C201EBF25202EA0009B44421EACA
:10BDA000000849EA080863444344DFF804C202EB90
:10BDB000B34303EA0109F44422EA010849EA080806
:10BDC0006044059E4044DFF8ECC103EB303000EAEC
:10BDD000020923EA0208B444614449EA080B0A9EB6
:10BDE0008B44654900EBFB6B0BEA0308314420EA06
:10BDF000030C48EA0C0C0A44624460490BEBF25A0B
:10BE00000AEA000C29442BEA00024CEA02020B4425
:10BE1000134404995A4A0AEBB3490A442AEA0B0329
:10BE200009EA0B010B4310441844099A554B09EBDE
:10BE3000303808EA0A01134429EA0A020A439B44FB
:10BE40009344514A08EBFB6C0CEA09013A4428EA96
:10BE500009030B439244039E9A444C4B0CEBFA505B
:10BE600000EA080A33442CEA08024AEA020299442A
:10BE70009144474B089A00EBB94101EA0C0A13447C
:10BE800020EA0C094AEA090998440D9EC844414B2E
:10BE900001EB383202EA000921EA000833449C44ED
:10BEA00049EA0803029E6344DFF80C8102EBF36366
:10BEB00003EA0109B04422EA010C49EA0C0C4044AF
:10BEC000079E6044DFF8F4C003EBF05000EA02097B
:10BED000B44423EA020849EA080861440C9E41443C
:10BEE000DFF8DCC000EBB14101EA030920EA0308F6
:10BEF000B444624449EA080C9444059A01EB3C3C82
:10BF0000A2F5B82AAAF2BE6A81EA0002089E53444A
:10BF100082EA0C0A204A53440CEB337332448CEA15
:10BF200001080B9E88EA030810441C4A404403EBB6
:10BF30007050324483EA0C0888EA0008114441E05A
:10BF400078A46AD756B7C7E8DB702024EECEBDC10F
:10BF5000AF0F7CF52AC68747134630A8019546FDEA
:10BF6000D8988069AFF7448BBED75C892211906B5B
:10BF7000937198FD8E4379A65314440281E6A1D8AB
:10BF8000C8FBD3E7E6CDE121D60737C3870DD5F44B
:10BF9000ED145A4505E9E3A981F6718722619D6D8B
:10BFA0002108B44962251EF640B340C0515A5E26AE
:10BFB000AAC7B6E95D102FD6F8A3EFFCD9026F67C8
:10BFC0008A4C2A8DA44A414400EB31413A4480EA2C
:10BFD000030A019E8AEA010A9444A04AD44401EB70
:10BFE0007C2C81EA0008324488EA0C08049E1A443A
:10BFF0009B4B42440CEB32728CEA0108334488EAD2
:10C000000208079E03449748434402EB73533044AD
:10C0100082EA0C080A9E88EA0308014492484144D7
:10C0200003EB3141304483EA02090D9E89EA01099C
:10C0300084448E48CC4401EB7C28304481EA0309D7
:10C0400089EA080902448A484A4408EB327C704471
:10C0500088EA010282EA0C02034413448548039AE9
:10C060000CEB735310448CEA0802069E014482EAEA
:10C070000300814A084403EB3040324483EA0C0950
:10C08000099E89EA000990447C4AC84400EB782163
:10C09000324480EA03080C9E88EA01089444784AF6
:10C0A000C44401EB3C7C81EA0008324488EA0C0875
:10C0B0001A44744B42440CEB72528CEA01082B4434
:10C0C000029E88EA020803446F48434402EB33436C
:10C0D000304482EA0C0888EA0308014441446B4872
:10C0E00003EB7121704461EA020E84448EEA030E70
:10C0F000079EE644664801EBBE6E30446EEA030CD0
:10C100008CEA010C0244624462480EEBB25238449D
:10C1100062EA010787EA0E0703443B445E48059F35
:10C1200002EB7343384463EA0E07574001440C9E08
:10C1300039445A4803EBF121304461EA02065E407B
:10C140008644039FB644564801EBBE6E6EEA030672
:10C15000384402444E400A9816440EEBB656A0F5F9
:10C16000801766EA0102A7F6833782EA0E023B4493
:10C1700013444C48019A06EB7343104463EA0E02E1
:10C18000014482EA06000844474F089903EBF02077
:10C190000F4460EA06025A40BE449644434900EB0D
:10C1A000BE6E29446EEA030545400E442E44404AC3
:10C1B000069D0EEBB6562A4466EA000181EA0E019E
:10C1C00013440D9F0B443B4A06EB73433A4463EA26
:10C1D0000E01104471400144374A049803EBF121E9
:10C1E000024461EA0600584072440B9D0244334801
:10C1F00001EBB262284462EA03054D400644029F07
:10C200002E442F4802EBB656384466EA01055540E5
:10C2100003442B442B48099D06EB734363EA020E4B
:10C220002844276D8EEA060E014471441F44606D58
:10C23000E56C07EBF127A16D03442A440E44E26448
:10C24000684627656365A665002140223BF02FFB09
:10C2500011B0BDE8F08F00BF0C38E5FD44EABEA484
:10C26000A9CFDE4B604BBBF670BCBFBEC67E9B2821
:10C27000FA27A1EA8530EFD4051D880439D0D4D936
:10C28000E599DBE6F87CA21F6556ACC4442229F48C
:10C2900097FF2A43A72394AB39A093FCC3595B654E
:10C2A00092CC0C8FD15D84854F7EA86FE0E62CFE8A
:10C2B000144301A3A111084E827E53F735F23ABD13
:10C2C000BBD2D72A91D386EB2DE9F843446C1746AD
:10C2D000D20013199A424364836CC4F3C50488BF27
:10C2E0000133C4F1400603EB5773B7420546884655
:10C2F000836409D20444601C002408EB04013A1B47
:10C30000BDE8F8433BF0AFBA20443246013005F1B6
:10C3100001093BF0A8FAC4F1800449462846FFF71A
:10C320003BFCA74202D212E026461C4608EB06015F
:10C330002846FFF731FC04F140039F42F4D24846FF
:10C3400008EB04013A1BBDE8F8433BF08CBA4846C1
:10C350003446D2E730B5037883B00446B3BB00F16E
:10C360004405294668460822FFF7FCFB626C20461C
:10C37000C2F3C502372A94BFC2F13802C2F1780273
:10C380001449FFF7A1FF204669460822FFF79CFFEA
:10C3900004F15C0004F14C011022FFF7E3FB0021E3
:10C3A0004022601C3BF083FA0022AB1C84F844203E
:10C3B0006A7003F8012B03F8012B03F8012B03F833
:10C3C000012B03F8012B01211A702170204603B0C4
:10C3D00030BD00BFD0000010F0B50B788BB0074621
:10C3E000C3B10D4601AC09AE204695F85C200D495D
:10C3F00002343BF059FDB44205F10105F4D10023AC
:10C4000001A938466A468DF8243036F03BFD38469F
:10C410000BB0F0BD044901AA36F034FD38460BB02C
:10C42000F0BD00BFCC2D0500D8340500002930B484
:10C4300019DD0E4C03464518002013F8012B82EA43
:10C44000000101F00F0154F82110AB4281EA1010F5
:10C4500080EA121202F00F0254F8222082EA101031
:10C46000EBD130BC70470020FBE700BFD42D0500A6
:10C470005D4BF0B5D3F884E05C4DD3F88440D3F83D
:10C480000471D3F8C4601FFA8EFE0EFB055546F406
:10C490008056C3F8C460D3F8A861240C013407F1B6
:10C4A000010C95FBF4F426F0407E561E83B0054641
:10C4B0008F0194FBFCF4C3F8A8E1072E7AD8DFE8DB
:10C4C00006F07169793D79797904474BD3F8A81161
:10C4D00041F04071C3F8A81194FBF2F494FBF7F11A
:10C4E000FF2936DC002976D04E1E360246F40016AF
:10C4F0003F4F94FBF1F1B942296035DC3D4B0022FE
:10C500001E601868114620F0FF0018606A642B4610
:10C510000722013A501C19621964A3F10403F8D1EF
:10C52000354B162035491D6034F0D8FB314B284679
:10C53000DA6822F48072DA6003B0F0BD2A4B94FB13
:10C54000F2F4D3F8A811C3F8A81194FBF7F1FF296E
:10C55000C8DD2B483BF05EFA254FFF2194FBF1F13B
:10C56000B942284E2960C9DD89112748274A3BF086
:10C5700051FABC4236DD3A460123013394FBF3F114
:10C580009142FADC0029B8BF3F31891120483BF0C5
:10C5900041FAB3E7144BD3F8A81141F00071C3F886
:10C5A000A81199E7104BD3F8A81141F08071C3F896
:10C5B000A81191E71146174801923BF02BFA164853
:10C5C0003BF0DCFA084B019AD3F8A81141F08071D6
:10C5D000C3F8A81180E711483BF0D0FA4FF40016D9
:10C5E000012185E72146CDE700C00F4000366E01EE
:10C5F000405DC600004003405C030010BDC6000063
:10C60000982E050000FE2000202F0500751903005C
:10C61000642F05003C2E0500842E0500EC2E05003D
:10C62000254940F201120B6B70B51A4004460AB15D
:10C630000A69426040F202221A4012B11E4A52694F
:10C64000A26040F204421A4012B11B4A9269E260B1
:10C6500040F608021A4012B1174AD269226141F22B
:10C6600010021A4012B1144A126A626142F22002A8
:10C670001A4012B1104A526AA26144F240021A40B2
:10C6800012B10D4A926AE26148F280021A4012B178
:10C69000094BDB6A2362084B5E68C6F3026604EB53
:10C6A00086056B6A0BB168689847636C13B13046B6
:10C6B0006968984770BD00BF00400340014B18688F
:10C6C000FFF7AEBF5C030010034B0B44272B9ABF50
:10C6D000024AD05600207047E83FF6DF142E0500CE
:10C6E000904B0B44272B33D88F490120C95600FAB1
:10C6F00001F1D00730D5272B00F2F880DFE813F0E6
:10C70000680086009800F600F600F600F600F600D5
:10C71000F600F600F600F600F600F600F600F60069
:10C72000F600F600F600F600F600F600F600F60059
:10C73000F600F600F600F600F600F600F600F60049
:10C74000F600F600F600F600F600F600AA00BC00BF
:10C75000D0074FF00101CED4272B00F2D980DFE8BB
:10C7600013F09D00A700B100D700D700D700D70075
:10C77000D700D700D700D700D700D700D700D70001
:10C78000D700D700D700D700D700D700D700D700F1
:10C79000D700D700D700D700D700D700D700D700E1
:10C7A000D700D700D700D700D700D700D700BB00ED
:10C7B00028005E4BDA6822F04042DA60DA6C22F040
:10C7C0004042DA645A4B1A6822EA01011960704744
:10C7D000564B5A6822F440325A605A6842F480320A
:10C7E0005A605A6C22F440325A645A6C42F4003255
:10C7F0005A644F4B1A68D20303D41A6822F0FF021E
:10C800001A604B4B1A68114319607047474B5A68BE
:10C8100022F440225A605A6842F480225A605A6CCC
:10C8200022F440225A645A6C42F400225A64E0E72F
:10C830003E4B5A6822F440125A605A6842F4801201
:10C840005A605A6C22F440125A645A6C42F4001234
:10C850005A64CEE7354BDA6822F04052DA60DA6883
:10C8600042F04052DA60DA6C22F04052DA64DA6C5C
:10C8700042F00052DA64BCE72C4BDA6822F0404206
:10C88000DA60DA6842F04042DA60DA6C22F0404264
:10C89000DA64DA6C42F00042DA64AAE7234B5A68A1
:10C8A00022F440325A605A6C22F440325A6489E7CA
:10C8B0001E4B5A6822F440225A605A6C22F44022DD
:10C8C0005A647FE7194B5A6822F440125A605A6C36
:10C8D00022F440125A6475E7144BDA6822F0405291
:10C8E000DA60DA6C22F04052DA646BE70F4B5A6878
:10C8F00022F440425A605A6842F480425A605A6CAC
:10C9000022F440425A645A6C42F400425A6470E77E
:10C91000064B5A6822F440425A605A6C22F4404254
:10C920005A644FE7E83FF6DF142E050000C00240CE
:10C930000040034008B50D4BC9071A6803D422F420
:10C9400080321A6008BD12F0E06F05D1074B1A68FB
:10C9500042F480321A6008BD05491A680B68C2F3B8
:10C960000262D86803493AF06FFBEFE700400340EA
:10C9700000020010D42F0500174B10B40B44272BD6
:10C9800017D816480121C356012A01FA03F1144BA6
:10C9900014D0DA6822EA0101D960DB6813F0FF0FD6
:10C9A00004D1104B4FF48002C3F880205DF8044B93
:10C9B0007047012A4FF00101094BEAD1DC68094AAE
:10C9C00024F48074DC60DC684FF480002143D9607B
:10C9D0005DF8044B10607047E83FF6DF142E050049
:10C9E0000040034000E100E04164704700207047D0
:10C9F00004300321FEF750BCA0F10400FFF7F8BF9C
:10CA000008B5836C13B1013B836403B108BD806832
:10CA100008F056FEFEE700BFA0F10400FFF7F0BFEC
:10CA200010B5064B044603F108022833226040F893
:10CA3000043FFEF71BFC204610BD00BF7030050010
:10CA4000A0F10400FFF7ECBF10B5074B044603F15B
:10CA500008022833226040F8043FFEF707FC204616
:10CA6000FEF71EF9204610BD70300500A0F104004D
:10CA7000EAE700BF70B50C460546C97822891B4815
:10CA80003AF0C8FFE378062B2ED8DFE803F0042D38
:10CA90002D0F0D250D0080230020AB640121FAF736
:10CAA0000FFA1348FAF724FA012070BD002301227F
:10CAB0004FF4FA70A5F8400085F83F3085F8423011
:10CAC00085F8433085F8443005F13F06062122758C
:10CAD0001046E660216170BD0120002305F8433F48
:10CAE0002075E560206170BD002070BD48300500F4
:10CAF00090D003002DE9F047344B044688B040F84D
:10CB0000043B8846FEF7C2FBDFF8C8E0304BDEF896
:10CB10000000DEF80410764603F1080204F10C0769
:10CB2000283384E80C0103C756F80C0F01AD716877
:10CB3000B268F3689EF808E00FC530697169B269A0
:10CB40004FF0FE0C00264FF0040901234FF0090AB4
:10CB500087F800E084F81AC0E3762377C4F8214010
:10CB600084F815A084F81690E675267666766677C2
:10CB7000A677E67784F8206007C50DEB09050FCD91
:10CB8000C4F82500C4F8291003CD2D88C4F82D2041
:10CB9000C4F83130C4F83500C4F83910A4F83D5059
:10CBA00004F11501404600F0E9F904F1250704F10C
:10CBB0000C01A06800F0C6F93946A06800F09CFAA4
:10CBC00060772046A66408B0BDE8F08718300500FD
:10CBD0007030050020300500704700BF704700BF6F
:10CBE000704700BF704700BF0120704770B5002438
:10CBF00082B00B460D46164600942146052208F0E9
:10CC000061FD00280ADD074B294653F820303246E3
:10CC1000986803689B68984702B070BD204602B0D0
:10CC200070BD00BF60030010A0F10800FFF7DEBF79
:10CC300070B5002482B00B460D461646009421467E
:10CC4000052208F03FFD00280ADD074B294653F86E
:10CC50002030324698680368DB68984702B070BDA0
:10CC6000204602B070BD00BF60030010A0F10800B4
:10CC7000FFF7DEBFF0B5002583B00B4600952946CF
:10CC80000222064608F01EFD00282BDD1749441C31
:10CC900051F824201AB35378022B20D001EB8404DE
:10CCA0002F4614E0052B0CD1304655B9D378917836
:10CCB00003F00303012B0CBF02230023928809F029
:10CCC0001BFA54F8042F52B15378022B07D0042BCF
:10CCD000E8D15772D57854F8042F002AF4D10120F6
:10CCE00003B0F0BD284603B0F0BD00BF60030010E4
:10CCF000F0B5CEB283B0009217463346002104222D
:10CD0000054608F0DFFC041E30DD002133460091AB
:10CD10002846042208F0D6FC002827DD154951F8E2
:10CD200020305F7251F824205378042B1ED0022B40
:10CD30001CD001EB840406E054F8042F5378042B34
:10CD400014D0022B12D0052BF6D1D378917803F0B2
:10CD50000303012B0CBF022300239288284609F00D
:10CD6000CBF954F8042F5378042BEAD1002003B0F8
:10CD7000F0BD00BF6003001008B508F0BBFA00204A
:10CD800008BD00BF08B519B908F09AFC012008BD1C
:10CD900008F094FC012008BD10B5032104469C3026
:10CDA000FEF77AFA2046BDE8104008F087BC00BFC5
:10CDB000A0F19C00FFF7F0BF09F030BAA0F19C0091
:10CDC000FFF7FABF30B54B7883B0013B012B0C461F
:10CDD00002D9002003B030BD8B78012B19D0022B73
:10CDE000F7D18B7900210522009108F06BFC0546F4
:10CDF00036F02EFA0022002336F020FD0028E8D07D
:10CE0000104B214653F82530986803681B689847F3
:10CE1000E0E78B7900210422009108F053FC0546DD
:10CE200036F016FA0022002336F008FD0028D1D093
:10CE3000044B214653F82530D86803681B6898478F
:10CE4000C8E700BF60030010A0F10800FFF7BABFF9
:10CE5000F0B50C46497883B00139012916461D46C4
:10CE600002D9002003B0F0BDA378012B1BD0022B08
:10CE7000F7D10021A3790522009108F023FC074691
:10CE800036F0E6F90022002336F0D8FC0028E8D07E
:10CE9000124B214653F82730324698682B460468D7
:10CEA0006468A047DDE70021A3790422009108F01F
:10CEB00009FC074636F0CCF90022002336F0BEFC10
:10CEC0000028CED0054B214653F827303246D8688B
:10CED0002B4604686468A047C3E700BF60030010E6
:10CEE000A0F10800FFF7B4BFF0B585B004216A4691
:10CEF000124D0746ADF1040608F06CFF03A87368F5
:10CF0000A5F110042A4603F00F01092994BF30311E
:10CF1000373122F80219A2424FEA1313F3D146F82F
:10CF2000043F864205F11005E9D10549384608F06D
:10CF3000F3F9384609F024F905B0F0BD30010010CE
:10CF4000600300100A4B002002E0013030280CD0B2
:10CF500053F8042F002AF8D1064A074B42F8201054
:10CF600009785A880A445A8070474FF0FF3070475A
:10CF70005C0300106003001014010010002230B4A4
:10CF80001348144606E05D780132042D08BF1C46A4
:10CF9000302A19D050F8043F002BF4D10D4B1879EA
:10CFA00034B1E478CD78A5421CBF00F1FF30C0B2A7
:10CFB000094D441C887045F822101C7109785A8864
:10CFC00030BC0A445A8070474FF0FF3030BC704785
:10CFD0005C0300101401001060030010002270B404
:10CFE00017491446134607E04678042E08BF044646
:10CFF00008BF2B46302A1DD051F8040FD5B201329C
:10D000000028F1D1B4B1ABB12F2B11D80D4C54F88D
:10D0100023201AB912E054F823204AB15178013381
:10D02000052908BF0130DBB208BFC0B2302BF2D1F6
:10D0300070BC70474FF0FF3070BC70471046F7E788
:10D040005C03001060030010F8B5274E0F46A6F1F0
:10D05000C003002205E06578042D08BF2246B342D4
:10D060003AD053F8044F002CF5D1002A34D0FFF702
:10D07000B5FFF9781D4AC1F1010601E0302C16D048
:10D0800052F8043FE5B2013493B15D78052DF5D136
:10D09000DD788D42F2D19B78BD7803F00F0C6B40A8
:10D0A0001B06EBD46645B8BF6646302CE8D1254652
:10D0B000022914D003360F2E0EDCF6B2BB780C4AD0
:10D0C00023F07F031E430B4BBE7042F825705A8835
:10D0D00039780A445A80F8BD4FF0FF30F8BD0E2E63
:10D0E000E8D10F26EAE700BF1C0400105C03001023
:10D0F00060030010140100104B7810B4032B15D1FD
:10D1000000230D4C184607E052780133032A04BF70
:10D110000130C0B2302B09D054F8042F002AF3D1CB
:10D12000064A5DF8044B42F8231070474FF0FF3079
:10D130005DF8044B704700BF5C03001060030010F3
:10D14000F8B5044608F0FAFB04F19C00FEF79EF8DF
:10D15000194A1A481A4E1B4D02F1800102F15C0E69
:10D1600002F16807034684E80440C4F89C10A760F5
:10D1700000F1BC0143F8046F0560002243F8042F5E
:10D180008B42FBD120461049FFF7B6FF20460F49DE
:10D19000FFF7B2FF0E49A8732046FFF7ADFF0D4918
:10D1A000E8732046FFF7A8FF0B4928742046FFF7D5
:10D1B000A3FFB0712046F8BDE83005006003001001
:10D1C000140100106401001010010010C8300500A7
:10D1D000AC31050020010010983105000020704797
:10D1E0000020704700207047F8B50C4B00240C4D10
:10D1F00006460360274655F8043BB34207D0013486
:10D20000042CF8D1304634F033F93046F8BDE0B2A2
:10D21000002145F8047C0CF0D7FBF0E7D83105007D
:10D220002004001010B50446FFF7DEFF2046FDF78E
:10D2300037FD204610BD00BF30B5D0F84052ADF2EA
:10D24000A46D0B46144686A82A4620493AF02CFEC7
:10D25000A50730D414F0010F0CBF01220222A00553
:10D2600005D561054CBF42F0080242F0100286A9C4
:10D2700096A80CF0C1FB28BB23071ED40DF27C44FA
:10D2800096A94FF4097220463AF0EDFA4FF40A706D
:10D2900035F016F80DF5916105464FF406726846B3
:10D2A0003AF0E1FA94E80E00284600F0F3F8284638
:10D2B0000DF2A46D30BD0322D1E796A899990CF028
:10D2C00069FEDBE700200DF2A46D30BD10320500D1
:10D2D00008B508460CF08CFF003018BF0120404212
:10D2E00008BD00BF08B5084611460DF0EBF8003048
:10D2F00018BF0120404208BD08B500214FF400725C
:10D3000090F840020DF07EF9003018BF0120404235
:10D3100008BD00BF10B59AB0D0F840220B460AA84D
:10D320000A493AF0C1FD0AA901A80CF0F9FE50B96A
:10D330004FF4987034F0C4FF01A9044600F026F9B8
:10D3400020461AB010BD00201AB010BD10320500E2
:10D3500008B508460CF0ACFF003018BF0120404271
:10D3600008BD00BF40F2E730704700BFF8B5064681
:10D370000F4634F095F8104B104C3360002354F8EE
:10D38000045F65B10133042BF9D10D4B3A461B689C
:10D390000C49D86839F058FE012033F005FE0A4ADE
:10D3A000C6F84032D8B206F1100142F823600CF002
:10D3B0000BFB3046F8BD00BFD83105001C0400103F
:10D3C00000020010183205002004001000207047F1
:10D3D0000069704738B5044604300CF0D3FD0546AB
:10D3E0001CB1236820461B6A9847284638BD00BFF9
:10D3F00000B583B0043001AB0CF086FC18B901987D
:10D4000003B05DF804FB4FF0FF30F9E700B583B0DF
:10D41000043001AB0CF0ACFB18B9019803B05DF817
:10D4200004FB4FF0FF30F9E7022A10B5044609D09B
:10D43000012A04BFC368C918201D0CF0ABFD20B938
:10D44000E06810BD03691944F6E74FF0FF3010BDE6
:10D4500008B504300CF042FD003018BF01204042F6
:10D4600008BD00BF10B5034B0446036034F08EF8CE
:10D47000204610BD5832050010B5054B0446036028
:10D4800034F084F82046FDF70BFC204610BD00BFA9
:10D490005832050084B070B506460948354645F84F
:10D4A000040B05AC84E80E00284621464FF40972AF
:10D4B0003AF0D9F93046BDE8704004B0704700BF7B
:10D4C000583205004FF0FF30704700BF704700BF73
:10D4D000014B0360704700BF8832050008B510B1EA
:10D4E00003689B699847002008BD00BF0023438163
:10D4F000704700BF4089704741817047014B03600E
:10D50000704700BF8832050010B5034B0446036026
:10D51000FDF7C6FB204610BD8832050010B5034B51
:10D5200004460360FDF7BCFB204610BD88320500B1
:10D5300010B5154A88B004464FF48073043069462C
:10D54000069207930CF024FED0B99DF8090098B11B
:10D5500006990B7893B90D220DF1090104F1280306
:10D5600018463AF080F99DF80810009AC1F30011AE
:10D5700084F82C11C4F8282108B010BD079AEDE7F3
:10D58000002008B010BD00BF30040010074B70B47D
:10D59000044644F8043B0D4606460FCD0FC40FCD9C
:10D5A0000FC42B683046236070BC7047B032050052
:10D5B0008088431A58425841704700BF10B58368AD
:10D5C0000C4A04460C49A3F10C00904282B0216041
:10D5D00004D10A4B2046236002B010BD53F8042C3E
:10D5E000511E002A43F8041CF3DC01A935F0B0F900
:10D5F000EFE700BF640A0010D832050000270500DD
:10D6000010B583680D4A04460D49A3F10C00904201
:10D6100082B0216007D10B4B20462360FDF740FB11
:10D62000204602B010BD53F8042C511E002A43F8C6
:10D63000041CF0DC01A935F08BF9ECE7640A00105A
:10D64000D83205000027050070B584B000F108014C
:10D65000044602A835F089FB02A903A835F085FB32
:10D6600003A8FCF761FB039B134DA3F10C02AA4234
:10D6700006460AD10EB101232373029BA3F10C00CD
:10D68000A8420ED1207B04B070BD53F8041C481E84
:10D69000002943F8040CEDDC104601A935F058F9D7
:10D6A000E8E753F8042C511E002A43F8041CE9DC77
:10D6B00003A935F04DF9E5E7640A001038B5094BC8
:10D6C000094D04460560A36010460D46FCF75EF95F
:10D6D0002946A08004F1080035F053FB0023237392
:10D6E000204638BD700A0010D8320500F0B5A3B04E
:10D6F00007460E46144601A81A4683211D4639F0F6
:10D700008BFB30B33AF09DFC22AB184410F8853CFB
:10D710000A2B07D08CB9284639F002FB0A2801D021
:10D720000130F8D101A83AF08CFC01A9024630463C
:10D7300035F0BAF9012023B0F0BD01A823213AF059
:10D7400046FC0028E7D12146BA6803483AF062F95E
:10D75000E1E723B0F0BD00BFF832050030B50B7B28
:10D7600083B00D46044673B90846FFF76DFF50B904
:10D7700009483AF003FA2046084901AA35F082FB2D
:10D78000204603B030BD05F10801204635F0EDFA22
:10D79000204603B030BD00BF18330500D834050063
:10D7A0002DE9F043037B8BB0054688469146002B5C
:10D7B00076D008A84146FCF713F907A82946FFF7D9
:10D7C000CDFF07987D4939F035FC079B7C4E044618
:10D7D000A3F10C00B04240F0E480A3899A062BD458
:10D7E000784F05A92046049739F0ACFA04A92846D9
:10D7F00000222346FFF77AFF06A9002859D02046C9
:10D8000039F0A0FA2B6807A8D3F81CC004AA08AB0B
:10D810002946E0470798034653F80C2DB34240F0E1
:10D820009880002A55D1049BA3F10C00B04240F02F
:10D83000A080A3899B06D4D5204639F059F907A8C2
:10D840002946FFF78BFF07985F4939F0F3FB079BE9
:10D850000446A3F10C00B04240F0978021460A2014
:10D8600039F028FC2146D8F8000039F081FC234625
:10D8700009220121554839F031FF2146D9F800002D
:10D8800039F076FC234601211122514839F026FF58
:10D89000204639F02DF9012420460BB0BDE8F08375
:10D8A000FFF7D2FE0446002883D120460BB0BDE826
:10D8B000F083049BA3F10C00B042BDD053F8042CBC
:10D8C000511E002A43F8041CB6DC07A935F040F8C5
:10D8D000B2E7D8F80020D9F8003052F80C0C0599BE
:10D8E00053F80C2C069B02445B1A0332043B934210
:10D8F000204612D239F0FCF80024049BA3F10C005E
:10D90000B042C9D053F8042C511E002A43F8041C1D
:10D91000C2DC07A935F01CF8BEE7002239F048FD4B
:10D920002146D8F8000039F023FC2146202039F0A8
:10D93000C1FB2146D9F8000039F01AFC2346012129
:10D940000222244839F0CAFE204639F0D1F80124D9
:10D95000D3E750F8041C01F1FF3E002940F804EC25
:10D960003FF75FAF184603A9019234F0F1FF019A27
:10D9700057E753F8042C511E002A43F8041C3FF7C4
:10D9800058AF07A934F0E4FF53E753F8042C511EB5
:10D99000002A43F8041C3FF761AF06A934F0D8FF12
:10D9A0005CE753F8042C511E002A43F8041C3FF78F
:10D9B00014AF06A934F0CCFF0FE700BF38330500E1
:10D9C000640A0010700A0010741D05004033050041
:10D9D0004C3305003C3305002DE9F04784B00C467C
:10D9E0009146434903AA054635F04CFA237B002BA8
:10D9F00048D003A82146FFF7B1FE03983D4939F00E
:10DA000019FB039B3C4E8046A3F10C00B04263D14E
:10DA1000B8F80C309A062ED4DFF8E0A019E0276899
:10DA200003A8FF69B847284603A934F092FE03997A
:10DA3000A1F10C00B0422ED12B6853F80C3CABB9CD
:10DA4000029BA3F10C00B04230D1B8F80C309B0619
:10DA500011D402A9002243462046CDF808A0FFF7C2
:10DA600045FE02AA4B4621460028D8D1029BA3F1CD
:10DA70000C00B04225D1404639F03AF8284604B0AF
:10DA8000BDE8F0872046FFF7DFFD0028B1D128462A
:10DA900004B0BDE8F08751F8043C5A1E002B41F851
:10DAA000042CC9DC01A934F053FFC5E753F8042C5A
:10DAB000511E002A43F8041CC7DC03A934F048FFB8
:10DAC000C3E753F8042C511E002A43F8041CD2DC8F
:10DAD00003A934F03DFFCEE753F8042C511E002A71
:10DAE00043F8041C94DC02A934F032FF90E700BF35
:10DAF000D8340500D4A60500640A0010700A00108E
:10DB0000F8B50446084615460E463AF09AFA0A4B0E
:10DB1000074623602B68204653F80C1C394435F027
:10DB200068F831463A46204635F0ACF8204629469A
:10DB300035F07FF82046F8BD700A00102DE9F04F4F
:10DB400089B092460446884607A8114605AA35F0D2
:10DB500099F907A8FCF7E8F8079BB34FA3F10C026B
:10DB6000BA42054640F03A8115B909B0BDE8F08FD8
:10DB70005046AE4939F05EFA838906469A0600F1AE
:10DB80000E81DFF8C092012509E0049BA3F10C008F
:10DB9000B84240F05981B3899B0600F100812A46C2
:10DBA000204604A93346CDF810900135FFF79EFDBD
:10DBB000002800F0E580236842469B69204604A9BE
:10DBC000984782894AF6E6139A42DED107AA01688D
:10DBD00005A835F057F905A907A835F0C6F807A834
:10DBE000FCF7A2F8079B8346A3F10C02BA4240F06F
:10DBF0000281BBF1000F40F08680059B53F8042C96
:10DC0000002A03DB05A834F009FF059B1B782F2BA6
:10DC10000ED007A8864905AAFFF772FF05A807A935
:10DC200034F097FD079BA3F10C00B84240F03A8115
:10DC30000DF1180B514607AA584635F023F92F214C
:10DC40004FF0FF32584634F0D4FD594603460022C7
:10DC500007A835F0D3F8584607A934F07AFD079B9A
:10DC6000A3F10C00B84240F02B81594607A835F0CB
:10DC70007CF805A907A834F0DCFF07A8FCF754F8E6
:10DC8000079B8446A3F10C02BA4240F0F680BCF137
:10DC9000000F17D105AA07A86649FFF731FF07A8AB
:10DCA000FCF742F8079B8346A3F10C02BA4240F00E
:10DCB000D78007A8BBF1000F7CD05E4905AAFFF70B
:10DCC0001FFF07E0594607A835F04FF807A805A938
:10DCD00034F0AFFF05A807A934F03BFD079BA3F183
:10DCE0000C00B84240F00981069BA3F10C00B84239
:10DCF00009D053F8042C511E002A43F8041C02DCFE
:10DD000007A934F025FE05A907A835F02EF807A8C5
:10DD1000FCF70AF8079B8346A3F10C02BA4277D1BD
:10DD2000BBF1000F41D00599434839F073FE07A9B4
:10DD3000304639F007F83D493246059839F028FB5E
:10DD400020464146059AFFF7F9FE384950463246CB
:10DD500039F01EFB304607A939F0D0FB059BA3F133
:10DD60000C00B8423FF411AF53F8042C511E002AA6
:10DD700043F8041C3FF709AF07A934F0E9FD04E7B5
:10DD8000049BA3F10C00B84209D053F8042C511E97
:10DD9000002A43F8041C02DC07A934F0D9FD304600
:10DDA00038F0A6FE09B0BDE8F08F0599234839F098
:10DDB00031FED3E705AA2249FFF7A2FE07A8FBF729
:10DDC000B3FF079B8346A3F10C02BA4240F0848064
:10DDD000BBF1000F88D007A819496FE753F8041C5E
:10DDE000481E002943F8040C3FF7BEAE104606A9B2
:10DDF00034F0AEFDB8E653F8041C481E002943F881
:10DE0000040C3FF7F6AE104606A934F0A1FDF0E68B
:10DE100053F8041C481E002943F8040C80DC10460B
:10DE200006A934F095FD7BE7640A0010D4A605002E
:10DE3000E8280500603305006C33050088330500D1
:10DE400064330500700A001053F8042C511E002A98
:10DE500043F8041C3FF79FAE07A934F079FD9AE61A
:10DE600053F8041C481E002943F8040C3FF721AF67
:10DE7000104603A934F06CFD1BE753F8041C481E40
:10DE8000002943F8040C3FF702AF104603A9CDF870
:10DE900004C034F05DFDDDF804C0BCF1000F3FF4B8
:10DEA000F9AE0FE753F8042C0DF1180B511E002AA0
:10DEB00043F8041C3FF7BEAE594634F049FDB9E6BD
:10DEC00053F8042C511E002A43F8041C3FF7CDAE32
:10DED00003A934F03DFDC8E653F8041C481E002990
:10DEE00043F8040C3FF774AF104603A934F030FD3B
:10DEF000BBF1000F3FF4F8AE6DE753F8042C511E50
:10DF0000002A43F8041C3FF7EFAE03A934F020FDCC
:10DF1000EAE600BF30B5037B83B004460D4683B10B
:10DF200001A82146FFF71AFC2046019A2946FFF76F
:10DF300005FE019B0B4AA3F10C00904207D103B0F0
:10DF400030BDFFF781FB0028EAD103B030BD53F8A4
:10DF5000042C511E002A43F8041CF0DC694634F0FE
:10DF6000F7FCECE7640A00108088431A58425841D5
:10DF7000704700BF00207047014B0360704700BF2F
:10DF80000027050010B5034B04460360FCF788FE2C
:10DF9000204610BD002705002DE9F0438668C568BE
:10DFA00083B0AE42074688462AD2AE42DFF86C9074
:10DFB00023D23378741C0A2B08BF012204D106E057
:10DFC00014F8013B0A2B01D0AC42F9D1A21B314617
:10DFD0006B4601A834F06BFF3B6838469B6901A98A
:10DFE00042469847019BA3F10C0048450BD1FD68C0
:10DFF000AC4205D22646AE42DBD334460022E6E7E9
:10E0000003B0BDE8F08353F8042C511E002A43F8F6
:10E01000041CECDC694634F09BFCE8E7640A001061
:10E020002DE9F04784B00F469246354903AA804651
:10E0300034F028FFB968FE68B14247D2B142DFF838
:10E04000C49031D20B784C1C0A2B08BF012204D19A
:10E0500006E014F8015B0A2D01D0B442F9D1621A2E
:10E0600003AB02A834F023FF3B6803A8DD693946FF
:10E07000534602AAA847404603A934F06AFB039B13
:10E08000A3F10C00484525D1D8F8003053F80C3CDA
:10E090006BB9029BA3F10C00484526D1FE68B4423F
:10E0A00014D22146B142CDD30C460022D8E7029BC0
:10E0B000A3F10C00484509D053F8042C511E002A46
:10E0C00043F8041C02DC03A934F042FC404604B0CF
:10E0D000BDE8F08753F8042C511E002A43F8041CB5
:10E0E000D2DC01A934F034FCCEE753F8042C511EE5
:10E0F000002A43F8041CD1DC03A934F029FCCDE745
:10E10000D8340500640A0010064B10B504460360BD
:10E110000846FBF73BFC044A044BA080A260E36086
:10E12000204610BDC03305007EB2050029B40500AD
:10E1300010B5064B04464068236008B138F0D8FC9F
:10E14000034A002384E80C00204610BDE833050094
:10E15000A02D050010B5084B04464068236008B1A7
:10E1600038F0C6FC054A0023204684E80C00FCF782
:10E1700097FD204610BD00BFE8330500A02D050027
:10E1800070B544680D4654B1084639F05AFF23462D
:10E19000024601212846BDE8704039F09FBA20466A
:10E1A00070BD00BF0121FDF777B800BF10B58368CF
:10E1B0000C4A04460C49A3F10C00904282B0216045
:10E1C00005D12046FDF752F8204602B010BD53F8A5
:10E1D000042C511E002A43F8041CF2DC01A934F07F
:10E1E000B7FBEEE7640A00100037050010B583683E
:10E1F0000E4A04460E49A3F10C00904282B0216001
:10E2000008D12046FDF732F82046FCF749FD2046AC
:10E2100002B010BD53F8042C511E002A43F8041C10
:10E22000EFDC01A934F094FBEBE700BF640A0010B7
:10E23000003705002DE9F04F51F8043B95B0074633
:10E2400007A8069334F091FD07A902A834F08DFDCC
:10E25000029D55F80C3C002B00F0858055F8043CDD
:10E26000002B03DB02A834F0D9FB029D2C78242C70
:10E2700000F08F80204639F071FA0646002840F001
:10E280008880472C35D04D2C33D0542C31D0532C92
:10E290002FD04E2C00F055820246864902A8042356
:10E2A00034F0BCFAA0B1202C10D03B2C07D004F0E5
:10E2B000F703202B03D00A2C01D00D2C04D1069893
:10E2C0007D4903689B689847029B3DE00130F6D08A
:10E2D00006217A4A3B7D0EA839F0B4FD0EA839F02C
:10E2E000B0FE0EAA0346002102A834F015FC029DE0
:10E2F000B4E77B684FF0000803F1010902A87049F8
:10E300000022022334F08AFA451C10D0034602A9E9
:10E3100000220EA834F072FD02A80EA934F019FAFA
:10E320000E9B684EA3F10C00B04240F09D867A68C7
:10E330000132B8F1000F01D191452CD00698624905
:10E3400003689B689847029B5E4EA3F10C00B042A5
:10E3500040F08086079BA3F10C00B04240F0EC85B2
:10E3600015B0BDE8F08F069853490368554E9B6879
:10E370009847029DA5F10C00B042EBD055F8043C43
:10E380005A1E002B45F8042CE4DC0EA934F0E0FA08
:10E39000E0E74C4EEEE74E2CDFF83C8108BFC7F8B3
:10E3A0000490029B53F80C2C002ACDD00222134675
:10E3B00002A8464934F032FADFF820B104460130B1
:10E3C000CDF80CB000F0F4800EAD234602A9002277
:10E3D00028460DF10C0A34F011FD5046294634F060
:10E3E000B8F90E9BABF10C06A3F10C00B04240F063
:10E3F0004886029B53F80C3C9C4200F228864FF062
:10E40000FF33224602A9284634F0F8FC02A8294628
:10E4100034F09FF90E9BA3F10C00B04240F00A8645
:10E420007B7DD90704D53A69069B9A4200F0218387
:10E43000182033F045FFDFF8A890069A51460123D3
:10E4400004461AF037FFD9F80000267A90F8A85051
:10E45000AA0747D5B307216804D540F2E7339942AC
:10E4600000F092841A4B53F8042F91423AD043455E
:10E47000F9D16B0740F1A3820698164903689B689F
:10E4800098472CB120461AF00FFE2046FCF708FCF6
:10E490000C4E039BA3F10C00B04282D053F8042C25
:10E4A000511E002A43F8041C3FF77BAF0EA934F03D
:10E4B0004FFA76E7E836050024350500F03605000A
:10E4C00070340500640A0010DC3605007434050061
:10E4D00004340500C034050038340500700A00100B
:10E4E000E4020010760706D56368352B00F0D28170
:10E4F000032B40F2E181237A980765D52368B3F5B1
:10E50000FA7F00F0AE8300F297801E2B00F0A0830C
:10E5100000F2D481022B00F058821C2B54D12CB174
:10E5200020461AF0C1FD2046FCF7BAFB039B07F119
:10E53000080453F80C3C032B40F289855146042211
:10E540004FF0FF3308A834F059FC0021A14A0423FE
:10E5500008A834F0E1FA026814AD034645F8182D16
:10E560002046C3F800B0294634F0F3F80E9B9A4ECB
:10E57000A3F10C00B04240F05085089BA3F10C00C1
:10E58000B04240F03D85B868944938F053FDF860DA
:10E59000002800F0718406987A7D036842F0010239
:10E5A0009B688F497A75BA689847069B3B6170E70C
:10E5B0000DF10C0A02A9504634F0E3FB02A8894988
:10E5C000002234F071FA2BE7D9F80000864E22467B
:10E5D0000221FBF7B1F8237ADA0640F13F81D9F83E
:10E5E0000030069893F8A8305B07036848BF7F495E
:10E5F0009B6858BF7E4998472269069852F80C3CA0
:10E60000002B40F0A08103687A499B6898470698E0
:10E61000794903689B689847D9F8000007210022D0
:10E62000FBF78AF8002C3FF434AF20461AF03CFD8B
:10E630002046FCF735FB2CE740F2F712934200F03E
:10E640008F82B3F5FC7FC0F08C8100F0B682B3F509
:10E650007A7FB9D1039B53F80C3C042B40F2F7842A
:10E660000EAD4FF0FF3351460522284634F0C6FB6D
:10E67000284602A934F0DDFA0368574E0493C0F827
:10E6800000B00E9BA3F10C00B04218D000F09FBC6C
:10E69000049B53F80C3C002B00F0D9844FF0FF335F
:10E6A00004A90122284634F0A9FB04A8294634F025
:10E6B00050F80E9BA3F10C00B04240F08884049BFC
:10E6C00053F8042C002A03DB04A834F0A7F9049BB8
:10E6D0001878FBF73BFA0028DAD12CB120461AF063
:10E6E000E3FC2046FCF7DCFA049B53F80C3C002BBF
:10E6F00040F016833B4905AA284634F0C3FB3F4847
:10E700002946069A22F0BCFB0E9BA3F10C00B042F6
:10E7100040F0388406983A4903689B689847049B00
:10E72000A3F10C00B04200F0068153F8042C511EF6
:10E73000002A43F8041C00F3FE80294634F008F94F
:10E74000F9E00EAD334602A9069A28461AF0B2FD4A
:10E750002146324628461AF0D9FC35F0FBFB3246FA
:10E7600082462A2128461AF0D1FC35F0F3FB9DF8A9
:10E77000403080469A07D14603D50E9B6E2B00F0A1
:10E78000118120490022012302A834F047F80DF13D
:10E79000200A034602A900228346504634F02EFB8D
:10E7A00002A8514633F0D5FF089B0F4EA3F10C0091
:10E7B000B04240F0A983BBF1FF3F00F0F080029A25
:10E7C00013782A2B00F0858252F80C1C19B35018CC
:10E7D00000211BE030200500640A0010541F0500D2
:10E7E000F0340500D8340500640A001060360500D6
:10E7F00068360500703605007C360500803505005A
:10E80000243505005C340500824204D0594012F8DA
:10E81000013F2A2BF8D1C8EB010800220F2302A8E0
:10E82000AF4934F030F8029B024653F80C3C984252
:10E8300000F20D844FF0FF3302A9504634F0DEFAA7
:10E8400002A8514633F085FF089BA3F10C00B042AB
:10E8500040F0248428461AF027FC4FE5DD0700F13C
:10E86000F380226952F80C3C002B40F0F380D9F879
:10E87000003093F8A830D80640F18D80029B53F801
:10E880000C3C002B7FF4CEAE0698964903689B683B
:10E890009847C7E6029B53F80C3C002B40F04081A0
:10E8A0003B7D032B00F2F0826360C26892F8341063
:10E8B00041F0080182F834103B751CE6702B00F023
:10E8C0006681752B7FF480AE039B53F80C3C032BC1
:10E8D00040F2BD830EAD4FF0FF335146042228466F
:10E8E00034F08CFA284602A934F0A3F903687E4E6E
:10E8F0000893C0F800B00E9BA3F10C00B04240F0AA
:10E90000DD8243F6122044F24041002208ABFAF7C0
:10E9100049F82CB120461AF0C7FB2046FCF7C0F995
:10E920000698704903689B689847089BA3F10C0000
:10E93000B0427FF4FAAE039BA3F10C00B04240F06A
:10E940005383029D16E5036868499B6898472369CD
:10E95000002153F80C2C04F110000B4634F012F88F
:10E9600055E640F2F512934200F02781B3F5FB7FA4
:10E970007FF42AAE5E4832F063FF2CB120461AF0D5
:10E9800093FB2046FCF78CF906985A490368584ACD
:10E990009B6898477CE559073FF570AF74E74FF0E7
:10E9A00000083AE706984F490368C7F804A09B6837
:10E9B000984728461AF078FB4F4E029DDAE40698F5
:10E9C0004E4903689B6898475BE501260EAD3E758E
:10E9D00004AA4B4928460DF1200A34F053FA334675
:10E9E00029465046474A1AF065FC0E9B424EA3F159
:10E9F0000C00B04240F07A820DF1140BD9F80000FF
:10EA000002215246FAF798FE3F4901AA584634F0CF
:10EA100039FA0123284659463A4A1AF04BFC059B1D
:10EA2000A3F10C00B04240F0558202212A46D9F8E9
:10EA30000000FAF781FE28461AF036FB50461AF01D
:10EA400033FBD9F80000C2E50698304903689B689B
:10EA5000984706E706982E4903689B6898472369FC
:10EA6000002153F80C2C04F110000B4633F08AFF00
:10EA7000D8E50323514600220EA834F0BFF90EA8B2
:10EA8000244933F019FF0E9B1B4E0446A3F10C00E2
:10EA9000B04240F05E82002C00F0C881FB68002B81
:10EAA00000F096811C490122504634F0EBF803989F
:10EAB000FB68012150F80C2C38F010FE039B53F832
:10EAC0000C3C984200F073810698144903689B68D7
:10EAD0009847F86838F00CF80023FB60D9E400BFD1
:10EAE0006034050024350500640A0010A86F050095
:10EAF00050260500F0350500640A0010D4340500E6
:10EB00002C3505001003001030350500108205007B
:10EB100098360500A0360500907F0500BC3605003C
:10EB20002CB120461AF0C0FA2046FCF7B9F818209C
:10EB300033F0C6FB012302A9069A04461AF0BAFB79
:10EB400002A8A749002233F0AFFF237A5D0740F106
:10EB50009B816368012B00F29781D9F80000A4E63D
:10EB6000A048A14938F066FA002800F07F8137F00C
:10EB7000BFFF06989D4903689A4A9B689847237A85
:10EB8000D9F8000043F001032372994E1FE5D9F82C
:10EB9000000007210022FAF7CFFDD9F8003095498F
:10EBA000586803689B6898472CB120461AF07CFA95
:10EBB0002046FCF775F88E4EBDE60EAD5146284650
:10EBC00034F0D3F80DF1200A02A9284634F031F8C8
:10EBD00050462946FBF77AF80E9B854EA3F10C00B0
:10EBE000B04240F09D81089B53F80C1C002972D163
:10EBF00050467C49132233F057FF23687E4A7F48F2
:10EC000040F2F517BB4214BF074617465146284647
:10EC100034F0ABF838462946069A22F031F90E9BBB
:10EC2000A3F10C00B04240F0C681089BA3F10C0098
:10EC3000B04240F0B4812CB120461AF035FA20469B
:10EC4000FCF72EF806986E4903689B68984772E6B1
:10EC5000D9F8000090F8A83059073FF5B6AE644ED9
:10EC6000B5E4D9F800300121986904F0BBFA72B616
:10EC7000644D65495B480E9538F0DCF963490F90A7
:10EC80000EA8FCF735FB0F980E9508B137F030FF52
:10EC9000082033F015FB5E4B05462B60514839F0D8
:10ECA000B5F9022168602246D9F80000E560FAF75C
:10ECB00043FDE06810B103685B6898472CB12046BB
:10ECC0001AF0F2F92046FBF7EBFF62B651490698BD
:10ECD0005CE600219FE514312846CDF838B033F0CA
:10ECE00088FF14224C49284633F0CCFF5146284671
:10ECF00033F09FFF5046294633F02BFD0E9BA3F1C6
:10ED00000C00B0423FF479AF53F8042C511E002A96
:10ED100043F8041C3FF771AF05A933F019FE6CE707
:10ED200005A804A9FAF71CFF05A908A8FAF77EFFB1
:10ED3000089C05A9284634F018F82046069A29466A
:10ED400022F09EF80E9B0446A3F10C02B24240F062
:10ED50000C81002C00F08380089BA3F10C00B042D2
:10ED600040F0A080059BA3F10C00B0423FF4D2AC70
:10ED700053F8042C511E002A43F8041C3FF7CAAC78
:10ED8000294633F0E5FDC5E407210122FAF7D4FC5A
:10ED90000698224903689B689847069820490368AB
:10EDA0009B689847002C7FF46DABFFF771BB1D4C3F
:10EDB00023681844B0F5C87F206009DDF86837F093
:10EDC00097FEB868184938F035F90023F8602360D9
:10EDD00006980B4903689B689847FFF75ABB00BF2A
:10EDE000D834050050260500D4A6050028360500B5
:10EDF000640A0010343505003C3405004C3405002D
:10EE000024350500E8330500541F0500A035050032
:10EE1000D8260500BC350500D83505007834050036
:10EE2000708A050030050010741D0500F86837F081
:10EE30005FFE7B7DBA6864F300037B7507F1080011
:10EE400021462346FC6052F80C2C33F09BFD0698BB
:10EE50003C61036898499B689847FFF71ABB06987E
:10EE600096490368089A9B68984775E706989449FD
:10EE700003689B68984782E6069892490368BA68D7
:10EE80009B689847FFF791BB2CB120461AF00CF90C
:10EE90002046FBF705FF06988B4903688B4E9B685D
:10EEA000984748E553F8042C511E002A43F8041CE7
:10EEB0003FF758AF294633F04BFD53E753F8042C86
:10EEC000511E002A43F8041C3FF71BAD05A933F07F
:10EED0003FFD16E553F8042C511E002A43F8041C8C
:10EEE0003FF7A3AD04A933F033FD9EE553F8042C9E
:10EEF0000DF1140B511E002A43F8041C3FF77EADA0
:10EF0000594633F025FD79E553F8042C511E002AAB
:10EF100043F8041C3FF74FAC05A933F019FD4AE450
:10EF200053F8042C511E002A43F8041C3FF75BAE33
:10EF300005A933F00DFD56E653F8042C511E002AA6
:10EF400043F8041C3FF70CAA0EA933F001FDFFF7AC
:10EF500007BA53F8042C511E002A43F8041C3FF74B
:10EF60009AAD08A933F0F4FC95E553F8041C481E4B
:10EF7000002943F8040C3FF7ECAE104601A933F02A
:10EF8000E7FCE6E653F8042C511E002A43F8041C63
:10EF90003FF7C0AB08A933F0DBFCFFF7BBBB53F86E
:10EFA000042C511E002A43F8041C3FF744AE2946A6
:10EFB00033F0CEFC3FE653F8042C511E002A43F8F0
:10EFC000041C3FF732AE05A933F0C2FC2DE653F81E
:10EFD000042C511E002A43F8041C3FF770AB08A90B
:10EFE00033F0B6FCFFF76BBB53F8042C511E002A1C
:10EFF00043F8041C3FF7A5AC0EA933F0A9FCA0E42C
:10F0000053F8042C511E002A43F8041C3FF7BBAAF6
:10F01000294633F09DFCFFF7B6BA53F8042C511E75
:10F02000002A43F8041C3FF7A8AA05A933F090FC76
:10F03000FFF7A3BA53F8042C511E002A43F8041C0E
:10F040003FF7EEA908A933F083FCFFF7E9B92048A0
:10F0500033F0A5FF53F8042C511E002A43F8041C7A
:10F060003FF778A9FFF791B953F8042C511E002AF5
:10F0700043F8041C3FF75BA908A933F069FCFFF7CC
:10F0800056B953F8042C511E002A43F8041C3FF7CC
:10F09000B0A908A933F05CFCFFF7ABB953F8042C16
:10F0A000511E002A43F8041C3FF7D4AB05A933F0E6
:10F0B0004FFCFFF7CFBB00BFA43605008835050025
:10F0C000483605000C350500DC340500640A0010E4
:10F0D0006827050038B50446FCF7D8F8627D0023A0
:10F0E000064D074863F300024FF0FF312375A0601F
:10F0F0002560627523616160204638BD00370500D8
:10F10000700A001010B50B4682B0496802461868B4
:10F110006B4603C30B46D90707D55B10D45800993B
:10F12000D0186158884702B010BD02EB6300009907
:10F13000884702B010BD00BFD0F8100132F048B9C6
:10F14000A0F10400FFF7F8BF10B50446D4F8100191
:10F1500032F052F8D8B1D4F8100132F039F9C0B217
:10F160003F2815D018281AD0D4F80C21D4F80C3127
:10F170000D2808BF0A20013322441072DBB2C4F804
:10F180000C31D4F8100132F037F80028E3D110BD6B
:10F1900094F8143143F0010384F81431D6E794F85D
:10F1A000143143F0020384F81431CFE770B50546FB
:10F1B00008460C4638F045FFD5F8103101465B692A
:10F1C00020460122BDE8704038F088BAA0F1040062
:10F1D000FFF7ECBFD0F8100132F0EEB8A0F1040058
:10F1E000FFF7F8BF10B5044A044B044680E80C0052
:10F1F000FCF73CF8204610BD38370500A02D05006F
:10F20000A0F10400FFF7EEBF10B5064A064B044616
:10F2100080E80C00FCF72AF82046FBF741FD204669
:10F2200010BD00BF38370500A02D0500A0F1040077
:10F23000EAE700BF2DE9F041D0F8103182B0064670
:10F2400080B1324A00248DE81400314D6A4658627C
:10F250001C6203CA9D639862D96203F118000122FF
:10F2600031F04AFB96F81431304603F0FE036FF399
:10F27000410386F814310021FCF70EF830460321D3
:10F28000FCF70AF8234B04361B685F68FC6807F13B
:10F2900008080CB90FE01446216901258E4232BFDF
:10F2A000A268E2680025002AF5D12DB98E420CD85B
:10F2B00002B0BDE8F08144463B69A34205D0204638
:10F2C00033F0BFF801698E42F2D9002CF0D0A0458E
:10F2D0001AD02569AE422CBF00250125142032F03A
:10F2E000EFFF014628B1002306610370436083608D
:10F2F000C36043462846224633F0A5F8BB69013374
:10F30000BB6102B0BDE8F0810125E7E749F10000EB
:10F3100005F10000E402001030B590F8143183B01C
:10F32000D90704460DD49A0709D5174A6FF341034C
:10F33000106884F8143107210022FAF7FDF903B0B0
:10F3400030BD114902686FF3000380F81431096879
:10F3500001A8956BFAF75AF820460199A847019B36
:10F360000A4AA3F10C00904202D194F81431DAE772
:10F3700053F8042C511E002A43F8041CF5DC69469E
:10F3800033F0E6FAF1E700BFE4020010640A00106F
:10F390002DE9F047D0F8083184B0044607E00A7A36
:10F3A00001330A2A0BD0B3F5807F08BF0023D4F8BD
:10F3B0000C21E1189342F2D104B0BDE8F087DFF8E8
:10F3C000D88004AE46F80C8D3046142133F011FC81
:10F3D000A8F10C074FF0000919E0019B304653F8E3
:10F3E0000C5C53F8082C0135954203D853F8042CD3
:10F3F000002A03DD294633F0FCFB019B53F80C2C5B
:10F4000003F802A0019BA3F10C02BA4230D1D4F858
:10F410000821D4F80831224492F808A00133DBB265
:10F42000BAF10A0FC4F80831D7D1314603A8CDF894
:10F430000C8033F0A6FC174B0434186802AA012193
:10F440000294FAF779F9039BA3F10C00B84216D1A4
:10F45000019BA3F10C00B842AED053F8042C511E0E
:10F46000002A43F8041CA7DC02A933F071FAA3E7D1
:10F4700043F8049C43F80C5C03F80590C7E753F885
:10F48000042C511E002A43F8041CE1DC694633F0C9
:10F490005FFADDE7E4020010700A00102DE9F8437E
:10F4A0000446894690461F46FBF7F0FE0E480025AD
:10F4B00000F108034C3023606060C4F80C51582000
:10F4C000C4F8085132F0FCFE4946064642462B4637
:10F4D00031F062FE3046C4F81061394631F088FEE2
:10F4E0002046BDE8F88300BF3037050038B5164D1B
:10F4F0000022296813460446486941F29371FBF7DC
:10F50000E5F81249FBF7A4FEFBF7C8FD29680022C5
:10F510001346E06048694BF66D41FBF7D7F80C499C
:10F52000FBF796FEFBF7BAFD29680022134620611F
:10F53000486942F2C351FBF7C9F80021FBF788FE86
:10F54000FBF7ACFD606138BDE4020010CDCC4C3D52
:10F550000000C07F0022034610B503F8012B0133E1
:10F56000427003F8012B03F8012B03F8012B03F879
:10F57000012B03F8012B03F8012B03F8012B03F8EF
:10F58000012B03F8012B04461A70FFF7AFFF20464A
:10F5900010BD00BF2A4B2DE9F0471B6846699F69E3
:10F5A0008246BC6807F104082146404603F0ECFEA1
:10F5B0000546404603F060FC00283ED1FB689C42B3
:10F5C00015D095F86030DB0711D53146284603F099
:10F5D0002FFF21460646404603F022FF04462146FF
:10F5E000404603F0D1FEFB680546A342E9D1284618
:10F5F00003F054FFBB688146A3421ED0214640461B
:10F6000003F08CFD04462146404603F0BDFE49460A
:10F61000064603F073FF696A8146726A284604F061
:10F620001BF8BB683546A342E8D13046DAF814200F
:10F63000716ABDE8F04704F00FB82E46F5E700BF49
:10F64000E40200102DE9F04F8B4E8146306885B002
:10F65000806901939DF84830043090460F4602932C
:10F6600003F056FD0446B8F1000F00F08C81002530
:10F67000CDF80C904446AA4600954FF0010B814608
:10F68000B84614E009F150010AF01F020BFA02F229
:10F69000086820EA020008600AF1010A002FB8BFDA
:10F6A0007F42A24549F8057005F1040523D232686E
:10F6B00058F80510D26892685059F9F7EDFB0746E3
:10F6C0000028DFD06C480123026858F80510D06884
:10F6D0003A46806800934059F9F7D8FB002F0AF0AA
:10F6E0001F0280F27B810BFA02F2D9F8501011430D
:10F6F000C9F85010D0E7009B4C46DDF80C90002B69
:10F7000000F041814FF08A41119834F047FA35F00A
:10F710004BFA34F045FC94F860200299B4F862305A
:10F7200061F3041260F30B03D2B22568A4F86230CF
:10F7300042F00802D9F80C7084F86020002D00F027
:10F740008380109B04F11401E362234603E01A68EE
:10F75000954238BF154604339942F8D10E9B4FF0BD
:10F760000008656123624146184634F0D3FB002847
:10F7700000F00481019B2846E36134F0B7F9019958
:10F7800034F00CFA0E9934F0BDFAA0610F9BD9F851
:10F790001450002B00F0F0803368DFF8DC809869AB
:10F7A000043003F069FB002868D0D9F814001099E0
:10F7B000256401F10048014634F0F0F9414607465E
:10F7C000404634F0E3F8216A34F0E8F9014638465F
:10F7D00034F0DAF835F040FC07463946284634F074
:10F7E00099FB00B13D4665623946E06934F07EFB25
:10F7F00094F8603000283AD160F3410384F8603017
:10F8000094F8603043F0010384F860300F9B002BC4
:10F8100000F0C78019685A689B68C9F80010C9F8D9
:10F820000420C9F808304846FFF7B4FE94F8603069
:10F83000326843F00403906984F8603003F076FD89
:10F84000012005B0BDE8F08F6368002B7FF479AF2D
:10F85000A368002B00F09E80D9F8108040464146F6
:10F8600034F062FB00287FF46CAF474669E743F051
:10F87000020384F86030C3E7E4020010D8F80030D7
:10F880009B6903F104089968404603F0C9FD0146ED
:10F89000404603F079FD90F860200346120784D5B6
:10F8A00038460021D3F81C8034F034FB00283FF4A4
:10F8B0007CAF4046002134F02DFB00283FF475AFAB
:10F8C0000F9BD9F80000196800F1004034F066F988
:10F8D0000F9B83465968D9F8040034F05FF901465C
:10F8E000584634F051F80F9B83469968D9F80800C0
:10F8F00034F054F90146584634F046F83A49834604
:10F9000034F0EAFA00283FF450AFE5694046294652
:10F9100034F000FB00285FD05846344934F0FAFA3E
:10F9200000283FF442AF59464FF07E5034F02CF897
:10F930004FF07C5134F032F935F08EFB3946804679
:10F94000109834F02BF9414634F028F94146074627
:10F950004FF07E5034F018F80146384634F0D2F9B2
:10F9600035F07AFB07463946284634F0D3FA0028AA
:10F970003FF41BAF3D4618E7284618E7C4F81C8043
:10F98000C4F8188002E7204604F022F8002005B0F1
:10F99000BDE8F08F94F8603065F3C30384F86030FD
:10F9A000CFE60F984B4603F8010B013389F80100AD
:10F9B00003F8010B03F8010B03F8010B03F8010B2B
:10F9C00003F8010B03F8010B03F8010B03F8010B1B
:10F9D00003F8010B187026E745469DE7012309F15E
:10F9E0005001009352E600BF3333733F333373BF8C
:10F9F000014B0360704700BFA0370500002070472F
:10FA00000020704710B5034B04460360FBF748F92C
:10FA1000204610BDA03705002DE9F0470446D4F874
:10FA2000D830D0F8E800984227D0D4F8EC30D4F899
:10FA3000F420984223D0A0F10C0310F80CAC10F87D
:10FA40000B9C10F80A8C10F8097C50F8086C50F8E0
:10FA5000045CC4F8E83094F8343084F8A4A067F368
:10FA6000410368F3820369F30003C4F82451C4F826
:10FA7000206184F83430BDE8F087BDE8F08752F8A3
:10FA8000043C93F8ECA193F8ED9193F8EE8193F890
:10FA9000EF71D3F8F061D3F8F451FBF701F9D4F822
:10FAA000F4301A1FC4F8F42053F8043C03F5FC7139
:10FAB00003F5F672C4F8EC30C4F8F010C4F8E8208E
:10FAC000C9E700BF2DE9F04791F8A47001F13808AB
:10FAD00007EB4707BF0008EB07090C460546D9F8B6
:10FAE00008109068164633F04FFFD4F8B01033F08A
:10FAF0004DFFD4F8BC1033F047FFD9F8041082460C
:10FB0000706833F041FFD4F8AC1033F03FFFD4F805
:10FB1000B81033F039FF58F807108146306833F0D9
:10FB200033FFD4F8A81033F031FFD4F8B41033F019
:10FB30002BFFC5F804902860C5F808A02846BDE84A
:10FB4000F08700BF2DE9F0470C4694B0054690467B
:10FB5000994600293DD0042900F0BE80052900F017
:10FB6000A18087680026D7F800A00F96DAF82C004D
:10FB7000109611961296139633F0BCFFDAF8201007
:10FB800034F0C0F8D7F804A00F90DAF82C0033F066
:10FB9000B1FFDAF8201034F0B5F8BF681090F86AB9
:10FBA00033F0A8FF396A34F0ADF86B6811901A6829
:10FBB00018460FA9D36806AA9847012C4AD0022CF0
:10FBC00000F0A280032C00F0B480304614B0BDE8F1
:10FBD000F087D0F8F830D0F80061D0F8FC400FAAD8
:10FBE0000CA8294611930F961094FFF76BFF95F818
:10FBF00034300E98DA0719D433F03CFB04460D98E4
:10FC00000D4633F037FB06460C980F46CDE900450C
:10FC1000CDE9026733F02EFB5A4ACDE90401404694
:10FC2000494638F00FF914B0BDE8F087564934F072
:10FC300069F833F01FFB04460D460D98524934F025
:10FC400061F833F017FB06460F460C984E4934F026
:10FC500059F8DBE7069B089E079C09A829460CAAD1
:10FC60000E930C960D94FFF72DFF95F834300B98FA
:10FC7000DB0773D433F0FEFA04460A980D4633F0DE
:10FC8000F9FA064609980F46CDE90045CDE9026725
:10FC900033F0F0FA3D4ACDE904014046494638F0D8
:10FCA000D1F893E7D0F80C0133F0E4FACDE9000184
:10FCB000D5F8100133F0DEFACDE90201D5F81401D0
:10FCC00033F0D8FA324ACDE904014046494638F0CB
:10FCD000B9F814B0BDE8F087D0F8F80033F0CAFAEC
:10FCE000CDE90001D5F8FC0033F0C4FACDE90201FA
:10FCF000D5F8000133F0BEFA264ACDE904014046AA
:10FD0000494638F09FF861E7069833F0B3FACDE939
:10FD10000001079833F0AEFACDE90201089833F0FC
:10FD2000A9FA1D4ACDE904014046494638F08AF84F
:10FD30004CE70F9833F09EFACDE90001109833F0AC
:10FD400099FACDE90201119833F094FA134ACDE9FA
:10FD500004014046494638F075F837E70A4933F060
:10FD6000D1FF33F087FA04460D460A98064933F06E
:10FD7000C9FF33F07FFA06460F460998024933F06F
:10FD8000C1FF81E7283805003333CB4184380500B3
:10FD90006438050044380500A4380500C43805005F
:10FDA0002DE9F04F90F855A185B08146BAF1000FCA
:10FDB00039D0002402E00134A24534D9D9F8083002
:10FDC00053F82450D5F82080696A404633F0E6FEA7
:10FDD000164B07461E68B06B33F088FE83465946C3
:10FDE000384634F097F80028E5D04146584633F0BD
:10FDF00089FF34F047FE68628046384633F03AFAAD
:10FE000075682E68CDE90001404633F033FACDE93C
:10FE100002012246B36828460549984799F855A13A
:10FE20000134A245CAD805B0BDE8F08FE402001045
:10FE3000E438050070B50546406886B0046801AE38
:10FE4000C5F8F810C5F80C11C5F8FC20C5F810214C
:10FE5000C5F80031C5F8143105F58671A36832463E
:10FE600098470024AB68315918590434F8F7FEFF5D
:10FE70000C2CF7D106B070BD00EB8203022A10B43F
:10FE8000C3F8F81004DDC3F80C115DF8044B70479B
:10FE9000D0F8F810D0F8FC20D0F800315DF8044B11
:10FEA000FFF7C8BF2DE9F041D0F8088086B00546BD
:10FEB000002401AE58F80470F86A33F01BFE396A6A
:10FEC00033F020FF305104340C2CF3D1686805F571
:10FED000867403682246DB6831469847D5F80C21C2
:10FEE000D5F81401C5F8F820D5F81811D5F81C215B
:10FEF000D5F81071C5F800016868C5F80411C5F897
:10FF00000821C5F8FC700368214632469B68984773
:10FF10000024AB68315918590434F8F7A7FF0C2CAA
:10FF2000F7D106B0BDE8F08170B505460E46002455
:10FF3000AB68315918590434F8F798FF0C2CF7D1F5
:10FF40002846BDE87040FFF7ADBF00BF2DE9F04F78
:10FF50009BB090F8553106AF7A629A0002F10A031D
:10FF600003F4FF63ADEB030D06ACADEB030D0646EA
:10FF700006A8F86237F077FCF36923B1336A06F11B
:10FF80001400F96A984796F85551002D00F0408109
:10FF90004FF0000A0022BA62AD00D346D04606EB0D
:10FFA0000A03D3F80C11FB6A53F80A0033F0ECFC97
:10FFB000002144F80A00814633F084FF28B9BBF1E0
:10FFC000020F40F22A814FF001080AF1040AAA4503
:10FFD0000BF1010BE3D1B8F1000F00F01981256896
:10FFE0000021284633F06EFF70B16068002133F0C5
:10FFF00069FF48B1A068002133F064FF20B1002000
:020000021000EC
:1000000001223862BA6240E0B86A35F025F8AC499E
:10001000386233F061FF002840F0FA80D7F820B052
:10002000D7F824A080462846594633F06BFE06EBED
:100030000803D3F84851814607F13002002142F805
:100040000890284633F066FF08F10408494690B14D
:10005000504633F0A3FD20F000494946284633F0CE
:100060003BFF494638B1284633F04CFE0146504626
:1000700033F094FD8246B8F10C0F02D054F808001A
:10008000D2E70023C7F824A0BB6296F834309A0662
:1000900040F10081FB6A19685A689B68F9633A6409
:1000A0007B6496F8550100240328F86128D9FD6A7D
:1000B000D7F81CC04FF00C084FF0030A07F13C0BB7
:1000C00006F1240955F80820F36A48460AF1010AA6
:1000D0004BF8082053B1336B984701465BF8080092
:1000E00033F05CFD96F855C14BF80800BA6A002A57
:1000F00040F09F80D44508F10408E3D8C7F81CC03D
:10010000BB6A002B40F0CE80786A396A33F0FAFD82
:10011000D6F83C21FB69B8613A61002B00F0D4802D
:100120000024D6F808A0D7F81C90254607F13C0B10
:10013000FE605AF804605BF80400716B33F024FC35
:1001400020F000484046002133F0BCFE00283ED19C
:1001500096F839305B073AD5B969404633F01EFD51
:10016000736A78601946BB6033F0D4FE7A68BB6866
:1001700060B11146184633F0C5FD0146786A33F088
:100180000DFD396A786233F0BDFDB861B86A08B90F
:10019000022D1CD8B66A3046314633F0C5FEB0B9E0
:1001A0004046396A33F0AEFD396933F0F7FC20F090
:1001B00000484046314633F0ADFE40B1414630463E
:1001C00033F0A0FD0146386933F0E8FC38610135B1
:1001D0004D4504F10404ACD3FE683A4BBA6A1B687F
:1001E0001869002A46D0002396F83550D6F84041C9
:1001F0003A6A01933B6905F0010500920293594662
:10020000FA697B6A04950394FFF71CFA002834D13D
:1002100000205437BD46BDE8F08F4946484633F0CC
:10022000BDFC0146B86A33F0B1FB4FF00108B8627B
:10023000CBE6B3685BF8080053F80830596BC7F891
:1002400008C033F0A1FB33F015F802460B4633F03B
:1002500065F8C7E90401204633F00CF802460B4666
:10026000D7E9040132F0A8FE33F03AFBD7F808C012
:1002700004463FE707F13003B6E796F85521F96ADF
:10028000920006F5867037F0EEFA01205437BD462D
:10029000BDE8F08F7068F96A036807F13C029B685B
:1002A0009847FEE6204634F0D7FE0549386233F021
:1002B00013FE0028ACD196F85501F86124E700BF81
:1002C000ACC52737E402001007F13C0B85E700BFFF
:1002D0002DE9F84F214C814620680E4690F8A81071
:1002E00098468B0700AF924628D41046002133F081
:1002F000FDFD044610BB99F8552109F1F80B920059
:1003000002F10A0303F4FF63ADEB030D684659469F
:100310006D4637F0A8FAB8F1000F09D04FEA880807
:100320002859315933F032FB285104344445F7D170
:10033000524648462946FFF709FE18B90020BD4637
:10034000BDE8F88F99F8552158469200294637F0B4
:100350008AFA0120BD46BDE8F88F00BFE402001014
:100360002DE9F04F8BB0044600AF0D461846002132
:10037000BB61BA6033F0BAFD002840F0F480B96880
:100380000868D4F8F81033F0FFFABA688346D4F856
:10039000FC10506833F0F8FABB680646D4F8001138
:1003A000986833F0F1FA31468046304633F0F6FB78
:1003B00059460646584633F0F1FB0146304633F0C5
:1003C000E5FA41460646404633F0E8FB0146304632
:1003D00033F0DCFA34F040FE9A49064633F07CFDF7
:1003E000002840F0F980386D014633F09DFD02464B
:1003F000C8B92B7A590716D56B68012B13D13B6D01
:100400003146B8693B623A6033F07CFC3A68786206
:100410004EF289014AF6765007F12003F8F7C2FA46
:10042000002840F0F38094F83430C3F300113961B0
:10043000002940F0BC805A0640F1D980D4F83451EC
:100440004FF07E51284633F065FD002800F0A7806C
:10045000B969304633F056FC0146284633F09EFB1E
:1004600034F092FA4FF07E51054633F053FD0028E8
:1004700000F09D80284633F093FD80B278617B695F
:10048000012B40F2948094F85521C7F804D09200D3
:1004900002F10A0303F4FF63ADEB030DC7F80CD0C0
:1004A000ADEB030D684604F1F801C7F81CD037F036
:1004B000DAF994F85531FBB178693B6033F01AFBF7
:1004C0003B68D7F80C80D7F8089006469D004FF09F
:1004D000000B9A4604EB0B03D3F8F81059F80B0005
:1004E00033F052FA314633F00DFC48F80B000BF1B3
:1004F000040BAB45EED15346DFF854B1DBF80020D6
:1005000092F8A850C5F34005002D40F085800126E3
:10051000A3B1FB68D7F81C80A3F104094FF0000ACF
:10052000D8F8000059F8041F33F030FA48F8040BEB
:1005300094F855310AF1010A9A45F1DB2046F96930
:10054000BA69FFF703FD7B690136002D08BF054638
:100550009E4268D0DBF8003093F8A8309B075BD44C
:1005600094F85531D4E72B7AB86943F010032B7215
:10057000002133F0A7FC344B3449002805F1100565
:1005800008BF1946284614BF13220D2232F08CFAF8
:1005900000233B6138692C37BD46BDE8F08FD4F8A5
:1005A00028510021284633F08DFC00283ED000253C
:1005B000B968BA692046FFF7C9FC002818BF0125B1
:1005C00094F834303D6138696FF3C3032C3784F8F5
:1005D0003430BD46BDE8F08FB968BA692046FFF7F0
:1005E000B5FC386138692C37BD46BDE8F08F284628
:1005F000582118F077FD00287FF420AF28465921B4
:1006000018F070FD00287FF419AFD0E7B869796A57
:1006100033F0C4FAB86106E77B6838699D462C3729
:10062000BD46BDE8F08F7B689D46C1E72946304650
:1006300033F068FB34F0A8F933F0B2FC80B2786193
:100640001DE700BFACC527375C39050048390500F8
:10065000E40200102DE9F04F044691B00D46D0F8A9
:100660002401D4F838110B92039333F04BFB002193
:1006700005909DF86C8033F039FC002840F08381B0
:1006800094F83560039BC6F3410553F8257005F1D6
:100690003E0354F82310384633F078F9039BC6F331
:1006A000C10A53F82A900AF13E0354F82310069029
:1006B000484633F06BF9C6F341160B9A06F13E0338
:1006C00054F82310079052F8260033F05DF90B9B85
:1006D0000699064653F8250033F056F90B9A05465D
:1006E000079952F82A0033F04FF907F10047824684
:1006F0005146384633F052FA09F1004983462946FB
:10070000484633F04BFA0146584633F03DF9294646
:100710008346384633F042FA51460546484633F0A0
:100720003DFA0146284633F031F90146584634F087
:100730009FFA0546B8F1000F00F01981B64933F071
:10074000DFFB002840F03C811A99284633F026FA56
:1007500026F0004131F0E0FDB049824633F0BCFBA9
:10076000002840F02981D4F8308100214046D4F897
:100770002CB133F0CFFB68B11A98014633F006F97B
:10078000034619464046009333F0A6FB009B002821
:1007900040F01C815946504633F0B4FA34F0F4F876
:1007A00033F0FEFB1FFA80F8404633F0A3F982468F
:1007B0005146284633F0A6FA51460290304633F0AF
:1007C000A1FA4FF07C510890029833F0E7F90299B2
:1007D00033F0E4F901464FF07E5033F0D5F894F849
:1007E0003550B8F1010FC5F3411303F13E024FEA52
:1007F00083030193019954F8222010AB0B44099014
:1008000043F80C2C40F2F980854A136893F8A8301D
:10081000C3F34003002B40F0CF80A8F102081FFA79
:1008200088F808F101089B46CDF828809A460126F1
:100830005BE04846099933F0B1F9029980463846A1
:1008400033F0ACF9414633F0A1F8099980463846B7
:1008500033F0A4F902990746484633F09FF9014660
:10086000384633F091F80AF1010AC14607465FFAAB
:100870008AFAC5F341080698394633F087F810A97B
:1008800001EB880810AA48F80C0C49460798C5F3F4
:10089000C10502EB850533F079F8019B0DF14008A5
:1008A000984445F80C0C58F80C0C089933F06EF885
:1008B0000DA948F80C0C059A2046FFF747FB0A9B48
:1008C000BBF1000F08BF83469E4206F1010600F00F
:1008D000968053490B6893F8A8309B076CD494F822
:1008E0003550C5F341139B000193D4F844314FFABE
:1008F0008AF29A429DDB304633F0FCF8029933F0DD
:100900004DF9074634F084F88246384634F072F9DF
:10091000039FC5F3410857F82830C5F3C10203F11E
:10092000004351460490184657F82290009333F044
:1009300035F904990746484633F030F90146384600
:1009400033F024F8009B07461946049833F026F943
:10095000494603465046009333F020F9009B014678
:10096000184633F011F84FF0000A814683E72D490D
:1009700033F0BCFA00283FF4E7AE28462A4933F0AA
:1009800005F80546E0E62B7A059843F010032B7234
:10099000002133F097FA254B2549002805F1100571
:1009A00008BF1946284614BF13220D2232F07CF8E6
:1009B000002011B0BDE8F08F002011B0BDE8F08F2D
:1009C0002846194932F0E0FF0546BDE61846414683
:1009D00032F0DAFF0146404633F0E0F834F03CFBF9
:1009E000014632F0D3FFD4F82C11804633F092FA4E
:1009F00000283FF4CFAEC346CCE64FF0000B2046B4
:100A00000B99059AFFF7A2FA00280CBF584601205F
:100A100011B0BDE8F08F00BFBD3706B5ACC52737B4
:100A2000E4020010BD370635DB0FC9405C39050014
:100A3000483905002DE9F041054690F83500144687
:100A4000C0F34107C0F3C10282B00E4654F827003C
:100A500054F822101F469DF8208031F05DFCB8F15B
:100A600003025342534100900193284631463A46CF
:100A70002346FFF7EFFD02B0BDE8F0812DE9F04F0E
:100A80008DB0B84B02AF07F1180804460E469146E8
:100A90000FCB88E80F00002505F1580A5FFA8AFAA3
:100AA0005146304618F01EFB002840F00D810135FC
:100AB000032DF1D100234FF0000AFB603B617B6105
:100AC00049253046294618F00DFB002840F0EB8000
:100AD0000135EDB24C2D0AF1040AF2D194F85521FA
:100AE00004F1F80392007B6002F10A0303F4FF6350
:100AF000ADEB030D0DF1080A5046796836F0B3FEF0
:100B000094F834502B0700F11281C5F34005002DF5
:100B100000F09C80BD692846294633F005FA98B953
:100B200094F8A430284603EB430304EB8303196CC9
:100B300032F02CFFD4F8B01032F026FFD4F8BC10FD
:100B400032F024FFCAF80000FD692846294633F038
:100B5000EBF998B994F8A430284603EB430304EB6F
:100B60008303D96B32F012FFD4F8AC1032F00CFFD3
:100B7000D4F8B81032F00AFFCAF804003D6A2846DB
:100B8000294633F0D1F9A0B994F8A43004F1380221
:100B900003EB430352F82310284632F0F7FED4F853
:100BA000A81032F0F1FED4F8B41032F0EFFECAF81B
:100BB0000800002384F854313046452118F092FA99
:100BC000B0B194F85511032912DDA368DA6892F8E0
:100BD0003920500700F1EA800C33032505E053F873
:100BE000042F92F8392052077DD401358D42F6DB6F
:100BF00094F85451002D7FD1DFF8708130464621A2
:100C000018F070FA98B1B9F1010F30464FF0460173
:100C10004FF0000200F0BE8018F078FA94F83430FB
:100C2000D90702D5504932F0B9FFC4F82401304643
:100C3000532118F057FA002840F09A8009F1FF3349
:100C4000032B2CD8DFE803F08B15818158F805B011
:100C50005846594633F068F9621930B9D2F8F8109D
:100C6000584632F093FE4AF8050004350C2DEDD1BC
:100C70009FE7D4F82401D4F8381133F043F8CDF8C5
:100C800000800346314620465246FFF769FB30B1EB
:100C900094F8552178689200514636F0E4FD2C37DF
:100CA000BD46BDE8F08F29463046002218F02EFAE6
:100CB00094F834302C49DB0701D532F06FFF07F18F
:100CC0000C034AF8030003E751463046002218F0AF
:100CD0001DFA94F834302449DB0701D532F05EFF69
:100CE00048F82500E3E6EDB230464521002218F031
:100CF0000DFA84F854517862D7F824804046414672
:100D000033F012F900287FF477AF94F834305B07A2
:100D100036D594F854314AF8258003F13E0254F850
:100D200022105AF8230032F02FFE804666E7002595
:100D300058F805B05846594633F0F6F808B94AF85D
:100D400005B004350C2DF3D133E7CDF800903146D2
:100D5000204607F10C025346FFF76CFE97E7D4F8E4
:100D6000200188E7B83705003333CB410000C07F4E
:100D700030465321002218F0C9F9C4F840015DE75C
:100D800005F13E0354F82310404632F0FFFD4AF8C7
:100D9000250033E718F0BAF994F83430DD0702D5AE
:100DA000034932F0FBFEC4F8200140E703259BE72E
:100DB0003333CB418B684A680968C0F8B820C0F863
:100DC000BC10C0F8B4307047054B1B689B681B7D96
:100DD000013B022B8CBFD0F82001D0F824017047D2
:100DE000E402001070B50646006868B1756A74695F
:100DF0000435AC4206D254F8040BF9F751FFA54272
:100E0000F9D83068F9F74CFF304670BD0E4B10B57D
:100E1000044640F8D03BFFF7E5FFE36A23B104F155
:100E20002400014603229847E36923B104F114002A
:100E3000014603229847A06808B1F9F731FF204620
:100E4000FAF714FA204610BDF8370500104B10B51C
:100E5000044640F8D03BFFF7C5FFE36A23B104F135
:100E60002400014603229847E36923B104F11400EA
:100E7000014603229847A06808B1F9F711FF204600
:100E8000FAF7F4F92046F9F70BFF204610BD00BF32
:100E9000F8370500F8B5426803680446D31A9B107A
:100EA0000F4605D05A00934226D96FF0030600E0A2
:100EB0000426304631F004FA054694E809001B1A6E
:100EC0009B109A003968AF1807D045F8231094E8B2
:100ED00009001B1A9B109A00AF1823B1014628463F
:100EE00036F0CAFC2068043708B1F9F7D9FE2E4461
:100EF000A66084E8A000F8BDB2F1804FD5D2DE0034
:100F0000D7E700BF30B5184D83B02B680446D86AC8
:100F10000191FAF7D3FD94F85531042B06D92B68CB
:100F20001249586803689B68984700BEE3682269C5
:100F3000934211D0019A13B11A60E368019A043305
:100F4000E36094F8553182F8383094F85501431C29
:100F500084F8553103B030BD04F1080001A9FFF752
:100F600099FF019AEDE700BFE40200106C3905001B
:100F70002DE9F04F0446406897B010B103685B68F4
:100F80009847304D00222968134648694FF22141A5
:100F9000F9F79CFB0DF11C0805AA06462A494046B4
:100FA00031F070FF30464146FAF756F901460DA878
:100FB000FAF726F90DA8F8F7C1FC0D9BDFF8909021
:100FC0000646A3F10C00484540F0D9820DF1180BFC
:100FD000079BA3F10C00484540F0EB8241F6AE437D
:100FE0009E4200F048824EF29C539E4200F04382A3
:100FF0004EF29D639E4200F05E8245F208139E42CF
:1010000028D041F293139E4224D041F60C339E42E5
:1010100020D0B6F5F47F1DD041F2DE139E4200F0E1
:101020006B8245F60F539E4200F070824EF6866347
:101030009E4200F07582042031F042F9034B0360B8
:10104000606010E0E4020010A0390500508D05003A
:10105000640A0010402031F033F92B6806465969C4
:1010600021F088F866602B680022586941F6E91182
:101070001346F9F72BFBC249FAF7EAF8FAF70EF82C
:10108000296800221346C4F8240148694BF6FD0183
:10109000F9F71CFBBA49FAF7DBF8F9F7FFFF296803
:1010A00000221346C4F82001486947F2E051F9F7DD
:1010B0000DFB0021FAF7CCF8F9F7F0FF29680022C0
:1010C0001346C4F82801486943F65A71F9F7FEFA45
:1010D0000021FAF7BDF8F9F7E1FF2968002213466D
:1010E000C4F83401486943F66E41F9F7EFFA00217C
:1010F000FAF7AEF8F9F7D2FF296800221346C4F8D0
:101100002C0148694DF6A361F9F7E0FA9D49FAF719
:101110009FF8F9F7C3FF296800221346C4F830018D
:10112000486941F2D231F9F7D1FA0521FAF784F88A
:10113000F9F7B4FF32F00EFF296800221346C4F815
:10114000440148694FF6A751F9F7C0FA8E49FAF7FA
:101150007FF8F9F7A3FF8D4932F0D4FD296800220A
:101160001346C4F84801486940F6A861F9F7AEFA99
:101170008549FAF76DF8F9F791FF844932F0C2FD1D
:10118000296800221346C4F84C01486941F6A96158
:10119000F9F79CFA7E49FAF75BF8F9F77FFF7B498C
:1011A00032F0B0FD296800221346C4F850014869A6
:1011B00048F25B71F9F78AFA0121FAF73DF8FAF77C
:1011C00025F894F834302968002260F3861384F8F7
:1011D00034304869134645F6E271F9F777FA002191
:1011E000FAF72AF8FAF712F894F83430296860F31D
:1011F000C713002284F834304869134642F27F71E5
:10120000F9F764FA5A46064662490DA831F03AFEEB
:101210000DA93046FAF720F8014604A8F9F7F0FFC7
:101220000D9BA3F10C00484540F0B781049951F89B
:101230000C3C002B40F026812B680022586944F6B4
:10124000D6311346F9F742FA5349FAF701F8F9F79C
:1012500025FF524EC4F8400106F1200C0DF1340E6A
:1012600030687168B268F36877460FC71036664514
:10127000BE46F5D1306829680022134638604869B7
:1012800046F2EE21F9F722FA3D49F9F7E1FFF9F7C5
:1012900005FF0DAEC4F83C014FF0000A4046F6F7DA
:1012A00071FB09A8F6F76EFB0BA8F6F76BFB00279E
:1012B0002B680022F15B58691346F9F707FA02AA76
:1012C0000346374905A8009331F0DCFD009B05A9D2
:1012D0001846F9F7C1FF01465846F9F791FF08EBA8
:1012E00087005946F6F736FD8179069B8907A3F1F9
:1012F0000C0207F1020709D590F804E0016801200B
:1013000000FA0EFE08684EEA000008604A4540F008
:101310001181059BA3F10C00484540F01881062F70
:10132000C6D13C2030F0CCFF4146074609AA0BABA2
:10133000F7F71CFD20463946FFF7E4FD504508D07D
:101340002B6802465868174903689F685346B84798
:1013500000BE2B680022A768F1885869134657F829
:101360002A70F9F7B3F9BAF1020F0CBF0E490F4911
:101370004FEA8A0CCDF804C0F9F76AFF18E000BF05
:101380000000C8420AD7233C00606A470000704250
:1013900000009643D8340500CDCC4C3FC83705003B
:1013A000CC260500AC390500000020450000A04215
:1013B000F9F774FE01463846F7F74CFD2B6800221A
:1013C000DDF804C0A76831895869134657F80C70D6
:1013D000F9F77CF97D49F9F73BFFF9F75FFE7C49A6
:1013E00032F090FC2968D4F808E00022DDF804C04F
:1013F00078621346486971895EF80C70F9F766F9EE
:101400007449F9F725FFF9F749FE0AF1010ABAF123
:10141000030FB86206F10C066F4F7FF43FAF204612
:10142000FEF7BEFCA3689B68986A014632F07CFD1B
:1014300000284AD1606804F1F801036842469B68BD
:10144000984794F8553173B100252E46A36858F893
:1014500005105859F7F70AFD94F855310136B34293
:1014600005F10405F2D8049BA3F10C0048457AD19C
:1014700017B0BDE8F08F042030F022FF574B036017
:101480006060F0E50DA8F8F7BDFF0D980E9B1B1AE4
:101490009B10032B05D000283FF4CEAEF9F700FCDB
:1014A000CAE6816843680268C4F8A810C4F8B0208E
:1014B000C4F8AC30EFE70C2030F002FF2B68064692
:1014C000596921F0FFF86660CDE53B680022586954
:1014D0004EF6C8411346F9F7F9F83E49F9F7B8FE58
:1014E000F9F7DCFD0146054632F01EFD0028A1D1CA
:1014F000A3689B689D629DE70C2030F0E1FE2B689D
:101500000646596922F0C8FB6660ACE5282030F039
:10151000D7FE2B680646596921F046FD6660A2E5B4
:10152000282030F0CDFE2B680646596921F030FAAC
:10153000666098E553F8041C481E002943F8040C23
:101540003FF7E7AE104603A931F002FAE1E653F89F
:10155000042C511E002A43F8041C3FF7E0AE594604
:1015600031F0F6F9DBE653F8042C511E002A43F85B
:10157000041C3FF77DAF594631F0EAF978E753F89C
:10158000042C0DF1180B511E002A43F8041C3FF7E0
:101590001FAD594631F0DCF91AE553F8042C511E01
:1015A000002A43F8041C3FF741AE414631F0D0F920
:1015B0003CE653F8042C511E002A43F8041C3FF764
:1015C0000DAD0DA931F0C4F908E500BF0060EA4691
:1015D000000070420000C07FE4020010308C050063
:1015E00010B502210446F9F757FE2046BDE8104029
:1015F000FFF7BEBC2DE9F84305462A6840682B4B2F
:10160000821A921003FB02F38846002B45D05A0041
:10161000934244D96FF00306304630F051FE6C68B7
:10162000D5F800C00746CCEB040323F00303C3182E
:1016300000F10C091CBF98E8070083E80700A445E7
:101640001FD063463A462AB1196811605968516043
:10165000996891600C33A34202F10C02F3D10CF1B2
:101660000C09C9EB0303124A9B0802FB03F929F09A
:10167000404909F1010909EB490907EB890909F119
:101680000C09BCF1000F02D06046F9F709FB3E449B
:10169000AE6085E88002BDE8F8830C26BCE705490A
:1016A0008A42B7D802EB83039E00B5E7ABAAAAAA89
:1016B000ABAAAA2A555555152DE9F047002303601A
:1016C0004360836005460C20884691F8A49030F072
:1016D000F7FD6E682F680446F31B23F0030310EB3D
:1016E000030A09D03C4A0021E1504846CAF80420C8
:1016F00032F0FCF9CAF80800BE4268D03A462346E8
:101700002BB11168196051685960916899600C3269
:10171000964203F10C03F3D107F10C03F31A2F4A9D
:101720009B0802FB03F323F04043013303EB430325
:1017300004EB830909F10C0917B13846F9F7B0FA3F
:1017400008F1380308F1A40704F10C06BB422C6031
:10175000AE60C5F804903CD01C464B469E4221D05A
:101760001BB194E8070083E807000C336B600C346E
:10177000A742F3D1B34222D023B108F1A80207CA8D
:1017800083E807000C336B60B34212D02BB108F131
:10179000B40898E8070083E807000C336B6028461C
:1017A000BDE8F08728462146FFF724FF6B68AE6846
:1017B000DDE708F1B4012846FFF71CFFEFE72846F4
:1017C00008F1A801FFF716FF6B68AE68DCE7A146D9
:1017D000B0E74B46CEE700BF00001041ABAAAA2AF3
:1017E00070B50C46064609B90AE02C463046E16859
:1017F000FFF7F6FFA5682046F9F752FA002DF4D15D
:1018000070BD00BFD0F808C02DE9F843064600F1CE
:101810000408BCF1000F51D00A7847466446237C87
:10182000934223D2E468002CF9D13C46F368D6F801
:101830001490A34234D0A74208BF4FF0000912D041
:10184000204630F0EBFD41460546204630F057FE7D
:10185000F9F726FA7369BD4203F1FF332C46736131
:10186000EED1C3EB09094846BDE8F88304D9274601
:10187000A468002CD3D1D8E7A068E36838B1057C10
:1018800095422ABF0446C06880680028F7D1002B23
:10189000CCD0187C90428ABF1F46DB689B68F6E775
:1018A000B845C8D161463046FFF79AFF0023C6F815
:1018B0000C80C6F81080B3607361D4E74746B4E784
:1018C0002DE9F84F224D4FEA510AA5FB0A25AD0834
:1018D000EB1C082B38BF0823064643609800894656
:1018E00030F0EEFC736801355B1B4FEA530B00EBE5
:1018F0008B0707EB8505AF428046306038BF3C461A
:1019000007D24FF4FC7030F0DBFC44F8040BA54226
:10191000F7D80F4B7761A3FB0A2A58F82B202A230C
:101920004FEA9A0A03FB1A9902F5FC712B1F3161E9
:10193000F260736255F8043C09EB490903F5FC7049
:1019400003EB8901B260F3613062B161BDE8F88FE9
:10195000310CC3302DE9F0438BB08046F9F796FC8B
:10196000774B002408F1380921466C22C8F8003072
:10197000C8F80840C8F80C40C8F81040C8F81C4027
:10198000C8F82C40484635F092FF0023214688F8DD
:10199000A44088F8C040C8F8A830C8F8AC30C8F8EF
:1019A000B030C8F8B430C8F8B830C8F8BC30C8F89F
:1019B000C430C8F8C830C8F8CC30684600940194E8
:1019C000029403940494059406940794089409944B
:1019D000FFF776FFC8F8D040C8F8D440C8F8D84020
:1019E000C8F8DC40C8F8E040C8F8E440C8F8E8406F
:1019F000C8F8EC40C8F8F040C8F8F440214608F1B7
:101A0000D000FFF75DFF009C7CB3D8F8E05008F1F0
:101A1000D80E02AB0FCBD8F8D870D8F8DC6004959C
:101A2000D8F8E4508EE80F0005950AAD15E90F00CF
:101A3000D8F8E85008F1E80E0695D8F8EC5002976F
:101A40000795D8F8F05003960895D8F8F4508EE82A
:101A50000F000995D8F8D020C8F8D040D8F8D43075
:101A600001998DE80C00C8F8D4106846FFF7BAF960
:101A700098F8353098F83420012103F0F90361F328
:101A8000C40302F0FE02022161F3461342F0060293
:101A900088F8353088F834200021142208F1F80045
:101AA00035F005FF142208F58670002135F0FFFEA1
:101AB000244AD8F81C5000230024C8F83821C8F85C
:101AC000BC30C8F8B830C8F8B430C8F8044045B1E4
:101AD00008F1140001460322A847C8F81C40C8F8C2
:101AE0002040D8F82C304BB108F1240001460322E5
:101AF00098470023C8F82C30C8F8303000234846F7
:101B000008F1A4018360436040F80C3B88424FF029
:101B10000002F7D198F83430002103F0E7036FF3A7
:101B200045134046C8F8B020C8F8AC20C8F8A82033
:101B300088F8343088F855110BB0BDE8F08300BF49
:101B4000F8370500000070422DE9F84390E80C00DA
:101B5000456A0446A81AA3EBA00001280E4615D931
:101B60004FF4FC7030F0ACFB6860A3691BB196E8E1
:101B7000070083E80700636A1A1D62625B6803F569
:101B8000FC72E361A3612262BDE8F8836169C1EB85
:101B900005084FEAA80808F1010808F10107B3EBAE
:101BA000470F31D8002B3FD05B009D1CB5F1804F13
:101BB00045D2A80030F084FB636A61690433EF1BEF
:101BC0005B1A7F089A10814600EB870703D09200CA
:101BD000384635F051FE2068F9F762F8C4F80090F5
:101BE000656067613A6808F18043013B07EB830554
:101BF00002F5FC71E2606562216157F8233003F55C
:101C0000FC72E3612262ABE7DF1B7F0802EB870710
:101C10000435B942C1EB050508D9AA10E1D09200FC
:101C2000384635F029FEDCE70325C2E7AD10D8D0F1
:101C3000AA0007EB8800801A35F01EFED1E731F0CC
:101C4000A5F900BFF0B50346D0F8F01090F83420A5
:101C5000D3F8E84090F8A460D0F820510C39D0F8BF
:101C6000240185B0C2F3400CC2F380078C42C2F35A
:101C700000028DF807C08DF806708DF805208DF8EC
:101C80000460029503900CD034B104AD15E907004F
:101C900084E80700D3F8E8400C34C3F8E84005B006
:101CA000F0BD03F1D00001A9FFF74EFFF7E700BF39
:101CB0002DE9F04F0D46097AA3B0C1F38006044622
:101CC000002E00F0D0806B685C2B00F2BD80DFE856
:101CD00013F046013A01520150016E01BB00BB00F6
:101CE000BB00BB00BB005D00BB00BB00BB00BB007A
:101CF000BB00BB0061015401A7012002A001BB0091
:101D0000BB00BB00BB00BB00BB00BB00BB00BB00FB
:101D1000BB00BB00BB00BB00BB00BB00BB00BB00EB
:101D2000BB00BB00BB00BB00BB00BB00BB00BB00DB
:101D3000BB00BB00BB00BB00BB00BB00BB000B0279
:101D40000B020B020B020B020B02BB00BB00BB0021
:101D5000BB00BB00BB00BB00BB00BB00BB00BB00AB
:101D6000BB00BB00BB00BB00BB00BB00BB00BB009B
:101D7000BB00BB00BB00BB00BB00BB00BB00BB008B
:101D8000BB00BB00BB004901B401BD0128464C218A
:101D900017F0A8F9002857D028464C21002217F048
:101DA000D7F9022806D028464C21002217F0D0F996
:101DB000142849D12846502117F094F9002843D01F
:101DC00028465021002217F0E7F9002840F0C88586
:101DD00094F8A430082B37D803EB43034FEA830A67
:101DE00004F1380B0BEB0A0728464C210022D7F8E8
:101DF0000890D7F804805BF80A6017F0A9F9142856
:101E000000F01E8794F834202846C2F3400258217F
:101E1000002A00F0D58617F065F9002840F04A87BF
:101E20002846592117F05EF9002840F08E87284691
:101E30005A2117F057F9002840F07687C7F8089024
:101E4000C7F804804BF80A6094F835306FF300034C
:101E500084F8353094F834306FF3C30384F83430A9
:101E600023B0BDE8F08F8F07EED52B68782B00F0FC
:101E7000BD841DD8522B00F0B1844DD8112B00F039
:101E80008B8140F21C82122B00F039821E2BDBD199
:101E9000C54B1B6893F8A8305E07D5D594F834205D
:101EA000002342F0020284F8342084F8A430CBE707
:101EB000DC2B00F06D8200F28581CB2B00F03C81A1
:101EC00040F20182CC2B00F00482CD2BBCD12846FD
:101ED000582117F007F9002840F0B78528465A2105
:101EE00017F000F9002840F070852846532117F0BC
:101EF000F9F80028A8D028465321002217F006F947
:101F00000021054631F0E8FF002840F08786A64B07
:101F10001B681B695D6197E7542B00F00181C0F0DD
:101F200094825C2B00F05282722B8DD112AA490947
:101F30004023FDF707FE021E92DD05F1100012A9F5
:101F400030F0A0FE8CE7022294F83530294666F383
:101F5000000384F835302046FEF790FD7AE700262E
:101F60000122F1E790F8343043F0060380F8343072
:101F70006AE70422E8E70322E6E790F83530022218
:101F800003F0F90362F3C403012262F3461380F8FD
:101F9000353059E790F83530012203F0F90362F348
:101FA000C403022262F3461380F835304CE728461A
:101FB000502117F097F8002840F02D840646284657
:101FC000532117F08FF8002840F0F280002E3FF4E4
:101FD0003BAF754D01212B68986901F003F92EF094
:101FE000A9F84FF47A73074603FB06F608E0286861
:101FF000F7F7A2FB2B6893F8A83098073FF530AFAE
:102000002EF098F8C01BB0424FF003012246EED3E9
:102010001AE790F834306FF3000380F8343013E798
:1020200090F83530012262F34203022262F3C403C6
:102030006FF3461380F8353006E790F8343003F03C
:10204000FD036FF3820380F83430FDE64909CB1DB0
:1020500003F00703012B07D9284617F0C1F8002821
:1020600040F0E183297A49090023C4F8B030C4F86C
:10207000AC30C4F8A83000297FF4F2AE28464521E0
:1020800017F030F8002800F0528594F85571032FAE
:102090007FF7E6AEA068C36893F839305B0700F1BC
:1020A0001A861023032600E00B460136B74203F1DF
:1020B00004017FF7D5AEC25892F839205207F3D504
:1020C0001F462846452117F00DF8002840F0CF8420
:1020D000002104EB8606C6F80C11C6F8F810A368B8
:1020E000D859F6F7C3FEBBE6363BDBB280F8A43026
:1020F0006A683B2A7FF4A8AE2A7A52093FF4A4AE5C
:102100001344DBB2082B7FF6D0AE082380F8A4304E
:102110009AE690F8343043F0010380F8343093E6C7
:10212000214D01212B68986901F05CF8286808218D
:102130000022F7F701FB87E6284617F051F8002840
:1021400040F0D68307465826A146A846D8F80C404A
:1021500098F80820236852099D6818BFD9F80830FC
:1021600009EB070116BFDB59D1F84801586A31F075
:1021700081F83246CDE90001013620460B49A847D7
:102180005B2E07F10407E1D198F808304C4643F084
:10219000010388F8083057E6034B0821186801222C
:1021A000F7F7CAFA50E600BFE4020010E83905006C
:1021B00028465321002216F0CBFF4FF47A7303FB1D
:1021C000006603E7B3F5FA7F00F054816CD940F262
:1021D000F712934200F04E8140F2992293427FF42D
:1021E00033AE12AA104629460B9222AE17F0F6F82B
:1021F000532306F84C3D31460B98FFF703FB55235C
:1022000031460B988DF83C30FFF7FCFA179B002BFA
:1022100040F0ED830B981499FFF7E2FA0DF14C08AA
:1022200000226068CDF85480CDF85880149203687D
:102230000B9917925B699847C0B1159E464515D01A
:10224000706931F017F8EB68327C1F68CDE9000146
:10225000BF6818468049B8472B7A304643F00103DF
:102260002B7230F0C8F840450646E9D12846532184
:1022700016F038FF0646002800F01E83002228468C
:10228000532116F043FFED68C4F8340130F0F2FF3B
:102290002E6802460B46B66828467049B0470B9830
:1022A0001499FFF79DFACFE5B3F5C87F7FF4CCAD65
:1022B0006B4B01211B68986900F094FFC4E5022B69
:1022C0003FF4ECADC0E5792B7FF4BEADFDF7A4FB88
:1022D000BAE52846532116F005FF002840F0658333
:1022E000002606F15807FFB23946284616F0FAFED6
:1022F000002840F07F820136032EF2D1A4E5284663
:1023000016F06EFF00287FF70BAF94F85571B7B148
:10231000002637464FF00208022ED4BF06F15801BE
:1023200006F13E01C9B2284616F0DCFE10B108FAEB
:1023300006F31F4394F855310136B342ECDC2846CE
:10234000452116F0CFFEB8B194F85501032813DDEE
:10235000A268D36893F839305D0700F1F0830C323E
:10236000032306E052F8041F91F83910490700F1E1
:10237000E78301338342F5DB394D01212B689869EE
:1023800000F030FF28683A460821F7F7D5F95BE5F9
:102390002846532116F0A6FE002800F07C8228462D
:1023A0005321324616F0B2FE2E49054631F094FD17
:1023B000002840F0B18328462B4931F0ABFD0028BE
:1023C00000F009852948C4F838013DE52846582120
:1023D00016F088FE002840F024832846592116F084
:1023E00081FE002840F0098328465A2116F07AFE23
:1023F000002840F0A182D4F80880D5F80C90D8F8D5
:102400000030D9F800A0186A30F034FFD8F8043052
:102410000646186A0F4630F02DFFCDE90001D8F8C6
:102420000830186A30F026FFCDE9020132463B46FB
:10243000DAF8086048460E49B0472B7A204643F048
:1024400001032B72FDF7ACFC0AE590F8343066F31B
:10245000820380F83430F7E47C3B0500883B0500BC
:10246000E40200100000204100007A440000C04057
:10247000D8390500D4F80890D5F80CA0D9F8003068
:10248000DAF800B0186A30F0F5FED9F804300646E4
:10249000186A0F4630F0EEFECDE90001D9F8083099
:1024A0004FF00008186A30F0E5FECDE9020132462F
:1024B0003B46DBF808609F495046B047D4F83C01E2
:1024C00030F0D8FEEE68024637680B46BF683046EB
:1024D0009949B847A36808F1580753F8283008F11C
:1024E00001089E6A3046314631F01EFD58B930462B
:1024F00030F0C0FEEB683A461E68CDE90001184690
:102500008E49B3689847B8F1030FE3D1E8688C4966
:1025100003689B6898478B4BD5F80C901A68D9F8DC
:102520000030D2F81080D3F808A0D8F80C0030F0B2
:10253000A1FED8F810B006460F465846594631F06D
:10254000F3FC002840F03983584630F093FECDE983
:102550000001D8F8140030F08DFE32463B46CDE93C
:10256000020148467849D047D4F8480130F082FE4D
:102570000646D4F84C010F4630F07CFED5F80C909E
:102580000DF14C08D9F800A0CDE90001D4F85001B4
:1025900030F070FECDE9020132463B46DAF80860C1
:1025A00048466A49B047D4F80890D5F80CB0D9F835
:1025B0000030DBF800A0586A30F05CFED9F8043037
:1025C00012AA0646586A0B920F4630F053FECDE928
:1025D0000001D9F80830586A30F04CFECDE902010C
:1025E00032463B465A49DAF808605846B04700225E
:1025F00060681492CDF85480CDF8588003680B9928
:102600008DF84C2017925B69984700B3179BF3B184
:10261000E868504903689B689847159E464511D065
:10262000706930F027FEEB68327C1F68CDE900014D
:10263000BF6818464849B84730462FF0DCFE404591
:102640000646EDD1E8683E4903689B689847E8680C
:10265000424903689B689847EE680FA8336894F86E
:10266000A4109F68F7F718FD0F9A30463C49B84709
:102670000F9B3C4AA3F10C00904240F0BE8304F152
:10268000A40304F138069E420A9371D004F1440871
:1026900001270D940C9536E075680021284631F02D
:1026A00011FC00283BD158F80CBCAA460C9B0FA883
:1026B000DD68791E2B68D3F80890F7F7EDFC20460B
:1026C00030F0D8FDCDE90001504630F0D3FDCDE922
:1026D0000201584630F0CEFD0F9ACDE90401069272
:1026E00028463A462049C8470F9B1E4AA3F10C00D2
:1026F000904240F076830A9B0C36B34207F1010703
:1027000008F10C0832D0B4680021204631F0DAFB21
:102710000028C1D1D6F804A058F80CBCC6E758F878
:102720000CBC0021584631F0CDFB0028E3D1AA466D
:10273000BCE700BF103A05003C3A0500643A0500CA
:10274000907F0500E4020010703A0500E03A0500B1
:10275000203B0500083C0500603B05006C3B050084
:10276000D08A0500640A0010383C05000D9C0C9DC1
:1027700094F83430DB093FF492ADD4F8B060002116
:10278000304631F09FFBD4F8AC8060B10021404668
:1027900031F098FB38B1D4F8A800002131F092FB59
:1027A00000287FF47CAD304630F064FD064640469C
:1027B0000F4630F05FFDED68D5F80080CDE90001EF
:1027C000D4F8A80030F056FDCDE9020132463B4670
:1027D000D8F808602846B449B04760E590F834302E
:1027E00043F0040380F83430FFF72EBBFFF72AFADA
:1027F000FFF72ABB39462846002216F087FC002145
:10280000074631F073FB002840F08881A36853F835
:1028100026309F626FE528465021002216F098FC72
:102820000646FFF7CCBB2B7A5B09032B00F09B809D
:10283000D4F80071D4F8FC60D4F8F8300FA8214621
:1028400012AA129713961493D4F8B080D4F8AC70EF
:10285000D4F8A860FDF736F92846582116F042FC56
:10286000002840F00C812846592116F03BFC002836
:1028700040F03D8128465A2116F034FC002840F0F3
:102880002181297AC4F8B080C4F8AC70C4F8A8607B
:102890004909FFF7F0BBD4F83811844831F032FA17
:1028A00030F0E8FCED6802462E680B46B668284614
:1028B0007F49B047FFF7C8BA2846552116F012FCE9
:1028C00000283FF4ECAC32462846552116F01EFC99
:1028D0000023ED68C4F83431C4F8280130F0CAFC94
:1028E0002E6802460B46B66828467249B047D6E4C1
:1028F00058272846394616F0F5FB80B904360137CB
:102900000C2EFFB2F5D12B7A5B0900F01E81012B52
:102910007FF49AAA2046FDF743FAFFF795BA002202
:102920002846394616F0F2FB2B7AA2195B0940F0D3
:10293000F780C2F84801E1E7A3685A21002228463F
:102940009E6816F0E3FB94F834300146DA0703D5AD
:10295000594931F023F901463046F6F77BFA4AE54A
:10296000431EFFF737BA2846582116F0BBFB002854
:1029700040F0168100272846592116F0B3FB0028A5
:1029800040F00781002628465A2116F0ABFB0028AC
:1029900040F00D810020297AC4F8B070C4F8AC6012
:1029A000C4F8A8004909FFF766BB53212846002256
:1029B00016F0ACFB4FF07E51064631F08DFA002840
:1029C00040F02781C4F83C618AE45A21284600225D
:1029D00016F09CFB3949064631F088FA002840F091
:1029E0001B81374B1B681B691E61FFF77EBA60684D
:1029F0000B9903681B6998470CE4A3685921284682
:102A000000225E6816F082FB94F834300146DF073E
:102A100003D5294931F0C2F801463046F6F71AFAD3
:102A2000E2E4A3685821284600221E6816F06EFBD7
:102A300094F834300146DB0703D51F4931F0AEF876
:102A400001463046F6F706FAC7E458212846002228
:102A500016F05CFB0021064631F03EFA002840F0FB
:102A6000E080174B1B681B69DE60FFF737BA452112
:102A70002846002216F04AFB0146FFF72ABB5821E0
:102A80002846002216F042FB94F83430D90702D5CC
:102A9000094931F083F8119930F076FF014640463C
:102AA00030F074FF8046DEE6583C05000080BB45F0
:102AB000F4390500B03B05003333CB41000080BF43
:102AC000E40200105A212846002216F01FFB94F859
:102AD0003430D90702D5B04931F060F80F9930F0A1
:102AE00053FF0146304630F051FF0646C9E62846FE
:102AF0005921002216F00AFB94F83430DB0702D586
:102B0000A54931F04BF8109930F03EFF01463846A8
:102B100030F03CFF0746ADE6A04854E4A04F75E610
:102B2000012B7FF4EBAEA3689B595862E6E628467A
:102B300016F056FB00283FF4A8AAFFF791B903232B
:102B4000022202FA03F31F4316E42846412116F03D
:102B5000C9FA002867D0E8689249036800269B6894
:102B6000984706F14107FFB23946284616F0BAFAEF
:102B700028B90136032EF4D12B7A5B09C7E6394612
:102B80002846002216F0C2FAA36853F8263058628D
:102B9000EFE728465921002216F0B8FA0646F2E679
:102BA00028465821002216F0B1FA0746E3E62846E7
:102BB0005A21002216F0AAFAEDE600207A49C6E46E
:102BC000099216F08FFA099A002840F09B80284657
:102BD000592116F087FA002840F0818028465A21B2
:102BE00016F080FA00283FF429A928465A2100222D
:102BF00016F08CFA94F834300146DD0703D56649A7
:102C000030F0CCFF0146304630F0C0FE0646FFF7FC
:102C100015B94FF07E56D5E6614EE2E60025FFF786
:102C200076B900261DE72846422116F05BFA0028F7
:102C300091D12846432116F055FA00288BD19BE705
:102C4000D4F800C1D4F8FCE0D4F8F8300FA821463D
:102C500012AACDF848C0CDF84CE01493FCF732FF2F
:102C60002846582116F03EFA002840F09F8028465A
:102C7000592116F037FA002878D128465A2116F043
:102C800031FA00283FF4DAA85A210022284616F02B
:102C90003DFA94F83420D10702D53F4930F07EFF49
:102CA0000F9930F071FE0146304630F06DFE064659
:102CB000FFF7C4B800222846582116F027FA94F8E6
:102CC00034308146DA077FF5ABA8334930F066FF30
:102CD0008146FFF7A5B80C270326FFF7F2B9592163
:102CE0002846002216F012FA94F834300146DB0729
:102CF00003D5294930F052FF0146404630F046FEE8
:102D000080466BE75821284616F000FA94F83430D4
:102D10000146DA0703D5204930F040FF0146484616
:102D200030F034FE814652E75A212846002216F040
:102D3000EDF994F834300646D9077FF57FA8164997
:102D400030F02CFF0646FFF779B8284659210022BB
:102D500016F0DCF994F834308046DB077FF567A87D
:102D60000D4930F01BFF8046FFF761B8002228466E
:102D7000592116F0CBF994F83420D20702D5064930
:102D800030F00CFF109930F0FFFD0146404630F066
:102D9000FBFD804671E700BF3333CB410000164492
:102DA0000000C07FD43B05000000F0BF5821002286
:102DB000284616F0ABF994F83420D10702D515490E
:102DC00030F0ECFE119930F0DFFD0146484630F05E
:102DD000DBFD81464BE729460F4830F093FFFFF7B4
:102DE000F2BA53F8042C511E002A43F8041C3FF792
:102DF00082AC0EA92FF0ACFD7DE453F8042C511EDB
:102E0000002A43F8041C3FF73AAC0EA92FF0A0FDAE
:102E100035E400BF3333CB410080BB4538B50321D7
:102E20000446144DF8F738FA20460721F8F734FA2B
:102E30002B68002258694EF295211346F7F746FC9D
:102E40002021F8F7F9F9F8F729F931F0A9F82968FC
:102E500000221346E061486944F2E761F7F736FC67
:102E60006421F8F7E9F9F8F719F931F099F8A06158
:102E700038BD00BFE402001042688068131A58424F
:102E80005841704708B50430FFF7F6FFC8B10D4B45
:102E90001B68DA689368D1688B420FD01A6892F881
:102EA0003900C0F3400058B9043305E053F8042B4F
:102EB00092F83920920704D49942F7D1012008BD35
:102EC000002008BDE4020010002282604260816898
:102ED00002600261C160704710B50446F8F7D6F988
:102EE000104B204640F8043BFFF7EEFF94F82430E7
:102EF00000226FF3000384F8243094F82430226217
:102F00006FF3410384F8243094F8243020466FF3A3
:102F1000820384F8243094F824306FF3C30384F8D8
:102F2000243010BD783C050038B500238360436031
:102F30008168026905460360C1609AB152F8043C99
:102F4000642404FB032407E054F8103C184613B132
:102F5000F7F7A6FE2A69643CA242F5D1A2F1080067
:102F60002FF0D8F900232B61284638BD10B5054B4A
:102F7000044640F8043BFFF7D7FF2046F8F776F900
:102F8000204610BD783C050010B5074B044640F8BC
:102F9000043BFFF7C9FF2046F8F768F92046F7F72A
:102FA0007FFE204610BD00BF783C05002DE9F843A8
:102FB00088460646FFF760FF00284AD0B8F1000FA8
:102FC0004AD0B8F1A27F9BBF642000FB08F04FF00D
:102FD000FF3008302FF072F9642380E8080100F117
:102FE000080781463D4608F1FF342846013C00F0C1
:102FF0006DFD631C05F16405F7D157B3356972B6F1
:103000003046FFF739FF00284CD00023B36037610A
:10301000C6F80080736062B6002D5DD055F8043CA0
:10302000642606FB0356B5420BD03446A6F11007C2
:10303000A31BFB5818460BB1F7F732FE643CA542C0
:10304000F6D1A5F108002FF065F90120BDE8F8835D
:1030500062B60020BDE8F88372B63046FFF70CFF79
:103060000028F5D00023B3603360736062B6326924
:103070009AB152F8043C642404FB032407E054F89A
:10308000103C184613B1F7F70BFE3269643CA242BC
:10309000F5D1A2F108002FF03DF9002333610120A2
:1030A000BDE8F88362B6D9F80430642505FB0375E2
:1030B000AF420BD02C46A5F11006631BF3581846FF
:1030C0000BB1F7F7EDFD643CA742F6D148462FF06F
:1030D00021F90020BDE8F8830120BDE8F88300BF96
:1030E000074B10B5044619700430E169FFF75EFF25
:1030F00094F8243043F0010384F8243010BD00BF5D
:103100003C05001082680369642000FB02307047B0
:1031100042680369642000FB02307047006820B1F8
:10312000013188428CBF08460020704710B5016904
:1031300004460430FFF7F2FF206110BD10B541686E
:103140000446FFF7EBFFA368C31A5842584110BD6D
:10315000F8B5224D04462B680F46DA0715D5204EE8
:10316000251D2846FFF788FE68BBDFB12CF0E2FF83
:1031700094F8243030601B0706D494F8243043F0D0
:10318000040384F82430F8BDF8BD28462FF0ACF8CD
:103190000028E4D02CF0CEFF114E306028462FF0EE
:1031A000B1F8DDE72846FFF7C9FF0028DED12CF093
:1031B000C1FFA3694FF47A7202FB03F23368C01AAD
:1031C0009042D3D2F8BD94F824306FF3820384F890
:1031D00024302CF0AFFF3060F8BD00BF3405001084
:1031E00038050010F8B590F8243004466FF300035A
:1031F0000F4680F82430051D114E07E02046FFF7EA
:10320000A7FF306803212246F6F796FA2846FFF713
:1032100033FE01210028F1D05FB1094D02E028689A
:10322000F6F78AFA2046FFF72DFE032122460028F2
:10323000F5D094F8243043F0010384F82430F8BD2D
:10324000E402001090F8243010B56FF3820380F888
:10325000243090F82430044643F0080380F82430EA
:103260000021FFF7BFFF94F824306FF3C30384F805
:10327000243010BD38B504460D4690F8243021B1F5
:103280006FF3410380F8243038BD43F0020380F827
:10329000243090F8243061F3820380F8243090F8D1
:1032A000243043F0080380F82430FFF79BFF94F8A4
:1032B000243065F3C30384F8243038BD10B50446C8
:1032C000FFF7DAFD20B9A1682046FFF727FFA060CD
:1032D00010BD00BF10B590F824300446DB0713D4AE
:1032E000E26823699A420ED004342046FFF7C4FDF9
:1032F00008B100BE10BD2046FFF704FF00F068FBD8
:103300002046FFF7DBFF10BD0021FFF721FFE7E7B5
:1033100010B504462046FFF711FF0028FAD1616876
:103320002046FFF7FBFE606010BD00BF70B5051DB5
:1033300004462846134EFFF701FF68B194F8243085
:103340009A0709D4306803212246F6F7F5F9284692
:10335000FFF7F4FE0028F1D194F824309B070AD43B
:103360002846FFF7D5FFBDE87040064B08211868D6
:103370000122F6F7E1B92846FFF7CAFEBDE8704022
:1033800000F026BBE40200100369642000FB01305A
:10339000704700BF90F8243070B5044618070E46F9
:1033A0000DD52269A3689A4209D0251D21692846B6
:1033B000FFF7B4FE20612269A3689A42F6D194F81F
:1033C000243000229907226208D42269A3689A4215
:1033D00004D094F82450C5F3800515B9002528467B
:1033E00070BD2169201DFFF7CFFF90F860305A06AD
:1033F000F4D490F860305B0700D400BE90F86030E1
:10340000C26943F0200380F8603090F860306FF3B9
:10341000000380F8603022623060284670BD00BF33
:10342000006808B109B1481E70470138704700BFF5
:10343000F8B5066C456A04460F462846314630F01A
:1034400041FD50B994F860309B0704D430463946AA
:1034500030F060FD18B9666235462846F8BDE36A6B
:103460003946384603F1004630F098FB31460546B0
:10347000304630F08BFA216A30F090FB0146284646
:1034800030F082FA31F0E8FD256C0646294630F02E
:1034900041FD00B935466562DFE700BF70B590F8C1
:1034A000603004469A0625D490F860309B0702D518
:1034B000C469204670BD406AE36A014603F10046D4
:1034C00030F06CFB31460546304630F05FFA216A39
:1034D00030F064FB0146284630F056FA31F0BCFD6E
:1034E000E4690546214630F015FD0028E1D12C465F
:1034F000204670BD846A204670BD00BF70B5C669A5
:10350000044630460D4630F0E7FC00B92E46256CE7
:103510003046294630F0FEFC00B935462846616A3F
:1035200030F0E4FC30B194F8603065626FF3000372
:1035300084F860302046BDE87040FFF7AFBF00BFA1
:103540002DE9F04F054683B0406930F0CFFA0146CF
:103550004FF07E5030F0D6FB3D4B01901B78002B96
:1035600072D03C4A03F1FF385FFA88F8D2F800A025
:103570006C6D05EB8808A5F10409002732E0E361D2
:10358000A86BEB6B3146009330F008FB4FF09D4188
:1035900030F004FB31F008FB30F0DCFC009BA06055
:1035A0001946304630F0FAFA4FF09D4130F0F6FA05
:1035B00031F0FAFA30F0CEFC4042696BE060304600
:1035C00030F0ECFA594630F09DFB4FF09D4130F061
:1035D000E5FA31F0E9FA30F0BDFC2061C14504F1B3
:1035E000200431D059F8043F18466361002BF5D010
:1035F00030F07CFA019930F0D1FADAF82C30296BEE
:10360000D3F810B0064630F0C9FA594630F07AFBCC
:103610004FF09D4130F0C2FA31F0C6FA30F09AFC1A
:10362000E96C6B6C4A1C84E88100A761E261002BA5
:10363000A5D1A86CEB6B10B903F10040A2E7814261
:1036400018BFE06100209DE703B0BDE8F08F00BF28
:103650003C050010E40200102DE9F04F90F86040A6
:1036600087B0A3068346174602D507B0BDE8F08FA2
:10367000C5690846294630F045FBDBF8184001468D
:10368000204630F08BFA29460646384630F03AFBA1
:103690000146204630F082FA8046DBF8140030F014
:1036A00025FADBF82C10044630F078FADBF820100D
:1036B00030F028FB41468146404630F06FFA3146F3
:1036C0008246304630F06AFA49460546204630F0D8
:1036D00065FA29460446504630F058F94FF07C51BF
:1036E00030F05CFA0146204630F050F931F0B4FC7D
:1036F000DBF818500446294630F00CFC002840F056
:103700009E803146CBF83440204630F03DF94946A2
:10371000059030F0F7FA21468246404630F034F901
:1037200009F1004130F0EEFA29468146204630F09A
:10373000F1FB002840F0C580002225466249504632
:103740000968C96A0C690192214630F027FA31F004
:1037500099F930F025FC21460290484630F01EFAD7
:1037600031F090F930F01CFC49460390504630F09F
:103770000DF9019A114630F009F9214630F00EFAA0
:1037800031F080F930F00CFC0490029830F0AEF982
:10379000214630F0B7FA8146039830F0A7F9214668
:1037A00030F0B0FA00218246484630F0B3FB0028E2
:1037B00000F082804946059830F0A4FA81465046D0
:1037C000002130F0A7FB002879D02846414630F090
:1037D000DBF8514630F096FA0546049B03989BF8B7
:1037E0006020191A029B42F040028BF86020CBF84F
:1037F0004430CBF848102046214630F0CFF904463B
:103800002146484630F07EFA2146CBF8380028465B
:1038100030F078FA049BCBF83C00CBF84C30CBF876
:103820003060CBF828705846FFF78AFE9BF860207E
:1038300022F040028BF8602007B0BDE8F08F3146DF
:10384000CBF83450284630F09FF84946059030F0C8
:1038500059FA29468246404630F096F809F100416F
:1038600030F050FA8146DBF8140030F03FF9294679
:103870000446304630F08AF84FF07C5130F08EF933
:10388000514630F08BF90146204630F07DF829464C
:103890000446404630F07AF84FF07C5130F07EF923
:1038A000494630F07BF90146204630F06DF8294654
:1038B00030F028FA024641E74FF000097FE7002583
:1038C0008BE72546CFE700BFE402001008B5436D43
:1038D0004901585830F00EF94FF0425130F05EF97E
:1038E000034B1B68DB6A196930F058F908BD00BF4B
:1038F000E40200102DE9F8430D460646002955D094
:1039000047688368DB1BB1EB631F13D80C463B464B
:103910000022013C1A605A609A60DA601A615A61AA
:103920009A61DA6103F12003F3D107EB4515756065
:10393000BDE8F88301686FF078437F1A7F11DB1BC5
:103940009D423DD8AF422CBFFB197B199F422FD916
:103950006FF01F0840462EF0B3FC96E80A005B1A91
:103960005B1181461F467F0123B13A46484633F03A
:1039700083FF31684F443B462C460022013C1A60CD
:103980005A609A60DA601A615A619A61DA6103F1E9
:103990002003F3D107EB451511B10846F7F780F97D
:1039A00009EB0803B360C6F800907560BDE8F883C2
:1039B000B3F1006FCCD233B9984699463B46D2E773
:1039C00002482FF0E9FA4FEA4318C3E7983D050093
:1039D00090F86020F8B56FF382020446034680F841
:1039E00060200021143043F8041B83424FF0000292
:1039F000F9D194F86010B4F8623001F0FE0162F37E
:103A0000410184F8601094F8601062F30B0321F018
:103A1000200184F8601094F860102A4D62F30411BC
:103A200084F86010A06D616DA4F8623094F860C0F5
:103A30002D78461A244F761100232CF0400CB54205
:103A400062616264A2642265E26484F860C0A3617A
:103A5000E36123626362A36223632364A363E3637A
:103A6000E76206D025D804D201EB4510A0650A46CE
:103A700000E00A4682421BD002F12003C01A02F184
:103A8000400120F01F000144002243F8202C43F89D
:103A90001C2C43F8182C43F8142C43F8102C43F832
:103AA0000C2C43F8082C43F8042C20338B42ECD127
:103AB000F8BD04F15400A91BFFF71CFF626DA06D57
:103AC000D8E700BF3C0500100000C84210B5002335
:103AD000002204468263C263036543658365C36550
:103AE000FFF776FF204610BD10B50A4B044600696B
:103AF000236010B103685B689847606A08B1F7F704
:103B0000CFF8054B002220461A60F7F7AFFB20469E
:103B100010BD00BFC03D05004005001010B50446B3
:103B2000FFF7E2FF2046F7F7BBF8204610BD00BFC5
:103B30002DE9F0438A8842F60D039A42B9B00C464B
:103B4000054602D039B0BDE8F083CB8843F61B327E
:103B5000934265D048F293629342F3D190F83230A9
:103B600095F8341095F8352090F833008DE807006B
:103B7000C8212F4A06A834F065F995F83BC095F89E
:103B80003CE095F83D200646C0F1C80706A895F828
:103B90003A3039468DE8005030440292254A34F0DC
:103BA00051F995F837C095F838E095F839203F1A63
:103BB000064406A895F8363039468DE80050029242
:103BC00030441D4A34F03EF995F82FC095F830E0A6
:103BD00095F8312095F82D9095F82E8095F82C3099
:103BE000391A351806A8CDF808C0CDF80CE02844DD
:103BF0000492CDF80090114ACDF8048034F022F9F7
:103C00000544681C29F0CEFA06A92A4633F02BFE9B
:103C1000227C002142F00302E0604155227491E7CA
:103C20000B7C00F1320543F00303CD600B7489E790
:103C3000F03D0500083E05001C3E0500343E050031
:103C400010B50446F0F76CFAA36A00200133A362B2
:103C500010BD00BF10B50446E06800F087FE0028E4
:103C6000FAD110BD2DE9F04F171E85B0064601911F
:103C70009B469DF8388030DD0024254607F1FF394A
:103C80001CE03268431B52F80C2C954255D82A464A
:103C900003A831462FF0B2F8039B294AA3F10C0088
:103CA00090423DD10AF10105184600215A4635F0EF
:103CB00045F9019B18550134BC420ED0A14510DDD9
:103CC000304641462A462EF084FDB0F1FF3F824641
:103CD000D7D1002005B0BDE8F08F012005B0BDE8C8
:103CE000F08F336853F80C3C9D4226D82A464FF09B
:103CF000FF3303A831462FF081F8039B104AA3F14C
:103D00000C009042D0D053F8042C511E002A43F8E6
:103D1000041CC9DC02A900932EF01AFE009BC3E725
:103D200053F8042C511E002A43F8041CBADC02A9E3
:103D300000932EF00DFE009BB4E702482FF02FF900
:103D4000640A0010682705000146014833F062BE8E
:103D5000603E050038B50446F7F798FA0B4A0C4B5D
:103D600022601C201C602EF0ABFA054601F056F8CC
:103D7000227A002363F3820225612272A3626360C8
:103D8000636200F0AFFDE060204638BDC03D050035
:103D90004005001010B5037A0446DA070CD49B07DF
:103DA00004D520F001FC084833F0E8FEBDE81040DF
:103DB0004FF4E640F1F774B8F2F7CCFF034833F064
:103DC000DDFE237AEBE700BF903E0500783E05005C
:103DD0002DE9F04184B00391014603980292C1F8A5
:103DE000320002980193C1F8360001980E4AC1F8DA
:103DF0003A000E4BB1F832800D4CB1F834C0B1F836
:103E000036E00F8F4E8F8D8F0846A4F80080A4F8FF
:103E100002C0A2F800E057801E805D80FFF7BAFF65
:103E200004B0BDE8F08100BF800A0010900A0010C5
:103E3000880A001010B50446408D218D03020A0245
:103E40009BB243EA102392B282B0D8B242EA112266
:103E50000090110A1B0AD2B2234833F0DBFDE08D3B
:103E6000A18D03020A029BB243EA102392B2D8B298
:103E700042EA11220090110A1B0AD2B21B4833F009
:103E8000C9FD608E218E03020A029BB243EA102311
:103E900092B2D8B242EA11220090110A1B0AD2B2A1
:103EA000134833F0B7FDE08EA18E03020A029BB2E5
:103EB00043EA102392B2D8B242EA112200901B0AC0
:103EC000110A0C48D2B233F0A5FD616A0A4809BA5A
:103ED00033F0A0FD0948A16AE26A636B006802B092
:103EE000BDE81040FFF774BFA43E0500C03E0500CA
:103EF000DC3E0500F83E0500183F050040050010B7
:103F0000F0B53221044683B01430F1F75BFF04F1C1
:103F10001C004FF47A71F1F755FFF0F72FFF344B87
:103F200094F82F0094F8301094F83120D87019715B
:103F30005A7194F82C5094F82D0094F82E10227A8F
:103F40001D705870997013070DD504F12C00626A2A
:103F50000621F0F72BFAF0F757FB264803B0BDE82F
:103F6000F04033F00BBE94F8321094F8332094F8FC
:103F7000343094F8350042EA012740EA03261E4D0A
:103F80007FBA76BA00902F806E801C4833F042FDD5
:103F900094F83A1094F83B2094F83C3094F83D00A3
:103FA00042EA012740EA0326154D7FBA76BA00900F
:103FB0002F806E80134833F02DFD94F8390094F86B
:103FC000361094F8372094F8383042EA012740EA56
:103FD00003260D4D7FBA76BA00902F806E800B4875
:103FE00033F018FD204603B0BDE8F040FFF7D2BE25
:103FF0008C020010383F0500880A0010F03D0500D3
:10400000900A0010083E0500800A00101C3E0500C2
:1040100038B51E4B1B689988B1F5A04F18D0B1F583
:10402000E64F0DD0B1F5B85F04D0BDE83840184870
:1040300033F0F0BC174B1B681B7A9B0711D438BDBB
:10404000144C2368586880B1BDE8384020F034BC77
:10405000104B1B681B7ADA07F1D5BDE83840F2F740
:10406000D3B8BDE8384020F003BA8C202EF028F9F0
:10407000054620F0B9FA236828465D6020F06CFC04
:10408000054833F07BFD23685868DDE77C0A0010A3
:10409000683F050040050010503F050070B506461A
:1040A00000690D46036814465B6C98472946224612
:1040B00033F0D9FB30692946036822461B6C9847C8
:1040C00070BD00BF034A044B106804491A88FFF70B
:1040D000E5BF00BF400500109E0A001098000820B0
:1040E00030B5184C83B023887BB1174DAB89082BB2
:1040F0001AD0B3F5C16F0AD0190289B241EA13216F
:10410000124833F087FC0023238003B030BD0190B8
:10411000F0F742FB22880198002AF6D0294603B026
:10412000BDE83040FFF7BABF0120F0F7E7FE238873
:10413000002BEAD0F0F79CFB03B0BDE83040F1F76C
:10414000CDBD00BF9E0A001098000820843F0500E6
:104150002DE9F0430446006983B0837E13B903B0B0
:10416000BDE8F0834FF4CA7302AA42F8043D2C491B
:1041700001F05AF888B904F114052846F1F730FE29
:10418000A0B91C342046F1F72BFE0028E7D02046CA
:10419000F1F720FEF0F7CEFAE1E7224A019B204634
:1041A0001380FFF79DFF03B0BDE8F08328461D4E46
:1041B0001D4DF1F70FFEDFF8788005F1C007B1461D
:1041C00001E0BD4211D00220C8F80050F0F796FE81
:1041D00033882035002BF4D0F0F74AFB20461049F5
:1041E000B9F80020FFF75AFFEBE7104DDFF84480E5
:1041F000DFF8309005F588770520C8F80050F0F713
:104200007DFE3388443513B9BD42F5D1B9E7F0F7E7
:104210002FFB20460249B9F80020FFF73FFFF3E7E4
:10422000980008209E0A001038020820F802082092
:104230007C0A0010A00A0010F8B542680368044622
:10424000D31A9B100F4605D05A00934226D96FF01F
:10425000030600E0042630462EF032F8054694E8C6
:1042600009001B1A9B109A003968AF1807D045F84F
:10427000231094E809001B1A9B109A00AF1823B171
:104280000146284633F0F8FA2068043708B1F6F7FB
:1042900007FD2E44A66084E8A000F8BDB2F1804F6F
:1042A000D5D2DE00D7E700BF2DE9F0430C4D8DB02D
:1042B0002B6842F60D0147F2693204465869002323
:1042C000F6F704FA0021F6F7B7FFF6F79FFF48B9B3
:1042D0001CB1236820465B6898470DB0BDE8F083A9
:1042E000E40200102B6842F6D81242F60D0158691C
:1042F00047F26933F6F7EAF90021F6F79DFFF6F782
:1043000085FF237A2A6860F300032372506947F21D
:1043100069334FF28E1242F60D01F6F7D7F90021FC
:10432000F6F78AFFF6F772FF237A2A6860F34103F3
:104330002372506947F2693341F6E56242F60D0196
:10434000F6F7C4F90021F6F777FFF6F75FFF237A57
:104350002A6860F3820323725069002342F60D013C
:1043600041F2F462F6F7B2F907AE074605AAA4498E
:1043700030462EF087FD38463146F6F76DFF014690
:1043800004A8F6F73DFF079B9E4FA3F10C00B8422F
:1043900040F01482049B53F80C3C112B00F08681F2
:1043A00072B63A230CA840F8183D3146964B984710
:1043B00062B6102108A8F8F739F84FF0000C4FF05A
:1043C0001F0E11210222042384F8310084F82CC02E
:1043D00084F82DE084F82E1084F82F2084F83030F3
:1043E00004F12C082069414603681B6B98472B6831
:1043F00042F60D01586945F622320023F6F766F9B8
:1044000003AA8046814930462EF03CFD31464046A5
:10441000F6F722FF014605A8F6F7F2FE079BA3F187
:104420000C00B84240F08E8105A878492EF044FA7D
:10443000002800F0F780237A2E226FF3C303237243
:1044400005A8009204F1320104220A23FFF70AFCB6
:10445000002800F064814FF000082B6842F60D013F
:10446000586948F6E6520023F6F730F902AA814669
:10447000674906A82EF006FD06A94846F6F7ECFEA9
:1044800001463046F6F7BCFE05A831462EF061F92C
:10449000079BA3F10C00B84240F0A881069BA3F152
:1044A0000C00B84240F096812E23009305A804F139
:1044B000360104220A23FFF7D5FB002800F03681DD
:1044C0002B6842F60D0158694AF22E720023F6F766
:1044D000FDF802AA81464F4906A82EF0D3FC06A992
:1044E0004846F6F7B9FE01463046F6F789FE05A8BC
:1044F00031462EF02EF9079BA3F10C00B84240F094
:104500003981069BA3F10C00B84240F027812E238D
:10451000009305A804F13A0104220A23FFF7A2FB45
:10452000002800F0D880B8F1000F40F0D880216951
:104530002868F5F7FBF82B6818209D6A2DF0C0FE5F
:104540008046F6F729FA344A344B1068CDF81880C3
:104550008008A3FB002040092FF0C8FA30F092FA3F
:104560002FF0F8FC03462E480021C8F80440C8F894
:10457000103008F108020790089196E8030082E8DD
:104580000300C8F8143072B62B69632B04D8642179
:1045900029612846F6F7DAFCAB68EA68934200F036
:1045A000CC80069A0BB11A60AB680433AB6062B67C
:1045B00003212046F6F770FE20460021F6F76CFE38
:1045C00020460521F6F768FE2046FFF799FC059B7B
:1045D000A3F10C00B84240F0D980049BA3F10C0079
:1045E000B8423FF47AAE53F8042C511E002A43F827
:1045F000041C3FF772AE06A92EF0AAF96DE600BFC3
:10460000D8340500640A0010F11FFF1FF03F0500B9
:104610001040050038400500980100101F85EB513F
:10462000413C0100217A2A6841F0080103462172C9
:10463000506942F60D0146F66202F6F747F8014668
:104640003046F6F7DDFD05A831462EF082F8079BCF
:10465000A3F10C00B84240F0A580DDF814E05EF84C
:104660000C1C00293FF463AF3F2953D8002301F10C
:10467000FF381EF8032022F0200041381928A2F14B
:10468000300C08D9002B45D0BCF1090F03D94345A4
:1046900040D02D2A3ED101338B42EAD1581C2DF057
:1046A0000DFE0599606233F0A9FC40E73A2304F15E
:1046B0002C08009304A8414606221023FFF7D2FAE3
:1046C00000287FF48FAE0499544833F0A3F954487E
:1046D00033F0A0F90CE05348059933F09BF95048AA
:1046E00033F098F9059BA3F10C00B84240F08A80A2
:1046F000049BA3F10C00B8423FF4EFAD53F8042C37
:10470000511E002A43F8041C3FF7E7AD31462EF056
:104710001FF9E2E57146444833F07CF907E7434866
:10472000059933F077F94FF0010896E6404805996E
:1047300033F070F94FF00108C2E6281D06A9FFF713
:104740007BFD34E753F8042C511E002A43F8041C67
:104750003FF76AAE06A92EF0FBF865E653F8042C85
:10476000511E002A43F8041C3FF7D1AE31462EF00B
:10477000EFF8CCE653F8042C511E002A43F8041C31
:104780003FF7BFAE03A92EF0E3F8BAE653F8042CC6
:10479000511E002A43F8041C3FF71FAF06A92EF054
:1047A000D7F81AE753F8042C511E002A43F8041CCA
:1047B0003FF753AF06A92EF0CBF84EE753F8042C81
:1047C000511E002A43F8041C3FF7E4AD06A92EF061
:1047D000BFF8DFE553F8042C511E002A43F8041CEF
:1047E0003FF762AE31462EF0B3F85DE653F8042C85
:1047F000511E002A43F8041C3FF750AE03A92EF0C7
:10480000A7F84BE653F8042C511E002A43F8041C69
:104810003FF76EAF31462EF09BF869E7A83F0500E1
:10482000C43F0500444005005C400500F83F05001A
:104830002040050008B50C202DF042FD002242600A
:104840000260826008BD00BF38B504460C200D46EA
:104850002DF036FD6368002280E82C0003B118605B
:10486000236860601BB1A3680133A36038BDA368EF
:1048700020600133A36038BD8068704738B5036895
:1048800002468068596801389D689060186871B167
:1048900008601C682CB118466160F6F701FA2846DA
:1048A00038BD18465160F6F7FBF9284638BD106050
:1048B000EFE700BF10B5044618B90DE0FFF7DEFFC3
:1048C00038B9A3682046002BF8DCBDE81040F6F7A5
:1048D000E7B928F06DFCF4E710BD00BF08B5FFF79D
:1048E000CDFF08BD38B5084D2C680CB1204638BD49
:1048F00010202DF0E5FC054A054B046044608460FF
:1049000028601060C36038BD4805001044050010E1
:1049100010030010F8B504460846154633F076FB40
:104920000746CDB12E4610202DF0CAFC626800214A
:104930008760C66080E8060002B11060226860608F
:1049400042B1A0680130A0601DB12B6901332B6119
:10495000A068F8BD2060F4E7E668E4E7024B0A4689
:1049600001461868FFF7D6BF4405001070B583688C
:1049700084B0044613B9184604B070BD0068013B0A
:10498000011D62C9A3600368002930D00B60036871
:10499000002B2AD05960F6F783F91B4B2846039366
:1049A00033F04FFB2946024603A82EF07DF8284637
:1049B000029628F0FDFB154B02AA18680121F4F7B6
:1049C000BBFEE3680298984206D0036800215B6949
:1049D0009847029800F0A4F8039B0D4AA3F10C003D
:1049E000904206D1012004B070BD6160D3E723601E
:1049F000CDE753F8042C511E002A43F8041CF1DCC7
:104A000001A92DF0A5FFEDE7700A0010E4020010E7
:104A1000640A0010084A10B512680446074B106873
:104A20002360436822469B68054904309847054B3C
:104A30002046236010BD00BFE4020010B84005000E
:104A400074400500A02D0500094A10B512680446FF
:104A5000084B106823604368224607499B6804306E
:104A60009847064B20462360F6F71AF9204610BDFA
:104A7000E4020010B840050074400500A02D0500B8
:104A8000F8B5037B04460D46A3B90846C1B133F01F
:104A9000D8FA0D4F064663682846A1689847431C1C
:104AA0000AD008B13046F8BD024603213868F4F751
:104AB00043FEF0E70020F8BD012330462373F8BD24
:104AC0006368A1689847F8BDE402001070B50A4C0D
:104AD0000A4B256804462868236043680E4615463D
:104AE0009B68224606490430984700236660A5600B
:104AF00023732361204670BDE4020010B840050016
:104B00009040050002690121002A08B5017300DD0B
:104B100008BD0028FCD003685B68984708BD00BF4B
:104B20000269017B013A08B5026109B1002A00DD82
:104B300008BD0028FCD003685B68984708BD00BF2B
:104B400070B5064614200D462DF0BAFB094B0A4AF3
:104B50001B680446026018682246416804308B686E
:104B60000649984700236660A560237323612046A9
:104B700070BD00BFE4020010B84005009040050081
:104B800002690121002A08B5017300DD08BD002873
:104B9000FCD003685B68984708BD00BF4068704759
:104BA00081607047704700BF4FF0A043D3F81401F5
:104BB000D3F81831C01A18BF01207047A0F10400C3
:104BC000FFF7F2BF4FF0A04210B4094BD2F81841E2
:104BD000D2F818014FF4167202FB043200F59670F9
:104BE00053F830005DF8044BC0F30A000A607047C8
:104BF00008040820A0F10400FFF7E4BF4FF0A04232
:104C0000D2F82831D2F824110133D2F82C018B428A
:104C100088BF0023C01A18BF01207047A0F104000C
:104C2000FFF7ECBF4FF0A043D3F8281110B4501E8B
:104C30000E4CC0F30A0001F5977104EBC10140F07E
:104C40007040C1F8A409D3F82811D3F824410131E8
:104C5000D3F82C01A14288BF0021814216BF104623
:104C60000020C3F828115DF8044B704708040820A1
:104C7000A0F10400FFF7D6BF4FF0A043D3F82831CE
:104C8000034A03F5977302EBC303D3F8A0097047F7
:104C900008040820A0F10400FFF7EEBF021D8A42BD
:104CA00008B501D0002008BD03685B6C984708BDBB
:104CB000A0F10400FFF7F2BF08467047A0F104001E
:104CC000FFF7FABF104810B4104B00F51A64091B27
:104CD000A3FB01439B09032B13DC4FF4167404FB65
:104CE000131171B903F5977300EBC300D0F8A41941
:104CF000C2F30A0221F4FF6121F007011143C0F859
:104D0000A4195DF8044B704708040820B5814E1BB8
:104D1000A0F10400FFF7D6BFF8B505680446ED6BB7
:104D200017461E46A84728B12368394632461B6CF1
:104D300020469847F8BD00BFA0F10400FFF7ECBF84
:104D400018467047A0F10400FFF7FABF0B684361F3
:104D50008B880383704700BFA0F10400FFF7F6BF04
:104D600038B501224FF0A04340F4807199621D468E
:104D70005A624FF4A02201E0013A08D06B6B4FF069
:104D8000A04413F00103F7D16362206B38BD0146E4
:104D9000024832F03FFE4FF0FF3038BDB041050011
:104DA00038B50A464FF0A04340F4807199621D4621
:104DB000DA624FF4A02401E0013C05D06B6B13F0E4
:104DC0000103F9D1184638BD0146034832F022FEEE
:104DD0004FF0FF3038BD00BFC841050010B5054B8E
:104DE000044603F108026C3380E80C00F6F73EFA43
:104DF000204610BD1041050010B5074B044603F1D5
:104E000008026C3380E80C00F6F730FA2046F5F71C
:104E100047FF204610BD00BF10410500F8B504460D
:104E2000F6F734FA1E4B1F4A03F164011E4D23604E
:104E3000616002F5166013460021C3F8802902F56F
:104E400016728242C3F88459C3F86019C3F8641912
:104E500003F10803F1D1154B154F03F65C1103F56F
:104E600016661A460020C2F8703903F51673B3426D
:104E7000C2F874794FF0000541F8040F02F10802FE
:104E8000F1D1052028F08EF90A4A03460A4EA060A7
:104E9000A57692E803001860197134602046F8BDC9
:104EA000184105000804082057020080A80D0820BA
:104EB000570200F0144205004C05001030B50446BE
:104EC00085B00120FFF74CFF00F02403242B0ED007
:104ED00010F0040001D1A37E0BB905B030BDA0765F
:104EE000A168244805B0BDE8304032F093BDA37EF0
:104EF000002BEDD10123A3761F20FFF731FFA1681E
:104F000005461D4832F086FDC5F38203013B052BA3
:104F10002BD8DFE803F026222A2A1E03174832F096
:104F20002DFE4FF0A040816C826C436C456C046C8C
:104F3000006CC5F30725E4B2C0F307200290C9B2A4
:104F4000C2F30722DBB2009501940D4832F062FDF6
:104F5000C3E70C4832F012FEE3E70B4832F00EFED6
:104F6000DFE70A4832F00AFEDBE72946084832F05C
:104F700051FDD6E7D04205001C42050068420500FD
:104F80009C42050040420500544205002C420500A9
:104F90007C420500FFF792BF80B588B000AF786013
:104FA0004FF080400121F1F725FF4FF0A0434FF46F
:104FB0004F421A604FF0A0433822C3F800214FF44B
:104FC0008073FB6002E0FB68013BFB60FB68002B29
:104FD0000CBF00230123DBB2002BF4D14FF0A04320
:104FE00002221A604FF0A04331225A604FF0A043D2
:104FF0004FF4C0625A616D4B1A686D4BA3FB0213EC
:105000001B0DBB610023FB610BE06A4AFB69134483
:105010001B781A46BB699A4200DB06E0FB69013344
:10502000FB610722FB699A42EFDCFB690133FB61FC
:105030004FF0A043FA6902F00F02920042F40042DE
:105040001A624FF0A0434FF0A042126A22F40042CD
:105050001A624FF0A04343F20F721A614FF0A0435F
:105060001222DA604FF0A0434FF40072C3F800211F
:105070004FF0A0434FF400629A614FF48073FB60DD
:1050800002E0FB68013BFB60FB68002B0CBF0023C8
:105090000123DBB2002BF4D14FF0A0434FF4807218
:1050A0009A6100204FF40041FFF77AFE4FF480131D
:1050B000FB6113E00020FFF753FE78617B6903F486
:1050C0000843002B00D10CE0FB69002B03D13A48C8
:1050D00032F054FD67E0FB69013BFB61FB69002B8B
:1050E000E8D100204FF44051FFF75AFE7B6814339B
:1050F0003B613B695B791A023B691B791A434FF0AC
:10510000A0431A643B69DB781A023B699B781A4317
:105110004FF0A0435A643B695B781A023B691B78E5
:105120001A434FF0A0439A644FF0A043234AC3F8B8
:1051300008214FF0A043224AC3F80C214FF0A043AE
:105140000322C3F810214FF0A0431E4AC3F81C21CC
:105150004FF0A0431C4AC3F820214FF0A043032284
:10516000C3F824214FF0A0432222C3F800224FF0BD
:10517000A0438822C3F8E42F4FF0A0434FF6FF72FC
:10518000C3F8E82F4FF0A04340F24362C3F8002178
:105190004FF0A0434FF0A042126842F001021A60A3
:1051A0000A4832F0EBFC2037BD4680BD9801001064
:1051B0006BCA5F6B04410500D8400500880D0820CC
:1051C000680D08201817082008170820EC40050073
:1051D000104B10B510499C68104A2143996099689A
:1051E00004460A409A60DA680D4842F00502DA6027
:1051F000DA6822F00A02DA6032F0C0FC2046FFF7DB
:10520000CBFE084832F0BAFC20460421BDE810402D
:10521000F6F742B800C0024005011550F5FDD55F14
:10522000E0420500EC420500F8B5036804465B6BFC
:105230000E461546984710B900242046F8BD23684D
:105240002046DB6B984704460028F5D04FF0A0437A
:10525000D3F818E1144A0EF5967352F833102B6800
:10526000C1F30A0701379F4216DC4FF4167101FBA8
:105270000E2130463A4632F0F6FA2F604FF0A04247
:10528000D2F81831D2F8101101338B4288BF0023B5
:10529000C2F818312046F8BD3A460448002432F0DE
:1052A000B9FB2C60EAE700BF08040820F4420500BF
:1052B000704700BF002070470020704700207047F3
:1052C000A0F10800FAE700BF00207047A0F1080035
:1052D000FAE700BF00207047A0F10800FAE700BF1E
:1052E00000207047A0F10800FAE700BF00207047D7
:1052F000002070470023022280F8542080F85530A7
:1053000080F856300120704701870120704700BFA8
:10531000A0F10400FFF7F8BF90F85430042B02D03E
:10532000416301207047406B0B1A58425841704747
:105330002DE9F84F454BC66C8364731C834659D0E6
:10534000002E4FDD0025DBF83400DFF808A1404FC8
:1053500027E0C5F1400E5FFA8EFEB645C4EB0202AF
:10536000C8BF5FFA86FE5FFA82FC3848E64534BF64
:10537000F046E04621442844424632F074FADBF815
:105380003400444450F82920E4B212784544A24243
:10539000C8EB06063C70EDB20BD93F2D22D8002E8B
:1053A00020DD9AF800903C7850F829100A78A24243
:1053B000CFD8494602E05278032A0CD14B1CDBB20D
:1053C00050F823201946002AF5D18AF800303A70A7
:1053D0001046BDE8F88F8AF800303F2D4FF00003EB
:1053E0003B70DCD9DBF84C00B042D4BF0020012078
:1053F000BDE8F88F406B0268002AE9D0002304E082
:1054000050F8042F0133002AE2D051780229F7D155
:10541000BBF84040517904F00F04A14203D00129A8
:10542000EED1002CECD15688BBF84420CBF84C6070
:10543000964202DDCBF84C201646DFF818A0044F48
:1054400000228AF800303A707AE700BF5405001055
:1054500094050010500500100B78DB0913700B78D1
:10546000C3F3411353700B7803F01F0393704B7811
:10547000D370C8788B7843EA0023938048790B79FE
:1054800043EA0023D380C8798B7943EA0023138150
:10549000704700BF70B590F8503004460BB1002043
:1054A00070BD816C00F048FDE36C9842F7DCA26CA3
:1054B0001D1A0244E564A26495B994F8523043B1D0
:1054C000214651F83C6B034676692046B04784F884
:1054D0005250002120460A4600F032FD012070BDE6
:1054E000204600F027FD012070BD00BF10B5044626
:1054F000FFF7D0FF00B110BD2046BDE8104000F01E
:1055000077BD00BF70B5C56C04465DB990F85130E9
:10551000002B32D194F8523053B9204600F00AFDE6
:10552000012070BD90F85060012E11D0002070BD98
:10553000214651F83C3B00225D6920461346A847AE
:105540000023204684F8523000F0F4FC012070BDA6
:10555000402D28BF40252A46816C00F0F1FCE36B0A
:10556000E26C03F0FF23521BB3F1C06FE2640FD073
:10557000A36C01201D44A56470BD29462A4600F095
:10558000DFFC94F8523084F85150002BC5D0CFE79F
:10559000B4F840301B12022BEAD12046FFF7C8FEB8
:1055A000304670BD10B50446FFF7ACFF00B110BD2A
:1055B0002046BDE8104000F01BBD00BF90F8401031
:1055C00010B5044680F8551061B10368DB6B98474D
:1055D00000B910BD204600F047FC042384F8543085
:1055E000012010BD00F060FC032384F8543001203A
:1055F00010BD00BF08B590F85430042B02D0B0F8AD
:10560000423093B990F83E30022B0ED1B0F84030C2
:105610005BB9B0F8423003F00F01C3F3C01303EBE2
:10562000410100F0C9FC012008BD002008BD00BFF9
:1056300008B590F85430042B02D0B0F8423033B99A
:1056400090F83E30022B02D1B0F840300BB1002070
:1056500008BD90F8421000F0CFFC012008BD00BF4B
:1056600090F8543010B5042B044602D0B0F8423004
:10567000B3B994F83E30012B18D013D3022B0FD1BD
:10568000204694F8421000F0CDFC0B4B90B1012263
:105690001A800120022284F85000A364E26410BD45
:1056A000002010BD044B01221A80F2E7024B0022B9
:1056B0001A80EEE71880ECE79605001000F0ACBB0E
:1056C00000F0D0BB2DE9F00F012A9DF820B03ED0AC
:1056D000022A40D0456B4FEA810C55F821406544C1
:1056E00084B3A2F102095FFA89F94FF0010A0AFABC
:1056F00009FAC1EB81780AF00D0A4FEA8808002701
:1057000008E0B2420BD0043508EB050050F80C401D
:105710000131BCB16678022EF3D10027F3E7B9F16D
:10572000030F03D8BAF1000F00D0A7789F4202D030
:105730000137FFB2E7E7042A02D1E0785845F7D1F4
:10574000084601E04FF0FF30BDE8F00F7047002041
:10575000BDE8F00F70470120BDE8F00F704700BFB3
:1057600070B5B0F8403082B000251E0A324603F012
:105770000F03009529460446FFF7A4FF00280DDB20
:10578000022E0ED0636B53F820301A78A364E264C3
:105790000125284684F8505002B070BD284602B05A
:1057A00070BD4FF0FF33E3642046FFF7C1FDEFE724
:1057B00010B590F83D3004467BB990F83F300B2B84
:1057C0000BD8DFE803F00C100A140A18240A28305A
:1057D000063490F85430042B41D0002010BDBDE8B1
:1057E0001040FFF73DBFBDE81040FFF721BFBDE807
:1057F0001040FFF7FFBE94F8401000F073FBB4F8C0
:1058000040303BBB022384F85430012010BDBDE87A
:105810001040FFF7A5BF00F15503012084F85000A8
:10582000A364E06410BDBDE81040FFF7C7BE036885
:10583000B4F842101B6C94F8402098470028CCD054
:10584000B4F84030B4F8422084F89A30A4F8982094
:10585000012010BD032384F85430012010BDB0F89E
:10586000982000F19A03012084F85000A4F8422007
:10587000A364E06410BD00BF70B500F15705044695
:1058800000F13C06294600F051FB294632462046ED
:10589000FFF7E2FD00232268A56484F85030126906
:1058A0003146E36484F8513084F852302046904702
:1058B000E8B1B4F8443073B194F83C20012A94F86C
:1058C000502010D08AB9E26C9A420ED1204600F0E6
:1058D00031FB012070BDE16C39B920460A4600F069
:1058E0002FFB012070BD012A08D0002070BD20468A
:1058F000FFF75EFF0028DCD1002070BDE16C99420B
:1059000005DDE3642046FFF7FDFD012070BDF9DAF7
:105910008B0608BF84F851202046FFF7F3FD0120D5
:1059200070BD00BF10B50446FFF7A6FF00B110BD63
:105930002046BDE8104000F05BBB00BF38B5044610
:1059400000F01EFA094B002203F1080503F1540090
:105950000121603384F8552060602560A36084F8DD
:10596000541084F85620204638BD00BF3843050047
:1059700070B5144606460D46012200F061FB304624
:105980002946224600F0E0FA431E5842584170BDB5
:1059900070B5049C0546A3420E4603D890F85440C7
:1059A000042C01D0002070BD00F074FB0128F9D157
:1059B0002846314600F0F4FAD0F1010038BF00204B
:1059C00070BD00BFF8B5044690F854000F46042897
:1059D00016461D4605D00020F8BD94F85430042B1F
:1059E00007D12046394632462B4600F0AFFA01284F
:1059F000F3D0D0F1010038BF0020F8BD002070477F
:105A000000207047A0F10400FAE700BF704700BF14
:105A1000704700BF704700BF0D4B0E4A1021C3F8FE
:105A200008121946C3F81022D1F80032084ADB06E2
:105A3000FAD5000440F480701023C2F808321146F1
:105A4000C2F81002D1F80032DB06FBD5704700BF68
:105A500000C000500005FE000D4B0E4A1021C3F897
:105A600008121946C3F81022D1F80032084ADB06A2
:105A7000FAD5000440F480701023C2F808321146B1
:105A8000C2F81002D1F80032DB06FBD5704700BF28
:105A900000C000500005F30000F00F03C00940EA09
:105AA000430000040F4B102140F4A062C3F8081219
:105AB0001946C3F81022D1F800320A4ADB06FAD59B
:105AC00040F400702023C2F808321146C2F81002D8
:105AD000D1F80032034A9B06FAD5D2F81402C0B2BC
:105AE000704700BF00C0005000F00F02C00940EA3C
:105AF000420240320E4B1204102042F4A062C3F85E
:105B000008021846C3F81022D0F80032084ADB0613
:105B1000FAD5090441F480711023C2F80832104606
:105B2000C2F81012D0F80032DB06FBD5704700BF78
:105B300000C00050164B174A1021C3F8081219462E
:105B4000C3F81022D1F80032114ADB06FAD5124B05
:105B50002021C2F808121146C2F81032D1F80032E2
:105B60000B4A9806FAD5D2F814020B4B2021C2F842
:105B70000812C0B21146C2F81032D1F80032044AFD
:105B80009B06FAD5D2F81432DBB240EA0320704704
:105B900000C000500005F5000002F5000F4B104A50
:105BA0001021C3F808121946C3F81022D1F80032A8
:105BB0000A4AD806FAD50B4B2021C2F80812114622
:105BC000C2F81032D1F80032044A9B06FAD5D2F856
:105BD000140200F0FE00FFF71FBF00BF00C000501E
:105BE0000005FE000002FE0070B5064600F00F0042
:105BF000194B800040F00200C3F82802C3F82422A9
:105C0000D3F82822900710D58A78C8780D78120426
